:020000020000FC
:080000000C9499040C9400001B
:100008000C9400000C9400000C9400000C94000068
:100018000C9400000C9400000C9400000C94000058
:100028000C9400000C9400000C94FA7E0C940000D0
:100038000C9400000C9400000C9488350C9400007B
:100048000C9400000C9400000C9400000C94E5B88B
:100058000C9413B90C9400000C9400000C942036F6
:100068000C9400000C9400000C9400000C94000008
:100078000C9400000C9400000C9400000C940000F8
:100088000C9400000C9400000C9400000000000088
:100098000102030400060705010006FF050402FF2C
:1000A80009080CFF0AFF0F0E0106080705020403E2
:1000B8000C0B100A090D0F0E0406080203010705B0
:1000C8000C10090F0D0B0E0A0101010101010101BC
:1000D800010101010101010101FF02FF04FFFFFF0E
:1000E80003FF05FF06FF00FF0000000000000000FE
:1000F800436F4465496E466F00C9020C0800000F43
:10010800AA558A6170722020392032303236203167
:10011800383A35353A303600006701016564000029
:10012800000101010202020303030404040505059A
:1001380006060607070741424341424341424341FD
:10014800424341424341424341424341424300000A
:100158000000EF006A0290080000000000000000A4
:100168000000000000000000000000000000640023
:100178002301C602D504820F000000000000000021
:100188000000000000000000000000000000F00077
:10019800F0005402D203F60900000000000000003D
:1001A80000000000000000000000000000002A031A
:1001B800C8032105E3064D10000000000000000000
:1001C80000000000000000000000000000000E0019
:1001D8000208040A0C000000F800000043414E72B7
:1001E800783A20253033580A000043414E696E7032
:1001F8007574436E743D25752121210A0043414ED3
:100208002D25753A20300A0043414E2D25753A2098
:10021800310A0043414E2D25753A2025750A0043C1
:10022800414E2025750044656C61792074696D65BF
:10023800722025750000466163746F7279446566A3
:1002480061756C740A004850383434330045727252
:100258004C6F67506F733D25752C204E6F3D25758B
:100268000A004572723A2025752025750A00257501
:10027800204F66660A002575204F6E0A00466C619D
:1002880073682074696D657220257500485038348C
:1002980034330043666753756D3D253034580A0082
:1002A80020557064617465640A00485038343433EA
:1002B800207665722E2025752E25752E25752061D0
:1002C800707220203920323032362031383A3535B4
:1002D8003A30360A0053657269616C3A2025750A0E
:1002E80000596561723A203230253032752C20571A
:1002F80065656B3A2025750A004857207665723A7D
:100308002025632E25632C204F7074696F6E733A15
:1003180020253032580A00436C6F636B3A20253031
:10032800386C580A0043666743686B53756D3A200A
:100338002530345820004F4B0A0020457272210A9C
:10034800004366675665724572723A202575202803
:10035800257529210A004545507665724572723A1D
:100368002025752028257529210A00526573746F88
:100378007265436E743D25752025752025750A0024
:10038800446174614572723D2530325820253032FF
:10039800580A004850383434330A00004144436D49
:1003A800696E4572726F725B25755D3D25752121F9
:1003B800210A0000496E707574733A002025753D56
:1003C800257500496E2D313A2025750A00496E2D94
:1003D800323A2025750A00496E2D333A2025750AD0
:1003E80000496E2D343A2025750A00496E2D257571
:1003F8003A2025750A00496E412D2575204F6666FD
:100408003A2025755B6D565D0A00496E412D2575AC
:10041800204F6E3A2025755B6D565D0A005377694B
:1004280074636820257500416E616C6F6720332EF8
:10043800257500416E616C6F6720342E25750000AC
:100448004B65795061643D00426C696E6B3A2530AA
:10045800325820253032580A004772617968696C31
:100468006C2043414E6F70656E0A0047726179686F
:10047800696C6C204A313333390A004850393634B4
:10048800320A004E6F6E650A00004B657950616450
:100498002E436F6E6E2025750A004B657950616496
:1004A8002E4469736F6E6E6E2025750A00004F75B5
:1004B800745075736850756C6C3A2025750A004F36
:1004C800757448696768536964654F6E6C793A203A
:1004D80025750A0043202532753A202534750043D6
:1004E800616C69627261746520004F4B0A006F7518
:1004F80074707574202575206661696C65642121A6
:10050800210A002532753A2025352E32665B415D79
:100518000A002532753A204E6F206665656462616F
:10052800636B2C204F75742D25750A002532753A9A
:1005380020466565646261636B206572726F722C18
:10054800204F75742D25750A004F757470757420C9
:100558007465737400426174742063616C6962200D
:10056800203A20257500416E616C6F672063616CCD
:1005780069623A20333D25752C20343D25750043AA
:10058800616C6962726174696F6E4D61736B3A2058
:1005980025580A0020202532753A202533752C204D
:1005A8002534692C202534692C202534692C2025F4
:1005B80034690042617474657279206661696C659A
:1005C800642121210A00416E616C6F6720666169B0
:1005D8006C65642121210A00206E6F7420636F6DA1
:1005E800706C657465642121210A004F757452731B
:1005F800744572725B25755D0A004F75742D2575FB
:100608003A204F6E0A004F75742D25753A205325F0
:10061800752D3E25752C204F6E3D25752C20536574
:10062800743D25750A004144433A002025753D254F
:1006380075002020426174743D2575004C6F774227
:100648006174744F66663D2025750A004C6F7742C9
:100658006174744F6E3D20257530300A0042617414
:1006680074657279536B697046423A20252E31665B
:100678005B565D0A00426174746572794642204F88
:100688004B3A20252E31665B565D0A002020416ECC
:10069800612D333D202575002020416E612D343DAC
:1006A800202575004F75742D25753A2025750A008B
:1006B8004F757420257520474E442D31210A004F6F
:1006C800757420257520474E442D32210A004F7538
:1006D80074202575206C696D6974210A004F757442
:1006E800412D25753A205325752D3E25752C204F13
:1006F8006E3D25752C205365743D25750A004F7590
:1007080074707574733A0A002534753A2046423D70
:100718002575204144433D25752025755B6D415D58
:100728000A0052657365744572726F720A004F75DC
:1007380074707574202575004F75742D25753A20D1
:100748005325752C204F6E3D25752025632C2025BB
:1007580075305B6D415D0A004F7574707574206764
:10076800726F757020257500506F776572446F77CA
:100778006E0A0057616B6555703A2025750A0000AE
:100788004F7574412D25753A205325752D3E2575D5
:100798002C204F6E3D25750A000043616C69622E5E
:1007A8002073746172742025755B416D705D0A0059
:1007B80054657374206F75740A0043616C69622E06
:1007C80020626174740A0043616C696220616E6121
:1007D80028352C3056207265662E290A0043616C34
:1007E80069623F00633000633100633300633600A1
:1007F80063323000636200636100746573746F75FF
:10080800740050617373776F72643F0050573A20D9
:10081800272573270A0050573A204E6F6E650A0045
:10082800505772657365740050577265736574200C
:100838002D204F4B0A004144433F00496E707574A8
:100848003F004C6F61643F00485073746174757366
:100858003F0052526573746F7265005252204F4BBD
:100868000A005265736574005365744F75742025CA
:10087800753D2025750A005265736574206572728E
:100888006F720A004F7074696F6E3A2025303258C3
:100898000A0052657365740A000053657120256368
:1008A8003A20004F66660A0025630A005365717591
:1008B800656E63652025750020204F4B0A002020B7
:1008C8004661696C65642121210A000056696E2D14
:1008D80025753A2025750A005669727475616C2071
:1008E8002575000057697065723A205325752D3EAD
:1008F8005325750A000001002D4E414E00494E4611
:1009080000002D4E414E000001000200DE010000F3
:100918000700BC034E0200000700C3039402000056
:100928000100B90DFE0800000000F894EE27EFBBA7
:10093800F1E0F5BFE5BFE0937400E09375008DE04A
:10094800A2E0BB27ED938A95E9F780EF9FE0A0E04E
:10095800B1E0ED930197E9F7E0E1F9E0D0E0DBBF22
:1009680087919791009781F0A791B7910790179079
:10097800C791D791BF01DBB7F001CBBF07900D92AC
:100988000197E1F7FB01EBCFE0E0EEBBEFEEEDBF47
:10099800E0E1EEBFCCEBD3E00C9438330E948FCA71
:1009A800AD014093D2035093D303A5E2B1E00E9476
:1009B80086CCE07111F0E1E001C0E0E0AFECB3E01B
:1009C800E170EE0F0E2EEC91ED7FE029EC93A6E797
:1009D800B2E00E9486CCE093D103A7E7B2E00E9480
:1009E80086CCE0935C04A091D103A13010F0AD3027
:1009F80008F004C0E091CF03E46003C0E091CF03A6
:100A0800EB7FE093CF03E1E0E093D800FA01E4360E
:100A1800A0E0FA0741F4E2E1E093E200ECE0E093C1
:100A2800E300E7E335C0ED37A0E0FA0741F4EEE074
:100A3800E093E200ECE0E093E300E7E329C0E83C60
:100A4800A0E0FA0741F4E8E0E093E200ECE0E0938C
:100A5800E300E7E31DC0EA3FA0E0FA0741F4E6E05F
:100A6800E093E200ECE0E093E300E7E311C0E43F49
:100A7800A1E0FA0711F4E6E005C0E83EA3E0FA07B2
:100A880049F4E2E0E093E200E4E0E093E300E3E12C
:100A9800E093E40010E1103F88F41093ED002EEE8F
:100AA80030E0E8EFF0E02E173F0730F4D901E0E03E
:100AB800EC932F5F3F4FF5CF105FEDCFE091D8005B
:100AC800E260E093D80010E4103FA0F41093ED002A
:100AD8002EEE30E0E8EFF0E02E173F0730F4D901B2
:100AE800E0E0EC932F5F3F4FF5CFE8E8E093EF00AD
:100AF800105FEACF0E9496CA2696089564970E94CE
:100B08008FCAE091D003E03009F414C2E17089F093
:100B1800E0E0E093ED00E091EE00E17551F0E09146
:100B2800D003EE7FE093D003E0E0E093EE00E093A3
:100B3800EF00E091D003E27089F0E0E1E093ED008E
:100B4800E091EE00E17551F0E091D003ED7FE09384
:100B5800D003E0E0E093EE00E093EF00E091D003F3
:100B6800E47089F0E0E2E093ED00E091EE00E175D9
:100B780051F0E091D003EB7FE093D003E0E0E09305
:100B8800EE00E093EF00E091D003E87089F0E0E335
:100B9800E093ED00E091EE00E17551F0E091D003B3
:100BA800E77FE093D003E0E0E093EE00E093EF000E
:100BB800A091D003AF3009F4BDC1A0915604E091D3
:100BC8005704EA1709F4B6C1A4EDB3E0E09156045E
:100BD800F0E0BD01ADE0B0E00E9444CBDB01AE0F18
:100BE800BF1FEC91E071B1F041E0A4EDB3E0E091FA
:100BF8005604F0E0BD01ADE0B0E00E9444CBDB015B
:100C0800AE0FBF1F11960E9401CCEB8BFC8B6D8B36
:100C18007E8B13C040E0A4EDB3E0E0915604F0E011
:100C2800BD01ADE0B0E00E9444CBDB01AE0FBF1FB9
:100C38001196ED91FD91EF8BF88FA4EDB3E0E09163
:100C48005604F0E0BD01ADE0B0E00E9444CBDB010A
:100C5800AE0FBF1FEC91EF700E2F098F403019F0C7
:100C6800E98DE061E98FE091D003E17009F051C0AE
:100C7800E0E0E093ED00E98DE093EF004030D1F043
:100C8800EB89EE0FEE0FEE0FE093F000AB89BC8915
:100C9800E5E00E94CACAE093F100AB89BC898D895E
:100CA8009E89EDE00E94F2CAE093F200E5E10E941D
:100CB800F2CA0AC0EF89E295E07FEE0FE093F200F6
:100CC800EF89F88D0E941DCBE093F30010E0101718
:100CD800B0F4A4EDB3E0E0915604F0E0BD01ADE05E
:100CE800B0E00E9444CBDB01AE0FBF1F1596EE2784
:100CF800A10FBE1FEC91E093FA001F5FE8CFE98DCA
:100D0800E05CE093EF00E091D003E160E093D00372
:100D180003C1E091D003E27009F051C0E0E1E09333
:100D2800ED00E98DE093EF004030D1F0EB89EE0F54
:100D3800EE0FEE0FE093F000AB89BC89E5E00E946E
:100D4800CACAE093F100AB89BC898D899E89EDE020
:100D58000E94F2CAE093F200E5E10E94F2CA0AC0DA
:100D6800EF89E295E07FEE0FE093F200EF89F88DCE
:100D78000E941DCBE093F30010E01017B0F4A4ED2F
:100D8800B3E0E0915604F0E0BD01ADE0B0E00E94B0
:100D980044CBDB01AE0FBF1F1596EE27A10FBE1F78
:100DA800EC91E093FA001F5FE8CFE98DE05CE093F7
:100DB800EF00E091D003E260E093D003ADC0E09192
:100DC800D003E47009F051C0E0E2E093ED00E98D52
:100DD800E093EF004030D1F0EB89EE0FEE0FEE0F0D
:100DE800E093F000AB89BC89E5E00E94CACAE093B1
:100DF800F100AB89BC898D899E89EDE00E94F2CA19
:100E0800E093F200E5E10E94F2CA0AC0EF89E29598
:100E1800E07FEE0FE093F200EF89F88D0E941DCB82
:100E2800E093F30010E01017B0F4A4EDB3E0E09104
:100E38005604F0E0BD01ADE0B0E00E9444CBDB0118
:100E4800AE0FBF1F1596EE27A10FBE1FEC91E093C2
:100E5800FA001F5FE8CFE98DE05CE093EF00E091D6
:100E6800D003E460E093D00357C0E091D003E8706A
:100E780009F051C0E0E3E093ED00E98DE093EF0065
:100E88004030D1F0EB89EE0FEE0FEE0FE093F0005B
:100E9800AB89BC89E5E00E94CACAE093F100AB893E
:100EA800BC898D899E89EDE00E94F2CAE093F20028
:100EB800E5E10E94F2CA0AC0EF89E295E07FEE0FF1
:100EC800E093F200EF89F88D0E941DCBE093F300C8
:100ED80010E01017B0F4A4EDB3E0E0915604F0E090
:100EE800BD01ADE0B0E00E9444CBDB01AE0FBF1FF7
:100EF8001596EE27A10FBE1FEC91E093FA001F5F35
:100F0800E8CFE98DE05CE093EF00E091D003E86082
:100F1800E093D00301C00EC0E0915604EF5FE09368
:100F28005604E150A0915604AA3018F0E0E0E0938E
:100F3800560443CEE0E05E2F2E2F30E4303F08F019
:100F480032C13093ED00E091EE00E07209F41EC169
:100F5800E091EF00EF700E2EEE81E07FE029EE8346
:100F6800EF70E93020F0EE81E07FE860EE83E091F9
:100F7800EF00E07109F46DC0E091F300FF276627E8
:100F88007727EB8BFC8B6D8B7E8BAB89BC898D892E
:100F98009E89E8E00E94DBCAEB8BFC8B6D8B7E8B15
:100FA800E091F200AB89BC898D899E89FF2766276D
:100FB8007727EA2BFB2B682B792BEB8BFC8B6D8B24
:100FC8007E8BAB89BC898D899E89E8E00E94DBCA4B
:100FD800EB8BFC8B6D8B7E8BE091F100AB89BC8930
:100FE8008D899E89FF2766277727EA2BFB2B682B9D
:100FF800792BEB8BFC8B6D8B7E8BAB89BC898D89B8
:101008009E89E5E00E94DBCAEB8BFC8B6D8B7E8BA7
:10101800E091F000F0E00E9414CBAB89BC898D8987
:101028009E896F2F660F660B762FEA2BFB2B682B9A
:10103800792BEB8BFC8B6D8B7E8BEE81E061EE83E5
:10104800EB89FC896D897E89EF83F88769877A87C0
:101058001DC0E091F300F0E0EF8BF88F0E940BCBFE
:10106800EF8BF88FE091F200F0E0F595E7950E949C
:1010780012CBAF89B88DEA2BFB2BEF8BF88FEE8163
:10108800EF7EEE83EF89F88DEF83F88710E0EE812D
:10109800EF701E1758F4E12FF0E0DE011B96AE0F3B
:1010A800BF1FE091FA00EC931F5FF1CF2F5FE09133
:1010B800CF03E17081F0E4EEF1E060E070E00E94BF
:1010C80018CCEB8DFC8D662777270E9418CC84E01E
:1010D8000E9416CA2896A091D103A03069F0AF8962
:1010E800B88D109749F4EE81EF70E23028F0E09166
:1010F800D103AC85EA1709F017C0EB85F0E0E130C1
:10110800A0E0FA0721F4E091CF03EB7F0BC0E230B7
:10111800A0E0FA0721F0E038A0E0FA0729F4E0910E
:10112800CF03E460E093CF03E091CF03E47069F567
:10113800DE0116960E94C419E0918C09E27021F034
:10114800DE0116960E942282E091AB07F0E0E130C2
:10115800A0E0FA0729F4DE0116960E94844615C01D
:10116800E230A0E0FA0721F0E330A0E0FA0729F422
:10117800DE0116960E94745208C0E430A0E0FA0717
:1011880021F4DE0116960E94635A05C0E091EE0034
:10119800EE7039F05F5FE0E0E093EE00E0E8E093A6
:1011A800EF00305FCBCE222319F4552309F44DC04C
:1011B800213078F0E091CE03E03041F4E091E50889
:1011C800E160E093E508E0E0E093E208EEE1E09317
:1011D800CE03A0915804B0915904A13FEFEFBE0788
:1011E80040F4A0915A04B0915B04A13FEFEFBE0711
:1011F80060F1E0915804F0915904F695E795E09371
:101208005804F0935904E0915A04F0915B04F69560
:10121800E795E0935A04F0935B04A0915804B091C9
:101228005904E22FF0E0EA0FFB1FE0935804F09313
:101238005904A0915A04B0915B04E52FF0E0EA0F3D
:10124800FB1FE0935A04F0935B040E9496CA6A96C7
:101258000895BA93AA9324970E948FCAE091CF0366
:10126800E47009F07FC1E0916304E07821F0AA8579
:10127800BB850E94C419AA85BB85EC91EF700E2F1F
:10128800202FEC91E07151F031E0206111960E941D
:1012980001CCEE83FF836887798706C030E0AA8592
:1012A800BB8511964D915C91E091D003E17009F0F6
:1012B80047C0E0E0E093ED002093EF003030D1F03C
:1012C800EE81EE0FEE0FEE0FE093F000AE81BF81DE
:1012D800E5E00E94CACAE093F100AE81BF8188852B
:1012E8009985EDE00E94F2CAE093F200E5E10E94E0
:1012F800F2CA0CC0E0E0E093F000E42FE295E07F52
:10130800EE0FE093F200FA010E941DCBE093F30088
:1013180010E0101758F4AA85BB851596EE27A10F83
:10132800BE1FEC91E093FA001F5FF3CFE22FE05C61
:10133800E093EF00E091D003E160E093D00312C1A5
:10134800E091D003E27009F047C0E0E1E093ED00DE
:101358002093EF003030D1F0EE81EE0FEE0FEE0F5C
:10136800E093F000AE81BF81E5E00E94CACAE09335
:10137800F100AE81BF8188859985EDE00E94F2CAAF
:10138800E093F200E5E10E94F2CA0CC0E0E0E093CD
:10139800F000E42FE295E07FEE0FE093F200FA010F
:1013A8000E941DCBE093F30010E0101758F4AA85B3
:1013B800BB851596EE27A10FBE1FEC91E093FA00AE
:1013C8001F5FF3CFE22FE05CE093EF00E091D003E2
:1013D800E260E093D003C6C0E091D003E47009F066
:1013E80047C0E0E2E093ED002093EF003030D1F009
:1013F800EE81EE0FEE0FEE0FE093F000AE81BF81AD
:10140800E5E00E94CACAE093F100AE81BF818885F9
:101418009985EDE00E94F2CAE093F200E5E10E94AE
:10142800F2CA0CC0E0E0E093F000E42FE295E07F20
:10143800EE0FE093F200FA010E941DCBE093F30057
:1014480010E0101758F4AA85BB851596EE27A10F52
:10145800BE1FEC91E093FA001F5FF3CFE22FE05C30
:10146800E093EF00E091D003E460E093D0037AC00A
:10147800E091D003E87009F047C0E0E3E093ED00A5
:101488002093EF003030D1F0EE81EE0FEE0FEE0F2B
:10149800E093F000AE81BF81E5E00E94CACAE09304
:1014A800F100AE81BF8188859985EDE00E94F2CA7E
:1014B800E093F200E5E10E94F2CA0CC0E0E0E0939C
:1014C800F000E42FE295E07FEE0FE093F200FA01DE
:1014D8000E941DCBE093F30010E0101758F4AA8582
:1014E800BB851596EE27A10FBE1FEC91E093FA007D
:1014F8001F5FF3CFE22FE05CE093EF00E091D003B1
:10150800E860E093D0032EC0E0915704EF5F1E2FF0
:101518001A3008F010E0E0915604E11759F4EF5F33
:10152800E0935604E150A0915604AA3018F0E0E088
:10153800E0935604A4EDB3E0E0915704F0E0BD0158
:10154800ADE0B0E00E9444CBE60FF71FFA93EA93B0
:10155800EC85FD85FA93EA93ADE0B0E00E947CC388
:10156800109357040E9496CA2C9608951A930A93CA
:101578008D011396ED91FD91A091D203B091D30303
:10158800EA17FB0721F0F801A381B48107DAE0919B
:10159800E508E07851F4E091E508E068E093E508B3
:1015A800E1E0E093E2080E949537F801E581EF70E9
:1015B800E93018F4D80115964CDE0991199108956F
:1015C800A091CE03A13078F0E091CE03E150E093F2
:1015D800CE03E03041F4E091E508EE7FE093E508C2
:1015E800E0E0E093E20808951A93A3E5B5E00E94CD
:1015F80086CCE0939E0D11E1163048F0A8E5B5E0E1
:10160800EE27A10FBE1F0E9486CCE03009F002C071
:101618001150F2CFE12FE550E0939F0DE0E0E09309
:10162800A00DAAE6B5E00E9486CCE093A10DAFE933
:10163800B5E00E9486CCE093A20DA4EDB5E00E942F
:1016480086CCE093A30DA9E1B6E00E9486CCE09396
:10165800A40DA091A40DA13019F4E2E0E093A40D2B
:10166800E091A40DE093A50DAAE1B6E00E947ECC1E
:10167800E093A70DF093A80D6093A90D7093AA0DA0
:10168800EFEFE093A60DAEE1B6E00E9482CCE093C6
:10169800AB0DF093AC0D309719F4E0E0E093A50D95
:1016A800ABE3B1E00E947ECC30976040704011F40B
:1016B800E0E00BC0AFE3B1E00E9486CCE093AD0D53
:1016C800A091AD0DA63018F0E5E0E093AD0D10E067
:1016D8001330B0F5AFEABDE0E12FF0E0EE0FFF1FE9
:1016E800EA0FFB1F3196FF93EF93A1E2B6E0E12FDB
:1016F800F0E0BD01A5E1B0E00E9444CBDB01AE0FF4
:10170800BF1F14960E9486CCAF91BF91EC93AFEAAD
:10171800BDE0E12FF0E0EE0FFF1FAE0FBF1FEC9111
:10172800E078E560EC93AFEABDE0E12FF0E0EE0F82
:10173800FF1FAE0FBF1FEC91EF77EC931F5FC8CF71
:101748001991089561970E948FCAE0916304E0742B
:1017580021F40E9496CA67960895A091A50DA1301C
:1017680008F4ABC6E091A50DE150E093A50DEF5F3D
:10177800E091A50DE03009F0A0C6E091A40DE0933A
:10178800A50DE091A60DEF5FE093A60DE150A091A5
:10179800A60DAF3018F0E0E0E093A60DEA85E07FF3
:1017A800E860EA87FE013F96FA93EA93E0E0EA935D
:1017B800A8E0B0E00E948EC3E091A60DF0E030975B
:1017C80009F056C1E091AB0DF091AC0DE17009F450
:1017D8004BC100E0E0919307E17009F00160E091EE
:1017E8009407E17009F00260E0919507E17009F053
:1017F8000460E0919607E17009F00860E0919707AE
:10180800E17009F00061E0919807E17009F0006269
:10181800E0919907E17009F00064E0919A07E1709E
:1018280009F000680F8700E0E0919B07E17009F07C
:101838000160E0919C07E17009F00260E0919D076A
:10184800E17009F00460E0919E07E17009F008601A
:10185800FE017096008300E0E091D60CE07409F078
:101868000160E091DE0CE07409F00260E091E60CA2
:10187800E07409F00460E091EE0CE07409F008608F
:10188800E091F60CE07409F00061E091FE0CE07460
:1018980009F00062E091060DE07409F00064E0913F
:1018A8000E0DE07409F00068FE017196008300E0F7
:1018B800E091160DE07409F00160E0911E0DE074EE
:1018C80009F00260E091260DE07409F00460E091EF
:1018D8002E0DE07409F00860E091360DE07409F00F
:1018E8000061E0913E0DE07409F00062E091460D60
:1018F800E07409F00064E0914E0DE07409F00068AE
:10190800FE017296008300E0E0917704E07809F028
:101918000160E0918504E07809F00260E0919304A9
:10192800E07809F00460E091A104E07809F008602B
:10193800E091AF04E07809F00061E091BD04E0783F
:1019480009F00062E091CB04E07809F00064E091CE
:10195800D904E07809F00068FE017396008300E07E
:10196800E091E704E07809F00160E091F504E0789F
:1019780009F00260E0910305E07809F00460E09165
:101988001105E07809F00860E0911F05E07809F09A
:101998000061E0912D05E07809F00062E0913B05D7
:1019A800E07809F00064E0914905E07809F0006802
:1019B800FE017496008300E0E0915705E07809F095
:1019C8000160E0916505E07809F00260E091730537
:1019D800E07809F00460E0918105E07809F008609A
:1019E800E0918F05E07809F00061E0919D05E078CD
:1019F80009F00062E0919D05E07809F00064E0914B
:101A0800B905E07809F00068FE017596008300E0EA
:101A1800E091C705E07809F00160E091D505E0782C
:101A280009F00260E091E305E07809F00460E091D4
:101A3800F105E07809F00860E091FF05E07809F029
:101A48000061E0910D06E07809F00062E0911B0664
:101A5800E07809F00064E0912906E07809F0006870
:101A6800FE0176960083EFC4E1E0E093A60D05C081
:101A7800E130A0E0FA0709F0DCC0E091AB0DF0918D
:101A8800AC0DE27009F4D1C0E091F708E077E033DB
:101A980021F4E091F708E47009F403C0E6E6EF8763
:101AA8000DC0E091F708E295E770FF2766277727D2
:101AB800E05EFE4F6F4F6BBF06900F86E091000906
:101AC800E077E03321F4E0910009E47009F403C001
:101AD800E6E6E88B0DC0E0910009E295E770FF2784
:101AE80066277727E05EFE4F6F4F6BBF0690088A28
:101AF800E0910909E077E03321F4E0910909E47005
:101B080009F403C0E6E6E98B0DC0E0910909E29506
:101B1800E770FF2766277727E05EFE4F6F4F6BBFA2
:101B28000690098AE0911209E077E03321F4E09108
:101B38001209E47009F403C0E6E6EA8B0DC0E091EF
:101B48001209E295E770FF2766277727E05EFE4FC8
:101B58006F4F6BBF06900A8AE0911B09E077E0336C
:101B680021F4E0911B09E47009F403C0E6E6EB8B6D
:101B78000DC0E0911B09E295E770FF2766277727DC
:101B8800E05EFE4F6F4F6BBF06900B8AE091240911
:101B9800E077E03321F4E0912409E47009F403C00C
:101BA800E6E6EC8B0DC0E0912409E295E770FF278B
:101BB80066277727E05EFE4F6F4F6BBF06900C8A53
:101BC800E0912D09E077E03321F4E0912D09E470EC
:101BD80009F403C0E6E6ED8B0DC0E0912D09E2950E
:101BE800E770FF2766277727E05EFE4F6F4F6BBFD2
:101BF80006900D8AE0913609E077E03321F4E09110
:101C08003609E47009F403C0E6E6EE8B0DC0E091F6
:101C18003609E295E770FF2766277727E05EFE4FD3
:101C28006F4F6BBF06900E8A0EC4E2E0E093A60DDC
:101C380005C0E230A0E0FA0709F0DCC0E091AB0D86
:101C4800F091AC0DE47009F4D1C0E0913F09E07760
:101C5800E03321F4E0913F09E47009F403C0E6E6BB
:101C6800EF870DC0E0913F09E295E770FF276627EF
:101C78007727E05EFE4F6F4F6BBF06900F86E091AF
:101C88004809E077E03321F4E0914809E47009F469
:101C980003C0E6E6E88B0DC0E0914809E295E770DD
:101CA800FF2766277727E05EFE4F6F4F6BBF0690D2
:101CB800088AE0915109E077E03321F4E091510975
:101CC800E47009F403C0E6E6E98B0DC0E091510920
:101CD800E295E770FF2766277727E05EFE4F6F4F94
:101CE8006BBF0690098AE0915A09E077E03321F446
:101CF800E0915A09E47009F403C0E6E6EA8B0DC0E6
:101D0800E0915A09E295E770FF2766277727E05E9A
:101D1800FE4F6F4F6BBF06900A8AE0916309E07728
:101D2800E03321F4E0916309E47009F403C0E6E6C6
:101D3800EB8B0DC0E0916309E295E770FF276627FA
:101D48007727E05EFE4F6F4F6BBF06900B8AE091DE
:101D58006C09E077E03321F4E0916C09E47009F450
:101D680003C0E6E6EC8B0DC0E0916C09E295E770E4
:101D7800FF2766277727E05EFE4F6F4F6BBF069001
:101D88000C8AE0917509E077E03321F4E091750958
:101D9800E47009F403C0E6E6ED8B0DC0E091750927
:101DA800E295E770FF2766277727E05EFE4F6F4FC3
:101DB8006BBF06900D8AE0917E09E077E03321F44D
:101DC800E0917E09E47009F403C0E6E6EE8B0DC0ED
:101DD800E0917E09E295E770FF2766277727E05EA6
:101DE800FE4F6F4F6BBF06900E8A2DC3E3E0E09362
:101DF800A60D04C0E330A0E0FA0721F4E4E0E09384
:101E0800A60D04C0E430A0E0FA0721F4E5E0E09371
:101E1800A60D05C0E530A0E0FA0709F0B0C0E091D2
:101E2800AB0DF091AC0DE07209F4A5C04091FE082D
:101E38005091FF084C3EE3E15E0738F4DA01E4E133
:101E4800F0E00E948ACB0E2F01C00FEF0F87A09100
:101E58000309A63319F4E0E0E88B13C040910709A1
:101E6800509108094C3EE3E15E0738F4DA01E4E1F9
:101E7800F0E00E948ACB0E2F01C00FEFFE01709692
:101E8800008340911009509111094C3EE3E15E072F
:101E980038F4DA01E4E1F0E00E948ACB0E2F01C0A9
:101EA8000FEFFE0171960083A0911509A63319F46E
:101EB800E0E0EA8B13C04091190950911A094C3E91
:101EC800E3E15E0738F4DA01E4E1F0E00E948ACB4E
:101ED8000E2F01C00FEFFE01729600834091220978
:101EE800509123094C3EE3E15E0738F4DA01E4E15E
:101EF800F0E00E948ACB0E2F01C00FEFFE0173960F
:101F0800008340912B0950912C094C3EE3E15E0778
:101F180038F4DA01E4E1F0E00E948ACB0E2F01C028
:101F28000FEFFE01749600834091340950913509F2
:101F38004C3EE3E15E0738F4DA01E4E1F0E00E94A8
:101F48008ACB0E2F01C00FEFFE01759600834091DA
:101F58003D0950913E094C3EE3E15E0738F4DA0151
:101F6800E4E1F0E00E948ACB0E2F01C00FEFFE01E2
:101F78007696008368C2E6E0E093A60D05C0E630D9
:101F8800A0E0FA0709F0A2C0E091AB0DF091AC0D0A
:101F9800E07409F497C040914609509147094C3EB6
:101FA800E3E15E0738F4DA01E4E1F0E00E948ACB6D
:101FB8000E2F01C00FEF0F8740914F095091500924
:101FC8004C3EE3E15E0738F4DA01E4E1F0E00E9418
:101FD8008ACB0E2F01C00FEFFE017096008340914F
:101FE8005809509159094C3EE3E15E0738F4DA018B
:101FF800E4E1F0E00E948ACB0E2F01C00FEFFE0152
:102008007196008340916109509162094C3EE3E169
:102018005E0738F4DA01E4E1F0E00E948ACB0E2F83
:1020280001C00FEFFE017296008340916A0950913A
:102038006B094C3EE3E15E0738F4DA01E4E1F0E0D5
:102048000E948ACB0E2F01C00FEFFE01739600830A
:1020580040917309509174094C3EE3E15E0738F4EE
:10206800DA01E4E1F0E00E948ACB0E2F01C00FEF05
:10207800FE017496008340917C0950917D094C3E85
:10208800E3E15E0738F4DA01E4E1F0E00E948ACB8C
:102098000E2F01C00FEFFE01759600834091850950
:1020A800509186094C3EE3E15E0738F4DA01E4E139
:1020B800F0E00E948ACB0E2F01C00FEFFE0176964A
:1020C8000083C1C1E7E0E093A60D04C0E730A0E0BB
:1020D800FA0721F4E8E0E093A60D04C0E830A0E098
:1020E800FA0721F4E9E0E093A60D04C0E930A0E086
:1020F800FA0741F5E091AB0DF091AC0DF270F1F0FB
:10210800A091ED08AA236AF0A091EC08B091ED081F
:10211800EAE0F0E00E9472CBAF010E941BCBAF0156
:1021280002C040E050E05F87FE0170964083E09176
:102138009A0DE98BE091990DEA8B85C1EAE0E0936D
:10214800A60D04C0EA30A0E0FA07D9F4E091AB0D7F
:10215800F091AC0DF47089F0A091F508B091F608F3
:10216800E4E1F0E00E948ACBAF015B8BFE0174963C
:102178004083E0E0ED8BEE8B66C1EBE0E093A60DCB
:1021880004C0EB30A0E0FA07C9F5E091AB0DF0917F
:10219800AC0DF87079F100E0E091560DE07409F0AB
:1021A8000160E0915E0DE07409F00260E091660D57
:1021B800E07409F00460E0916E0DE07409F00860C5
:1021C8000F87E0919209E17021F0E0919309E6957B
:1021D800EC8BE0919A09E17021F0E0919B09E6957A
:1021E800ED8BE091A209E17021F0E091A309E69559
:1021F800EE8B29C1ECE0E093A60D04C0EC30A0E022
:10220800FA07C9F5E091AB0DF091AC0DF07179F1D9
:10221800E2E0EF87ECE0E88BA6E1B0E00E9486CC34
:10222800E98BA5E1B0E00E9486CCEA8BE091AA098F
:10223800E17021F0E091AB09E695EB8BE091B209F2
:10224800E17021F0E091B309E695EC8BE091BA09D1
:10225800E17021F0E091BB09E695ED8BE091C209B0
:10226800E17021F0E091C309E695EE8BECC0EDE05A
:10227800E093A60D05C0ED30A0E0FA0709F0A6C06E
:10228800E091AB0DF091AC0DF07209F49BC0E091B8
:10229800AE0DEF5FE093AE0DE150EF8700E0E09107
:1022A8009C0DE03009F00160E0919D0DE03009F0EF
:1022B8000260E091F008E17009F00460E091F00834
:1022C800E27009F00860E091F008E07209F000613E
:1022D800E091EF08E07809F00062A5E3B1E00E9420
:1022E80086CCA091900DAE1708F00064A091CE03A3
:1022F800A13008F00068FE0170960083E091840D1B
:10230800F091850DFF70EF2FF0E0E98BE091840DDF
:10231800F091850DEA8BE0E01E2F0E2F31E018308A
:1023280060F4A3E01A9FF001ED5BF84FE081E270E2
:1023380009F0032B1F5F330FF2CFFE017396008362
:1023480000E018E031E0103160F4A3E01A9FF001DA
:10235800ED5BF84FE081E27009F0032B1F5F330F4C
:10236800F2CFFE017496008300E010E131E01431F1
:1023780060F4A3E01A9FF001ED5BF84FE081E27092
:1023880009F0032B1F5F330FF2CFFE017596008310
:10239800E0E01E2F0E2F31E0153080F4E12FAFE77B
:1023A800B7E0F0E00E940DCBAE0FBF1F1396EC9183
:1023B800E17009F0032B1F5F330FEECFFE01769615
:1023C800008341C0EEE0E093A60D04C0EE30A0E02B
:1023D800FA07C9F5E091AB0DF091AC0DF07479F105
:1023E800E0917508F09176080E941FCBAF015F87D6
:1023F800FE0170964083E0917708F09178080E947A
:102408001FCBAF01598BFE017296408300E0E0912B
:10241800F008E47009F00160E091F008E87009F054
:102428000260E091F008E07109F00460E091F008C2
:10243800E07209F00860FE017396008304C0E0E0D2
:10244800E093A60DB9C9A091A70DB091A80D8091F0
:10245800A90D9091AA0DE091A60DF0E06F2F660FDF
:10246800660B762FEA0FFB1F681F791FEE83FF8329
:1024780068877987AE81BF8188859985A030E8E033
:10248800BE07E0E08E07E0E09E0740F4EA85EF7EB5
:10249800EA87EE81FF81EB87FC870BC0EA85E06164
:1024A800EA87EE81FF8168857985EB87FC876D87F0
:1024B8007E87DE011A960E942D090E9496CA6796A9
:1024C800089564970E948FCAE0916304E07409F448
:1024D80024C4EF81E07FE860EF83A091AD0DA130C7
:1024E80008F450C0E091AD0DE150E093AD0DEF5F01
:1024F800E091AD0DE03009F045C0AFE3B1E00E94D6
:1025080086CCE093AD0DABE3B1E00E947ECCEC8BC2
:10251800FD8B6E8B7F8BAC89BD898E899F89A0309E
:10252800E8E0BE07E0E08E07E0E09E0740F4EF81B8
:10253800EF7EEF83EC89FD89E887F9870BC0EF818F
:10254800E061EF83EC89FD896E897F89E887F987E7
:102558006A877B87A9E3B1E00E9486CCEC87AAE36F
:10256800B1E00E9486CCED87E2E0EE87ECE0EF87F1
:10257800E8E0E88BE0E0E98BEA8BEB8BDE0117966D
:102588000E942D09A0919E0DA13008F421C1E0916F
:102598009E0DE150E0939E0DE03009F019C1FE0157
:1025A8003C96FA93EA93E0E0EA93A8E0B0E00E9450
:1025B8008EC3A3E5B5E00E9486CCE0939E0DA4E50A
:1025C800B5E00E947ECCEC8BFD8B6E8B7F8BAC894B
:1025D800BD898E899F89A030E8E0BE07E0E08E07BC
:1025E800E0E09E0740F4EF81EF7EEF83EC89FD8900
:1025F800E887F9870BC0EF81E061EF83EC89FD89FB
:102608006E897F89E887F9876A877B87A0919F0D04
:10261800A13090F1E091A00DEF5FE093A00DE150A3
:10262800A091A00DE0919F0DEA1718F4E1E0E09366
:10263800A00DE091A00DEC87A8E5B5E0F0E0349698
:10264800AE0FBF1F0E9486CC4E2F4F3010F04F3177
:1026580008F012C0E42FF0E03F97A9E0B0E00E9434
:1026680044CBE250F74FDF01ED91FD91DF01E4E14A
:10267800F0E00E948ACBEB8BADE5B5E00E9486CCFA
:102688004E2F4F3010F04F3108F012C0E42FF0E019
:102698003F97A9E0B0E00E9444CBE250F74FDF013A
:1026A800ED91FD91DF01E4E1F0E00E948ACBEA8B35
:1026B800ACE5B5E00E9486CC4E2F4F3010F04F317C
:1026C80008F012C0E42FF0E03F97A9E0B0E00E94C4
:1026D80044CBE250F74FDF01ED91FD91DF01E4E1DA
:1026E800F0E00E948ACBE98BABE5B5E00E9486CC8E
:1026F8004E2F4F3010F04F3108F012C0E42FF0E0A9
:102708003F97A9E0B0E00E9444CBE250F74FDF01C9
:10271800ED91FD91DF01E4E1F0E00E948ACBE88BC6
:10272800AAE5B5E00E9486CC4E2F4F3010F04F310D
:1027380008F012C0E42FF0E03F97A9E0B0E00E9453
:1027480044CBE250F74FDF01ED91FD91DF01E4E169
:10275800F0E00E948ACBEF87A9E5B5E00E9486CC1D
:102768004E2F4F3010F04F3108F012C0E42FF0E038
:102778003F97A9E0B0E00E9444CBE250F74FDF0159
:10278800ED91FD91DF01E4E1F0E00E948ACBEE8754
:10279800A8E5B5E00E9486CC4E2F4F3010F04F319F
:1027A80008F012C0E42FF0E03F97A9E0B0E00E94E3
:1027B80044CBE250F74FDF01ED91FD91DF01E4E1F9
:1027C800F0E00E948ACBED87DE0117960E942D0962
:1027D800A091A10DA13008F47CC0E091A10DE150B9
:1027E800E093A10DEF5FE091A10DE03009F071C019
:1027F800FE013C96FA93EA93E0E0EA93A8E0B0E0A1
:102808000E948EC3AAE6B5E00E9486CCE093A10D93
:10281800ABE6B5E00E947ECCEC8BFD8B6E8B7F8B9C
:10282800AC89BD898E899F89A030E8E0BE07E0E0C9
:102838008E07E0E09E0740F4EF81EF7EEF83EC899E
:10284800FD89E887F9870BC0EF81E061EF83EC89A8
:10285800FD896E897F89E887F9876A877B87E0E049
:102868000E2F1E2F2E2F51E0103300F5AFE6B5E0E6
:10287800EE27A10FBE1F0E9486CC4E2F403031F0AC
:10288800A42F0E947A3BE03009F0052B503859F408
:10289800E22F2F5FF0E0DE011C96EA0FFB1F00839A
:1028A80051E000E001C0550F1F5FDECFA091F50891
:1028B800B091F608AC39E3E6BE0728F4E4E6F0E0A8
:1028C8000E948ACB01C0EFEFEA8BDE0117960E94C7
:1028D8002D09A091A20DA13008F4A9C0E091A20D84
:1028E800E150E093A20DEF5FE091A20DE03009F016
:1028F8009EC0AFE9B5E00E9486CCE093A20DA0EAA5
:10290800B5E00E947ECCEC8BFD8B6E8B7F8BAC8907
:10291800BD898E899F89A030E8E0BE07E0E08E0778
:10292800E0E09E0740F4EF81EF7EEF83EC89FD89BC
:10293800E887F9870BC0EF81E061EF83EC89FD89B7
:102948006E897F89E887F9876A877B87E0E00E2FA1
:102958001E2F2E2F51E0103308F055C0A4EAB5E021
:10296800EE27A10FBE1F0E9486CC4E2F4030D9F112
:102978004F3010F04F3108F024C04F3108F5E42FE4
:10298800F0E03F97A9E0B0E00E9444CBE950F74F50
:10299800E081E295E770EE83E42FF0E03F97A9E04D
:1029A800B0E00E9444CBE950F74FE081E47039F47D
:1029B800AE81A13021F0A43011F0A53009F4052B27
:1029C80012C0473310F04C3308F007C0A42F0E9400
:1029D8008A7AE03009F0052B06C0A42F0E947A3BC2
:1029E800E03009F0052B503859F4E22F2F5FF0E062
:1029F800DE011C96EA0FFB1F008351E000E001C0D6
:102A0800550F1F5FA8CFA091EC08B091ED080024E6
:102A18000A160B0624F4EA89E295EF7001C0E0E09B
:102A2800EA8BE0E0EB8BDE0117960E942D09A0915E
:102A3800A30DA13008F4A8C0E091A30DE150E093E4
:102A4800A30DEF5FE091A30DE03009F09DC0FE01FA
:102A58003C96FA93EA93E0E0EA93A8E0B0E00E949B
:102A68008EC3A4EDB5E00E9486CCE093A30DA5ED3E
:102A7800B5E00E947ECCEC8BFD8B6E8B7F8BAC8996
:102A8800BD898E899F89A030E8E0BE07E0E08E0707
:102A9800E0E09E0740F4EF81EF7EEF83EC89FD894B
:102AA800E887F9870BC0EF81E061EF83EC89FD8946
:102AB8006E897F89E887F9876A877B87E0E00E2F30
:102AC8001E2F2E2F51E0103408F05AC0A9EDB5E0A2
:102AD800EE27A10FBE1F0E9486CC4E2F403009F46E
:102AE8003FC0103220F04F3010F04F3108F024C0B2
:102AF8004F3108F5E42FF0E03F97A9E0B0E00E94DD
:102B080044CBE950F74FE081E295E770EE83E42F7C
:102B1800F0E03F97A9E0B0E00E9444CBE950F74FBE
:102B2800E081E47039F4AE81A13021F0A43011F0D5
:102B3800A53009F4052B14C0103220F0473310F0EB
:102B48004C3308F007C0A42F0E948A7AE03009F0BD
:102B5800052B06C0A42F0E947A3BE03009F0052B14
:102B6800503859F4E22F2F5FF0E0DE011C96EA0F8F
:102B7800FB1F008351E000E001C0550F1F5FA3CF8A
:102B8800DE0117960E942D0910E0133008F0C5C029
:102B9800AFEABDE0E12FF0E0EE0FFF1FAE0FBF1F61
:102BA80011964C91403009F4B6C0AFEABDE0E12F70
:102BB800F0E0EE0FFF1FAE0FBF1FEC91EF773E2F37
:102BC800A42F0E947A3B0E2FAFEABDE0E12FF0E080
:102BD800EE0FFF1FAE0FBF1FEC91EE1FE0E0EE1FE0
:102BE800E1700E1799F031E0AFEABDE0E12FF0E0B7
:102BF800EE0FFF1FAE0FBF1FE02FE170E795E0E07B
:102C0800E7950E2EEC91EF77E029EC93313008F43C
:102C180073C03150303009F06FC0A0E2B6E00E94B6
:102C280086CC3E2FA1E2B6E0E12FF0E0BD01A5E1A0
:102C3800B0E00E9444CBDB01AE0FBF1F0E947ECCE8
:102C4800EC8BFD8B6E8B7F8BAC89BD898E899F89C0
:102C5800A030E8E0BE07E0E08E07E0E09E0740F421
:102C6800EF81EF7EEF83EC89FD89E887F9870BC058
:102C7800EF81E061EF83EC89FD896E897F89E887C0
:102C8800F9876A877B87EF81E07FE860EF83AFEAA7
:102C9800BDE0E12FF0E0EE0FFF1FAE0FBF1FEC917C
:102CA800E07869F0A1E2B6E0E12FF0E0BD01A5E12E
:102CB800B0E00E9444CBE60FF71F35960CC0A1E2A6
:102CC800B6E0E12FF0E0BD01A5E1B0E00E9444CB01
:102CD800E60FF71F3D96E88FF98FFE013C96FA93B1
:102CE800EA93EA8DFB8DFA93EA93A8E00E94E9251E
:102CF800DE0117960E942D09AFEABDE0E12FF0E052
:102D0800EE0FFF1FAE0FBF1FE32FEF770E2EEC91D4
:102D1800E078E029EC931F5F38CF0E9496CA6A9644
:102D280008951A93A3E5B5E0E0E00E94A2CCA4E5DB
:102D3800B5E0E0E0F0E060E070E00E9492CC10E0E6
:102D4800123148F4A8E5B5E0EE27A10FBE1F0E9496
:102D5800A2CC1F5FF5CFE0E2F6E0FA93EA93AAE689
:102D68000E941E26E0E9F6E4FA93EA93A0E5B0E0B3
:102D78000E94BE29AAE6B5E0E0E00E94A2CCABE63C
:102D8800B5E0E0E0F0E060E070E00E9492CC10E096
:102D9800103348F4AFE6B5E0EE27A10FBE1F0E943E
:102DA800A2CC1F5FF5CFAFE9B5E0E0E00E94A2CC6E
:102DB800A0EAB5E0E0E0F0E060E070E00E9492CCCC
:102DC80010E0103348F4A4EAB5E0EE27A10FBE1FC7
:102DD8000E94A2CC1F5FF5CFA4EDB5E0E0E00E9411
:102DE800A2CCA5EDB5E0E0E0F0E060E070E00E9484
:102DF80092CC10E0103448F4A9EDB5E0EE27A10F0D
:102E0800BE1F0E94A2CC1F5FF5CFA9E1B6E0E0E0AB
:102E18000E94A2CCAAE1B6E0E0E0F0E060E070E059
:102E28000E9492CCAEE1B6E0EFEFFFEF0E949ACCA1
:102E3800A5C21A93ACE6B2E00E9482CCDF010E94E0
:102E4800D204A5E7B2E00E9486CCE170A5EEB8E016
:102E5800E170E795E0E0E7950E2EEC91EF77E02939
:102E6800EC93E0E0E093E208EDE5F4E0FA93EA930E
:102E7800E0E0EA93A6EEB2E00E948EC3A0E7B2E0DB
:102E88000E9486CCE0935E04A0915E04A53018F4FD
:102E9800E5E0E0935E04A5E7B2E00E9486CCE69503
:102EA800E170A3E6B4E0E170E795E0E0E7950E2E67
:102EB800EC91EF77E029EC93A1E7B2E00E947ECC99
:102EC800E0935F04F093600460936104709362047C
:102ED800E0E0E0936A0410E0143308F01DC2ABE7A9
:102EE800B2E0E12FF0E0BD01AEE0B0E00E9444CBDB
:102EF800DB01AE0FBF1F1A960E9486CCE07809F45A
:102F080009C2ABE6B4E0E12FF0E0BD01AEE0B0E00D
:102F18000E9444CBDB01AE0FBF1F1A96EC91E0680C
:102F2800EC93ABE6B4E0E12FF0E0BD01AEE0B0E039
:102F38000E9444CBE60FF71FFF93EF93ABE7B2E095
:102F4800E12FF0E0BD01AEE0B0E00E9444CBDB0130
:102F5800AE0FBF1F0E947ECCAF91BF91ED93FD9342
:102F68006D937C93ABE6B4E0E12FF0E0BD01AEE0F9
:102F7800B0E00E9444CBE60FF71F3496FF93EF931F
:102F8800ABE7B2E0E12FF0E0BD01AEE0B0E00E94B7
:102F980044CBDB01AE0FBF1F14960E9482CCAF91C9
:102FA800BF91ED93FC93ABE6B4E0E12FF0E0BD01F7
:102FB800AEE0B0E00E9444CBE60FF71F3696FF93D1
:102FC800EF93ABE7B2E0E12FF0E0BD01AEE0B0E097
:102FD8000E9444CBDB01AE0FBF1F16960E9482CC25
:102FE800AF91BF91ED93FC93ABE6B4E0E12FF0E035
:102FF800BD01AEE0B0E00E9444CBE60FF71F389663
:10300800FF93EF93ABE7B2E0E12FF0E0BD01AEE054
:10301800B0E00E9444CBDB01AE0FBF1F18960E94A0
:1030280082CCAF91BF91ED93FC93ABE6B4E0E12F76
:10303800F0E0BD01AEE0B0E00E9444CBE60FF71F20
:103048003A96FF93EF93ABE7B2E0E12FF0E0BD01D2
:10305800AEE0B0E00E9444CBDB01AE0FBF1F1A9672
:103068000E9486CCEF70AF91BF91EF700E2EEC915D
:10307800E07FE029EC93ABE6B4E0E12FF0E0BD019E
:10308800AEE0B0E00E9444CBE60FF71F3A96FF93FC
:10309800EF93ABE7B2E0E12FF0E0BD01AEE0B0E0C6
:1030A8000E9444CBDB01AE0FBF1F1A960E9486CC4C
:1030B800E295E770AF91BF91E770E295E07F0E2E41
:1030C800EC91EF78E029EC93ABE6B4E0E12FF0E087
:1030D800BD01AEE0B0E00E9444CBE60FF71F3B967F
:1030E800FF93EF93ABE7B2E0E12FF0E0BD01AEE074
:1030F800B0E00E9444CBDB01AE0FBF1F1B960E94BD
:1031080086CCEF70AF91BF91EF700E2EEC91E07FFF
:10311800E029EC93ABE6B4E0E12FF0E0BD01AEE0CE
:10312800B0E00E9444CBE60FF71F3B96FF93EF9366
:10313800ABE7B2E0E12FF0E0BD01AEE0B0E00E9405
:1031480044CBDB01AE0FBF1F1B960E9486CCE295D5
:10315800EF70AF91BF91EF70E295E07F0E2EEC918A
:10316800EF70E029EC93ABE6B4E0E12FF0E0BD01AD
:10317800AEE0B0E00E9444CBE60FF71F3C96FF9309
:10318800EF93ABE7B2E0E12FF0E0BD01AEE0B0E0D5
:103198000E9444CBDB01AE0FBF1F1C960E9486CC59
:1031A800E170AF91BF91E1700E2EEC91EE7FE029B6
:1031B800EC93ABE6B4E0E12FF0E0BD01AEE0B0E0A7
:1031C8000E9444CBE60FF71F3C96FF93EF93ABE7C3
:1031D800B2E0E12FF0E0BD01AEE0B0E00E9444CBE8
:1031E800DB01AE0FBF1F1C960E9486CCE695E170EE
:1031F800AF91BF91E170EE0F0E2EEC91ED7FE029BB
:10320800EC93ABE6B4E0E12FF0E0BD01AEE0B0E056
:103218000E9444CBE60FF71F3C96FF93EF93ABE772
:10322800B2E0E12FF0E0BD01AEE0B0E00E9444CB97
:10323800DB01AE0FBF1F1C960E9486CCE695E69573
:10324800E370AF91BF91E370EE0FEE0F0E2EEC918D
:10325800E37FE029EC93ABE6B4E0E12FF0E0BD01B9
:10326800AEE0B0E00E9444CBE60FF71F3C96FF9318
:10327800EF93ABE7B2E0E12FF0E0BD01AEE0B0E0E4
:103288000E9444CBDB01AE0FBF1F1C960E9486CC68
:10329800E295E170AF91BF91E170E295E07F0E2E6B
:1032A800EC91EF7EE029EC93ABE6B4E0E12FF0E09F
:1032B800BD01AEE0B0E00E9444CBDB01AE0FBF1F02
:1032C8001C96EC91EC70E43089F0ABE6B4E0E12FA9
:1032D800F0E0BD01AEE0B0E00E9444CBDB01AE0FF0
:1032E800BF1F1C96EC91EC70EC3081F4ABE6B4E0B7
:1032F800E12FF0E0BD01AEE0B0E00E9444CBDB017D
:10330800AE0FBF1F1C96EC91E068EC93E12FEF5FC6
:10331800E0936A041F5FE0CDE4E6F4E0FA93EA93F1
:10332800E0E4F1E0FA93EA93A5E00E94E925E09150
:103338006504F091660460916704709168043097A1
:103348006040704021F4E0916404EF7E15C0E09184
:103358006404E061E0936404F0E0F695E795E370B7
:10336800F070E330A0E0FA0721F0E130A0E0FA07BE
:1033780029F4E0916404E860E093640419910895E5
:10338800BA93AA936D970E948FCAE0E0EE8BABA127
:10339800BCA1EC91E295E1703E2F3030C1F011965E
:1033A800ED91FD916D917D91ED8FFE8F6F8F78A3DB
:1033B800E0915F04F091600460916104709162048F
:1033C800AD8DBE8D8F8D98A10E943CCB0CC0ABA15A
:1033D800BCA111964D915C91A0915F04B0916004DD
:1033E800FA010E942ACBE88FE03099F1ABA1BCA189
:1033F800EC91EF70E13038F0EBA1FCA1A581A17050
:1034080011F00E94CB27ABA1BCA1EC91EF70E63084
:1034180000F120E0E1E0EA8FE98F2031D0F4ABA1A0
:10342800BCA11596EA8DF0E0AE0FBF1FEC91A98DF7
:10343800EA2319F0A22F0E94816AE98DEE0FE98F25
:10344800E03029F4EA8DEF5FEA8FE1E0E98F2F5F42
:10345800E4CFE0916404E07109F43FC0303079F0C2
:10346800E0916504F09166046091670470916804C6
:10347800AD8DBE8D8F8D98A10E943CCB07C0A091C9
:103488006504B0916604FA010E942ACBE88FE03007
:1034980021F1EBA1FCA1A581A17071F0E091640478
:1034A800E17021F0E0916404E77F03C0E0916404D7
:1034B800E860E09364040DC0E0916404E17021F0D9
:1034C800E0916404E86003C0E0916404E77FE0935E
:1034D8006404E0915E04E0936904E0916304EF7092
:1034E800E23011F4E1E0EE8BA0916A04A433A0F07D
:1034F800E2EFF1E060E070E00E9418CCE0916A042D
:10350800FF27662777270E9418CC84E00E9416CAF6
:103518002896E4E3E0936A0420E0E0916A042E1719
:1035280008F04FC5ABE6B4E0E22FF0E0BD01AEE035
:10353800B0E00E9444CBE60FF71F8F01E285E078E8
:1035480009F43DC5303061F0D801ED91FD916D91E0
:103558007D91AD8DBE8D8F8D98A10E943CCB07C00B
:10356800D801ED91FD91DF01FA010E942ACBE88F85
:10357800E03009F424C5E0916304E07409F40DC552
:10358800F801E485E07171F1ABE7B2E0E22FF0E019
:10359800BD01AEE0B0E00E9444CBDB01AE0FBF1F1F
:1035A8001C960E9486CCE295EF70E695E770ABA179
:1035B800BCA11596F0E0AE0FBF1FEC91EF93ABE7FF
:1035C800B2E0E22FF0E0BD01AEE0B0E00E9444CBF3
:1035D800DB01AE0FBF1F1D960E9486CCAF91EA1784
:1035E80009F0DBC4ABE6B4E0E22FF0E0BD01AEE0E9
:1035F800B0E00E9444CBDB01AE0FBF1F1D96E091E7
:103608005E04EC93E0E0E9A3EAA3F801E385EF7038
:10361800E13038F1ABA1BCA11596F801E385F0E0E3
:10362800EF70F0703197AE0FBF1FEC91F0E0E9A397
:10363800FAA3F9A1E0E0E9A3FAA3ABA1BCA115960E
:10364800F801E385F0E00E941BCBEF70F070319732
:10365800AE0FBF1FEC91A9A1BAA1F0E0EA2BFB2B9A
:103668000FC0ABA1BCA11596F801E385F0E00E945C
:103678001BCBEF70F0703197AE0FBF1FEC91F0E0ED
:10368800E9A3FAA3D8011896ED91FD91A9A1BAA1D1
:10369800EA23FB23E9A3FAA3F801E485E17059F0D2
:1036A800F801A085B185FD01F695E795A9A1BAA114
:1036B800EA17FB0708F00CC0D8011896ED91FD91A8
:1036C800E095F095A9A1BAA1EA2BFB2BE9A3FAA3EF
:1036D800F801E485E295EF70E695E695E170EF8BE9
:1036E800F801E485E17009F456C2E9A1FAA1EB8F6B
:1036F800FC8FF801E285F0E0EF70F070E630A0E0B2
:10370800FA0709F4C7C13097C9F4AB8DBC8D002402
:103718000A160B0624F4EB8DFC8DF29606C0AC8DD0
:10372800AA232AF4EB8DFC8DF297EB8FFC8FAB8DDF
:10373800BC8DE4E6F0E00E949DCBAAC1E130A0E098
:10374800FA07C9F4AB8DBC8D00240A160B0624F4C5
:10375800EB8DFC8D799606C0AC8DAA232AF4EB8DEF
:10376800FC8D7997EB8FFC8FAB8DBC8DE2E3F0E09D
:103778000E949DCB8DC1E230A0E0FA07C9F4AB8D61
:10378800BC8D00240A160B0624F4EB8DFC8D3A96AA
:1037980006C0AC8DAA232AF4EB8DFC8D3A97EB8FEB
:1037A800FC8FAB8DBC8DE4E1F0E00E949DCB70C135
:1037B800E330A0E0FA07C9F4AB8DBC8D00240A16EB
:1037C8000B0624F4EB8DFC8D359606C0AC8DAA2330
:1037D8002AF4EB8DFC8D3597EB8FFC8FAB8DBC8D70
:1037E800EAE0F0E00E949DCB53C1E430A0E0FA0784
:1037F800C9F4AB8DBC8D00240A160B0624F4EB8D9E
:10380800FC8D339606C0AC8DAA232AF4EB8DFC8D73
:103818003397EB8FFC8FAB8DBC8DE5E0F0E00E9419
:103828009DCB36C1E530A0E0FA07C9F4AB8DBC8D5D
:1038380000240A160B0624F4EB8DFC8D329606C084
:10384800AC8DAA232AF4EB8DFC8D3297EB8FFC8F7D
:10385800AB8DBC8DE2E0F0E00E949DCB19C1E73052
:10386800A0E0FA0741F5AB8DBC8D00240A160B06C3
:1038780074F4AF3FEFE3BE071CF0EFEFFFE704C0BF
:10388800EB8DFC8DEE0FFF1FEB8FFC8F13C0AC8D03
:10389800AA2382F4AB8DBC8DE0E0F0ECEA17FB07BD
:1038A8001CF0E0E0F0E804C0EB8DFC8DEE0FFF1F8C
:1038B800EB8FFC8FEFC0E830A0E0FA0761F5AB8D25
:1038C800BC8D00240A160B0684F4A939E9E1BE0769
:1038D8001CF0EFEFFFE706C0EB8DFC8DA5E0B0E034
:1038E8000E9472CBEB8FFC8F15C0AC8DAA2392F48B
:1038F800AB8DBC8DE7E6F6EEEA17FB071CF0E0E0BF
:10390800F0E806C0EB8DFC8DA5E0B0E00E9472CB1C
:10391800EB8FFC8FBFC0E930A0E0FA0761F5AB8DF3
:10392800BC8D00240A160B0684F4AC3CECE0BE0700
:103938001CF0EFEFFFE706C0EB8DFC8DAAE0B0E0CE
:103948000E9472CBEB8FFC8F15C0AC8DAA2392F42A
:10395800AB8DBC8DE4E3F3EFEA17FB071CF0E0E066
:10396800F0E806C0EB8DFC8DAAE0B0E00E9472CBB7
:10397800EB8FFC8F8FC0EA30A0E0FA0761F5AB8DC2
:10398800BC8D00240A160B0684F4A636E6E0BE07B2
:103998001CF0EFEFFFE706C0EB8DFC8DA4E1B0E073
:1039A8000E9472CBEB8FFC8F15C0AC8DAA2392F4CA
:1039B800AB8DBC8DEAE9F9EFEA17FB071CF0E0E0F4
:1039C800F0E806C0EB8DFC8DA4E1B0E00E9472CB5C
:1039D800EB8FFC8F5FC0EB30A0E0FA0761F5AB8D91
:1039E800BC8D00240A160B0684F4AF38E2E0BE074B
:1039F8001CF0EFEFFFE706C0EB8DFC8DA2E3B0E013
:103A08000E9472CBEB8FFC8F15C0AC8DAA2392F469
:103A1800AB8DBC8DE1E7FDEFEA17FB071CF0E0E09A
:103A2800F0E806C0EB8DFC8DA2E3B0E00E9472CBFB
:103A3800EB8FFC8F2FC0EC30A0E0FA0759F5AB8D67
:103A4800BC8D00240A160B0684F4A734E1E0BE07F7
:103A58001CF0EFEFFFE706C0EB8DFC8DA4E6B0E0AD
:103A68000E9472CBEB8FFC8F15C0AC8DAA2392F409
:103A7800AB8DBC8DE1E7FDEFEA17FB071CF0E0E03A
:103A8800F0E806C0EB8DFC8DA4E6B0E00E9472CB96
:103A9800EB8FFC8FF801E285F0E00E941BCBE7700A
:103AA800F070309769F4F801A481B581EB8DFC8D35
:103AB800EA17FB0711F4E1E001C0E0E0EF8B6AC010
:103AC800E130A0E0FA0769F4F801A481B581EB8D33
:103AD800FC8DEA17FB0711F4E0E001C0E1E0EF8B91
:103AE80059C0E230A0E0FA07D9F4EF89E03061F07C
:103AF800D8011696ED91FD91AB8DBC8DEA17FB07A9
:103B080014F0E0E0EF8B0BC0D8011496ED91FD9115
:103B1800AB8DBC8DEA17FB0714F4E1E0EF8B3AC0DC
:103B2800E330A0E0FA07D9F4EF89E03061F0D8017A
:103B38001696ED91FD91AB8DBC8DAE17BF0714F0B5
:103B4800E0E0EF8B0BC0D8011496ED91FD91AB8DA1
:103B5800BC8DAE17BF0714F4E1E0EF8B1BC0E43057
:103B6800A0E0FA07B9F4D8011496ED91FD91AB8D58
:103B7800BC8DAE17BF074CF0D8011696ED91FD919C
:103B8800AB8DBC8DEA17FB070CF402C0E1E001C065
:103B9800E0E0EF8B75C1F801E285F0E0EF70F070BE
:103BA800E630A0E0FA0709F4CCC0309761F4E9A147
:103BB800FAA1F296E9A3FAA3A9A1BAA1E4E6F0E072
:103BC8000E948ACBBCC0E130A0E0FA0761F4E9A109
:103BD800FAA17996E9A3FAA3A9A1BAA1E2E3F0E0D0
:103BE8000E948ACBACC0E230A0E0FA0761F4E9A1F8
:103BF800FAA13A96E9A3FAA3A9A1BAA1E4E1F0E0EF
:103C08000E948ACB9CC0E330A0E0FA0761F4E9A1E6
:103C1800FAA13596E9A3FAA3A9A1BAA1EAE0F0E0CE
:103C28000E948ACB8CC0E430A0E0FA0761F4E9A1D5
:103C3800FAA13396E9A3FAA3A9A1BAA1E5E0F0E0B5
:103C48000E948ACB7CC0E530A0E0FA0741F4E9A1E4
:103C5800FAA13196E9A3FAA3F695E79570C0E73083
:103C6800A0E0FA0781F4A9A1BAA1AF3FEFE7BE0728
:103C780028F4E9A1FAA1EE0FFF1F02C0EFEFFFEF52
:103C8800E9A3FAA35EC0E830A0E0FA0779F4A9A195
:103C9800BAA1A333E3E3BE0720F4E5E00E946CCBAE
:103CA80002C0EFEFFFEFE9A3FAA34BC0E930A0E0B1
:103CB800FA0779F4A9A1BAA1A939E9E1BE0720F464
:103CC800EAE00E946CCB02C0EFEFFFEFE9A3FAA392
:103CD80038C0EA30A0E0FA0779F4A9A1BAA1AC3C4F
:103CE800ECE0BE0720F4E4E10E946CCB02C0EFEFE9
:103CF800FFEFE9A3FAA325C0EB30A0E0FA0779F4B7
:103D0800A9A1BAA1AE31E5E0BE0720F4E2E30E9422
:103D18006CCB02C0EFEFFFEFE9A3FAA312C0EC30BF
:103D2800A0E0FA0771F4A9A1BAA1AF38E2E0BE0792
:103D380020F4E4E60E946CCB02C0EFEFFFEFE9A3AA
:103D4800FAA3F801E285F0E00E941BCBE770F0705F
:103D5800309769F4F801A481B581E9A1FAA1EA17BD
:103D6800FB0711F4E1E001C0E0E0EF8B89C0E1302E
:103D7800A0E0FA0769F4F801A481B581E9A1FAA1E4
:103D8800EA17FB0711F0E0E001C0E1E0EF8B78C033
:103D9800E230A0E0FA07D1F5F801E485E170D9F046
:103DA800EF89E03061F0D8011696ED91FD91A9A157
:103DB800BAA1EA17FB0714F0E0E0EF8B0BC0D801BB
:103DC8001496ED91FD91A9A1BAA1EA17FB0714F485
:103DD800E1E0EF8B1AC0EF89E03061F0D801169668
:103DE800ED91FD91A9A1BAA1EA17FB0710F0E0E057
:103DF800EF8B0BC0D8011496ED91FD91A9A1BAA142
:103E0800EA17FB0710F4E1E0EF8B3AC0E330A0E0DB
:103E1800FA07D9F4EF89E03061F0D8011696ED91F0
:103E2800FD91A9A1BAA1AE17BF0710F0E0E0EF8B92
:103E38000BC0D8011496ED91FD91A9A1BAA1AE17B6
:103E4800BF0710F4E1E0EF8B1BC0E430A0E0FA07F5
:103E5800B9F4D8011496ED91FD91A9A1BAA1AE17B4
:103E6800BF0748F0D8011696ED91FD91A9A1BAA116
:103E7800EA17FB0708F402C0E1E001C0E0E0EF8BBD
:103E8800F801E485E27009F448C0F801E485E074BB
:103E980019F4EF89E03009F43FC0F801E485E078CF
:103EA800F1F0D8011C96EC91EF77EC93E091630464
:103EB800E073E03298F0E5E0F2E060E070E00E9444
:103EC80018CCE22FF0E031966F2F660F660B762F35
:103ED8000E9418CC84E00E9416CA28961DC0D801FA
:103EE8001C96EC91E068EC93E0916304E073E03297
:103EF80098F0E0E1F2E060E070E00E9418CCE22F78
:103F0800F0E031966F2F660F660B762F0E9418CC63
:103F180084E00E9416CA289633C0F801E485EE1F93
:103F2800E0E0EE1FE170AE2FEF89EA1749F1D80102
:103F38001C96E170E795E0E0E7950E2EEC91EF779F
:103F4800E029EC93E0916304E073E032C8F0EBE120
:103F5800F2E060E070E00E9418CCE22FF0E03196C9
:103F68006F2F660F660B762F0E9418CCEF8DFF27F8
:103F7800662777270E9418CC88E00E9416CA2C96DC
:103F8800D8011C96EF89E170E295E07FEE0FEE0F05
:103F98000E2EEC91EF7BE029EC93E0916304EF7037
:103FA800E13059F0E0916304EF70AE2FE22FF0E0BA
:103FB8003396B0E0EA17FB0711F4E1E0EE8B2F5FD0
:103FC800ACCAE0916304EF70E23019F0EE89E0309A
:103FD800A1F1ABA1BCA1EC91EF70ED87AD85A93043
:103FE80010F0E8E0ED87ED85E85FEF83E6E0E8872D
:103FF800ABA1BCA1EC91E07121F011960E9401CC1B
:1040080007C0ABA1BCA11196ED91FD91662777275A
:10401800E987FA876B877C87FE013E96FA93EA93D5
:10402800EDA1FEA13596FA93EA93A989BB270E94D0
:104038007CC3DE0116960E94E7900E9496CAA59658
:1040480008951A930A93AEE6B2E00E9486CC0E2F2A
:10405800003029F0A02F0E947A3BE03021F0E09157
:104068006304E06403C0E0916304EF7BE0936304BE
:1040780010E0E0916A041E1708F07DC0ABE6B4E0DA
:10408800E12FF0E0BD01AEE0B0E00E9444CBDB01DF
:10409800AE0FBF1F1D96AC91A13008F46AC0ABE605
:1040A800B4E0E12FF0E0BD01AEE0B0E00E9444CB07
:1040B800DB01AE0FBF1F1D96EC91E150EC93ABE610
:1040C800B4E0E12FF0E0BD01AEE0B0E00E9444CBE7
:1040D800DB01AE0FBF1F1D96EC91E03009F049C01F
:1040E800ABE6B4E0E12FF0E0BD01AEE0B0E00E9445
:1040F80044CBDB01AE0FBF1F1C96EC91F0E00E9491
:104108001FCBE370F070309781F4ABE6B4E0E12F99
:10411800F0E0BD01AEE0B0E00E9444CBDB01AE0FA1
:10412800BF1F1C96EC91EF7713C0E130A0E0FA07AF
:1041380001F5ABE6B4E0E12FF0E0BD01AEE0B0E0A0
:104148000E9444CBDB01AE0FBF1F1C96EC91E068C8
:10415800EC93ABE6B4E0E12FF0E0BD01AEE0B0E0F7
:104168000E9444CBDB01AE0FBF1F1C96EC91EF7B86
:10417800EC931F5F7ECFA0916904A13000F1E0911C
:104188006904E150E0936904EF5FE0916904E0306D
:10419800B1F4E0916404F0E0F695E795E370F0700F
:1041A800309721F4E0916404E77F07C0E130A0E094
:1041B800FA0729F4E0916404E860E09364040C943D
:1041C800E625A0971A93A1E4B1E0E0E0F0E060E012
:1041D80070E00E9492CCACE6B2E0E4EFF1E00E941D
:1041E8009ACCAEE6B2E0E0E00E94A2CCAFE6B2E044
:1041F8000E94A2CCA7E7B2E0E0E10E94A2CCA0E72F
:10420800B2E0E5E00E94A2CCA1E7B2E0E0E0F0E095
:1042180060E070E00E9492CCA5E7B2E00E9486CCF4
:10422800E1600E94A2CCFE017196FA93EA93E0E065
:10423800EA93A0E1B0E00E948EC3FE013196FA93A2
:10424800EA93E0E0EA93A0E1B0E00E948EC310E0B8
:10425800143308F046C1ABE7B2E0E12FF0E0BD014E
:10426800AEE0B0E00E9444CBDB01AE0FBF1FE0E040
:10427800F0E060E070E00E9492CCABE7B2E0E12FA2
:10428800F0E0BD01AEE0B0E00E9444CBDB01AE0F30
:10429800BF1F1496E0E0F0E00E949ACCABE7B2E0D2
:1042A800E12FF0E0BD01AEE0B0E00E9444CBDB01BD
:1042B800AE0FBF1F1696E0E0F0E00E949ACCABE785
:1042C800B2E0E12FF0E0BD01AEE0B0E00E9444CBE7
:1042D800DB01AE0FBF1F1896EFEFFFEF0E949ACCDD
:1042E800ABE7B2E0E12FF0E0BD01AEE0B0E00E9444
:1042F80044CBDB01AE0FBF1F1A960E9486CCE07F2D
:10430800E6600E94A2CCABE7B2E0E12FF0E0BD018D
:10431800AEE0B0E00E9444CBDB01AE0FBF1F1A969F
:104328000E9486CCEF78E0620E94A2CCABE7B2E0B4
:10433800E12FF0E0BD01AEE0B0E00E9444CBDB012C
:10434800AE0FBF1F1A960E9486CCEF770E94A2CCB0
:10435800ABE7B2E0E12FF0E0BD01AEE0B0E00E94D3
:1043680044CBDB01AE0FBF1F1C960E9486CCEE7FAC
:104378000E94A2CCABE7B2E0E12FF0E0BD01AEE0D5
:10438800B0E00E9444CBDB01AE0FBF1F1B960E941A
:1043980086CCE07F0E94A2CCABE7B2E0E12FF0E050
:1043A800BD01AEE0B0E00E9444CBDB01AE0FBF1F01
:1043B8001B960E9486CCEF700E94A2CCABE7B2E0BD
:1043C800E12FF0E0BD01AEE0B0E00E9444CBDB019C
:1043D800AE0FBF1F1C960E9486CCED7F0E94A2CC18
:1043E800ABE7B2E0E12FF0E0BD01AEE0B0E00E9443
:1043F80044CBDB01AE0FBF1F1C960E9486CCE37F27
:104408000E94A2CCABE7B2E0E12FF0E0BD01AEE044
:10441800B0E00E9444CBDB01AE0FBF1F1C960E9488
:1044280086CCEF7E0E94A2CCABE7B2E0E12FF0E0B1
:10443800BD01AEE0B0E00E9444CBDB01AE0FBF1F70
:104448001C960E9486CCEF710E94A2CCABE7B2E02A
:10445800E12FF0E0BD01AEE0B0E00E9444CBDB010B
:10446800AE0FBF1F1D96E0E00E94A2CCFE01719620
:10447800FA93EA93E7E2F2E060E070E00E9418CC79
:10448800E12FF0E031966F2F660F660B762F0E94B2
:1044980018CC84E00E94DBC92A96E12FF0E0A0E660
:1044A800BBE30E9409CBEA0FFB1FFA93EA93FE01D4
:1044B8007396FA93EA93A0E10E94B428E12FF0E002
:1044C800A0EABEE30E940BCBEA0FFB1FFA93EA9324
:1044D800FE013396FA93EA93A8E00E94B4281F5F7E
:1044E800B7CE0E941D171881A19608951A93E3E488
:1044F800F7E0FA93EA93E0E0EA93ACE3B0E00E94D5
:104508008EC310E0143108F040C0AEEBB6E0E12FE6
:10451800F0E0BD01A6E0B0E00E9444CBDB01AE0FA5
:10452800BF1F0E9486CCE03071F1A3E01A9FF00112
:10453800ED5BF84FDF01EC91E160EC93A3E01A9F8B
:10454800F001ED5BF84FFF93EF93AEEBB6E0E12F90
:10455800F0E0BD01A6E0B0E00E9444CBDB01AE0F65
:10456800BF1F12960E9482CCDF01EEE00E94CACAE9
:10457800E370AF91BF91E370E295E07F0E2EEC916E
:10458800EF7CE029EC931F5FBDCF199108950E943D
:104598008FCA10E0143108F013C2A3E01A9FF0018B
:1045A800ED5BF84FE081E17009F408C2AEEBB6E0CC
:1045B800E12FF0E0BD01A6E0B0E00E9444CBDB01B2
:1045C800AE0FBF1F0E9486CCAE2F0E947A3B0E2FE3
:1045D800A3E01A9FF001ED5BF84FE081F0E00E9444
:1045E8001BCBE370F070309709F07AC0003009F403
:1045F8005BC01A9FF001ED5BF84FE081E47009F0B1
:1046080052C0AEEBB6E0E12FF0E0BD01A6E0B0E0AD
:104618000E9444CBDB01AE0FBF1F12960E9482CCD2
:10462800FF73AF0100240416050688F4A3E01A9F5F
:10463800F001ED5BF84FDF01EC91E860EC93A3E04B
:104648001A9FF001EC5BF84F408351832CC0A3E024
:104658001A9FF001ED5BF84FDF01EC91E77FEC93D7
:10466800A3E01A9FF001ED5BF84FDF01EC91E260E7
:10467800EC93A3E01A9FF001EC5BF84FFF93EF93E4
:10468800AEEBB6E0E12FF0E0BD01A6E0B0E00E949D
:1046980044CBDB01AE0FBF1F14960E9482CCAF91B2
:1046A800BF91ED93FC931BC0A3E01A9FF001EC5B54
:1046B800F84FA0E0B0E0A083B183A3E01A9FF00117
:1046C800ED5BF84FDF01EC91E77FEC93A3E01A9FD5
:1046D800F001ED5BF84FDF01EC91ED7FEC931DC12C
:1046E800E130A0E0FA0709F063C0A091900DAB306B
:1046F80008F413C1003041F4A3E01A9FF001ED5B08
:10470800F84FE081E47009F452C0AEEBB6E0E12F57
:10471800F0E0BD01A6E0B0E00E9444CBDB01AE0FA3
:10472800BF1F12960E9482CCFF73AF0100240416AB
:10473800050688F4A3E01A9FF001ED5BF84FDF014E
:10474800EC91E860EC93A3E01A9FF001EC5BF84F62
:10475800408351832CC0A3E01A9FF001ED5BF84F12
:10476800DF01EC91E860EC93A3E01A9FF001ED5BA8
:10477800F84FDF01EC91E260EC93A3E01A9FF0019F
:10478800EC5BF84FFF93EF93AEEBB6E0E12FF0E070
:10479800BD01A6E0B0E00E9444CBDB01AE0FBF1F15
:1047A80014960E9482CCAF91BF91ED93FC93B5C053
:1047B800E230A0E0FA0709F05EC0003041F0A3E063
:1047C8001A9FF001ED5BF84FE081E47009F052C0E8
:1047D800AEEBB6E0E12FF0E0BD01A6E0B0E00E944C
:1047E80044CBDB01AE0FBF1F12960E9482CCFF7331
:1047F800AF0100240416050688F4A3E01A9FF0010F
:10480800ED5BF84FDF01EC91E860EC93A3E01A9FB1
:10481800F001EC5BF84F408351832CC0A3E01A9F52
:10482800F001ED5BF84FDF01EC91E860EC93A3E059
:104838001A9FF001ED5BF84FDF01EC91E260EC9319
:10484800A3E01A9FF001EC5BF84FFF93EF93AEEBF8
:10485800B6E0E12FF0E0BD01A6E0B0E00E9444CB55
:10486800DB01AE0FBF1F14960E9482CCAF91BF919F
:10487800ED93FC9352C0E330A0E0FA0709F04DC075
:10488800A091900DAB3008F448C0003099F0A3E037
:104898001A9FF001ED5BF84FDF01EC91E260EC93B9
:1048A800A3E01A9FF001EC5BF84FA0E0B0E0A08312
:1048B800B18333C0A3E01A9FF001ED5BF84FE081AC
:1048C800E47059F11A9FF001ED5BF84FDF01EC91AC
:1048D800E77FEC93A3E01A9FF001ED5BF84FDF014F
:1048E800EC91E260EC93A3E01A9FF001EC5BF84FC7
:1048F800FF93EF93AEEBB6E0E12FF0E0BD01A6E049
:10490800B0E00E9444CBDB01AE0FBF1F14960E949B
:1049180082CCAF91BF91ED93FC93A3E01A9FF00175
:10492800ED5BF84FDF01E02FE170EE0FEE0F0E2E7A
:10493800EC91EB7FE029EC93AEEBB6E0E12FF0E0F1
:10494800BD01A6E0B0E00E9444CBDB01AE0FBF1F63
:1049580011960E9486CC3E2F3030A1F0A3E01A9F1A
:10496800F001ED5BF84FE081E87039F41A9FF0012F
:10497800ED5BF84FE081E27029F0A32F0E947A3BAB
:10498800E03009F41BC0A3E01A9FF001ED5BF84F7B
:10499800DF01EC91E77FEC93A3E01A9FF001ED5B58
:1049A800F84FDF01EC91ED7FEC93A3E01A9FF00143
:1049B800EC5BF84FA0E0B0E0A083B1831F5FEACDC5
:1049C8000E9496CA49C11A9310E0143108F069C0D0
:1049D800A3E01A9FF001ED5BF84FE081E17061F010
:1049E8001A9FF001EC5BF84FDF01ED91FC911197F4
:1049F80000240E160F0608F052C0A3E01A9FF0011B
:104A0800EC5BF84FDF01ED91FD913197FE93EE934A
:104A1800A3E01A9FF001EC5BF84FDF01ED91FC91E8
:104A280011973097E1F5A3E01A9FF001ED5BF84F7D
:104A3800E081E87059F11A9FF001ED5BF84FDF0152
:104A4800EC91E77FEC93A3E01A9FF001EC5BF84F41
:104A5800FF93EF93AEEBB6E0E12FF0E0BD01A6E0E7
:104A6800B0E00E9444CBDB01AE0FBF1F14960E943A
:104A780082CCAF91BF91ED93FC93A3E01A9FF00114
:104A8800ED5BF84FDF01EC91E26008C0A3E01A9FEC
:104A9800F001ED5BF84FDF01EC91ED7FEC931F5FC8
:104AA80094CF0C948F2A60971A93FE013196FA934B
:104AB800EA93E0E0EA93A0E1B0E00E948EC310E040
:104AC800143108F047C0FE013196FA93EA93E0E00A
:104AD800EA93A6E0B0E00E948EC3AEEBB6E0E12F09
:104AE800F0E0BD01A6E0B0E00E9444CBE60FF71F5E
:104AF800FA93EA93FE013396FA93EA93A6E080D0FC
:104B0800FE013196FA93EA93EEE2F2E060E070E09B
:104B18000E9418CCE12FF0E031966F2F660F660BDC
:104B2800762F0E9418CC84E00E94DBC92A96E12FD8
:104B3800F0E0A0E1B1E40E9409CBEA0FFB1FFA9371
:104B4800EA93FE013396FA93EA930E94B428A89553
:104B58001F5FB6CF1881619608951A930A93EEE302
:104B6800F2E060E070E00E9418CC80E00E9416CA73
:104B780024960FE010E0E5E4F1E00E171F0738F483
:104B8800D801E0E00E94A2CC0F5F1F4FF4CF0E9433
:104B98003B2DA0E0B0E0E0E50E94A2CCA1E0B0E0AF
:104BA800E3E40E94A2CCA2E0B0E0EDE40E94A2CC33
:104BB800A3E0B0E0E0E50E94A2CCA4E0B0E0E0E031
:104BC8000E94A2CC0991199108950E948FCA0A2FB8
:104BD8002E813F814885598510E0101778F4E12F20
:104BE800F0E0E40FF51F0F01D901EE27A10FBE1F5A
:104BF8000E9486CCD001EC931F5FEFCF0C94BA29AA
:104C08000E948FCA0A2F2E813F814885598510E05E
:104C1800101778F4E12FF0E0E40FF51F0F01D90128
:104C2800EE27A10FBE1FEC91D0010E94A2CC1F5FFE
:104C3800EFCF9CC30E9491CA0A2F2C813D8110E0BE
:104C4800101740F4D901EE27A10FBE1F0E94A2CC75
:104C58001F5FF6CF0E9498CA269608950E948FCAB1
:104C68003A2F4E815F8110E0E32FF0E03197A12FBA
:104C7800B0E0AE17BF078CF4DA01EE27A10FBE1F14
:104C88000C91003051F0A885B985EE27A10FBE1F01
:104C9800E02F0E94A2CC1F5FE7CFA885B985EE2739
:104CA800A10FBE1F0E94A2CCE12F60C30E948FCA31
:104CB8003A2F4E815F8110E0E32FF0E03197A12F6A
:104CC800B0E0AE17BF0794F4DA01EE27A10FBE1FBC
:104CD8000E9486CC0E2F003049F0E12FA885B985B7
:104CE800F0E0EA0FFB1F00831F5FE6CFA885B985B8
:104CF800EE27A10FBE1FEC93E12F38C32E97D1509A
:104D08000E9491CA10E0133030F5FE01E250FF4FC7
:104D1800FA93EA93E0E0F0E0FA93EA93A4E1B0E0D2
:104D28006CD1E03089F0E0918B0DEE7FE0938B0D34
:104D3800FE01E250FF4FFA93EA93ACEBB3E00E9416
:104D48009EC3E03041F005C0E0918B0DE160E09337
:104D58008B0D1F5FD8CF133011F42CD194C0E0E035
:104D6800F0E0E093CC03F093CD0320E030E0283E60
:104D7800E3E03E0708F059C0203DE3E03E0710F4A9
:104D880009E103C0E8EEE21B0E2FFE013496FA9308
:104D9800EA93E091CA03F091CB0360E870E0AAE0DF
:104DA800B0E00E9444CBE60FF71FFA93EA93EAE0DB
:104DB800E09FF001DF0121D1E030A1F110E01017F0
:104DC80088F52F5F3F4FAAE01A9FF001DE01149685
:104DD800AE0FBF1F1696EC91E03021F1AAE01A9FA2
:104DE800F001DE011496AE0FBF1FED91FD91A09169
:104DF800CC03B091CD03AE17BF0790F4AAE01A9F79
:104E0800F001DE011496AE0FBF1FED91FC911197D2
:104E1800E093CC03F093CD032093CA033093CB03E4
:104E28001F5FCDCF101708F0A2CFACECB3E0ED9127
:104E3800FD913196FE93EE93A091CA03B091CB03F6
:104E4800A83EE3E0BE0728F0E0E0E093CA03E09361
:104E5800CB03E5E5F2E060E070E00E9418CCE09159
:104E6800CA03F091CB03662777270E9418CCE091FC
:104E7800CC03F091CD03662777270E9418CC88E0F1
:104E88000E9416CA2C960E9498CA6296DF5F0895FF
:104E98001A931A2F1A93E0E0EA93A0E0B0E001D049
:104EA8003AC32A970E948FCA9D0108895989EAE660
:104EB800F2E060E070E00E9418CCE52FFF2766273B
:104EC80077270E9418CCE02FFF27662777270E94B4
:104ED80018CC88E00E9416CA2C96543638F0ABE7F6
:104EE800B9E00E9482CC31960E949ACCE091CC0322
:104EF800F091CD03EE83FF83E091F410F091F5106B
:104F08006091F6107091F710E887F9876A877B87B8
:104F18005C870D872E873F8710E01330A0F5E0915E
:104F2800CA03F091CB0360E870E0AAE0B0E00E9409
:104F380044CBE60FF71FFA93EA93FE013896FA93EB
:104F4800EA93AAE00DD1E030E1F0ACECB3E0ED91EA
:104F5800FD913196FE93EE93AAECB3E0ED91FD91AD
:104F68003196FE93EE93A091CA03B091CB03A83E6D
:104F7800E3E0BE0728F0E0E0E093CA03E093CB0348
:104F880002C01F5FCACF0E9496CA62960895E1E0E8
:104F9800F0E0E093CC03F093CD03E0E0E093CA03A4
:104FA800E093CB03E0E8F0E0FA93EA93A0E1B7E2FC
:104FB800E1D108956497FE01FA93EA93E0E0EA9359
:104FC800A4E1B0E00E948EC3FE01FA93EA93AEE436
:104FD800B2E080E090E00E94D6C3E2E0E887ECE02F
:104FE800E987E0E0F0E0FA93EA93FE013296FA935B
:104FF800EA93A4E1B5D0649608950E948FCAAD01E2
:1050080010E01436C0F41298EDB5E093820DE5E097
:10501800EEBDEDB5E7FFFDCFE0E0EEBDEDB5E7FF96
:10502800FDCF0EB5129A00FF06C080E991E0019706
:10503800F1F71F5FE6CF143659F4E885F985FA933E
:10504800EA93E0E0EA93DA010E948EC3E0E08EC1C1
:105058001298EDB5E093820DE3E0EEBDEDB5E7FF04
:10506800FDCFEF81F070EEBDEDB5E7FFFDCFEE812E
:10507800EEBDEDB5E7FFFDCF20E030E024173507A2
:1050880088F4EDB5E093820DE0E0EEBDEDB5E7FF05
:10509800FDCFA885B985A20FB31FEEB5EC932F5F9E
:1050A8003F4FECCF129A61C10E948FCA2A2F4E81BE
:1050B8005F8110E01436C0F41298EDB5E093820DCC
:1050C800E5E0EEBDEDB5E7FFFDCFE0E0EEBDEDB507
:1050D800E7FFFDCF3EB5129A30FF06C080E991E0A8
:1050E8000197F1F71F5FE6CF143629F4A885B98533
:1050F800E0E0EC933BC1213008F021501298EDB567
:10510800E093820DE3E0EEBDEDB5E7FFFDCFE52FBF
:10511800F070EEBDEDB5E7FFFDCF4EBDEDB5E7FF95
:10512800FDCF00E00217A0F4EDB5E093820DE0E0BA
:10513800EEBDEDB5E7FFFDCFA885B985EE27A00F39
:10514800BE1FEEB5EC93EEB5E03011F00F5FEACF7D
:10515800129AA885B985EE27A00FBE1FEC9305C14A
:105168000E948FCA5A2F10E0513008F47AC000E02C
:105178000436C0F41298EDB5E093820DE5E0EEBD7B
:10518800EDB5E7FFFDCFE0E0EEBDEDB5E7FFFDCF04
:105198003EB5129A30FF06C080E991E00197F1F719
:1051A8000F5FE6CF043611F4E0E0E0C01298EDB5E9
:1051B800E093820DE6E0EEBDEDB5E7FFFDCF129A74
:1051C800000000001298EDB5E093820DE5E0EEBD19
:1051D800EDB5E7FFFDCFE0E0EEBDEDB5E7FFFDCFB4
:1051E8003EB5129A31FF3AC0E885EF77A0E8AE1BCA
:1051F8002A2F521708F4252F1298EDB5E093820D47
:10520800E2E0EEBDEDB5E7FFFDCFE985F070EEBD5C
:10521800EDB5E7FFFDCFE885EEBDEDB5E7FFFDCFC6
:1052280000E0021780F4EDB5E093820DAE81BF81F6
:10523800EE27A10FBE1FEC91EEBDEDB5E7FFFDCF48
:105248000F5F1F5FEECF129A521BE22FF0E0A88586
:10525800B985EA0FFB1FE887F98702C0E0E086C03E
:1052680083CF83C00E948FCA5A2F10E0513008F4B0
:105278007CC000E00436C0F41298EDB5E093820DCE
:10528800E5E0EEBDEDB5E7FFFDCFE0E0EEBDEDB545
:10529800E7FFFDCF3EB5129A30FF06C080E991E0E6
:1052A8000197F1F70F5FE6CF043611F4E0E05EC036
:1052B8001298EDB5E093820DE6E0EEBDEDB5E7FF9F
:1052C800FDCF129A000000001298EDB5E093820D10
:1052D800E5E0EEBDEDB5E7FFFDCFE0E0EEBDEDB5F5
:1052E800E7FFFDCF3EB5129A31FF3CC0E885EF7766
:1052F800A0E8AE1B2A2F521708F4252F1298EDB5F7
:10530800E093820DE2E0EEBDEDB5E7FFFDCFE98564
:10531800F070EEBDEDB5E7FFFDCFE885EEBDEDB56C
:10532800E7FFFDCF00E0021780F4AE81BF81EE27D2
:10533800A10FBE1F3C91EDB5E093820D3EBDEDB5CA
:10534800E7FFFDCF0F5F1F5FEECF129A303069F095
:10535800521BE22FF0E0A885B985EA0FFB1FE8870A
:10536800F98702C0E0E002C081CFE1E00E9496CA5E
:105378002A9608950E948FCAAD0110E000240416F1
:10538800050608F07BC000E00436C0F41298EDB5BD
:10539800E093820DE5E0EEBDEDB5E7FFFDCFE0E07F
:1053A800EEBDEDB5E7FFFDCF3EB5129A30FF06C062
:1053B80080E991E00197F1F70F5FE6CF043611F429
:1053C800E0E05DC01298EDB5E093820DE6E0EEBD39
:1053D800EDB5E7FFFDCF129A000000001298EDB579
:1053E800E093820DE5E0EEBDEDB5E7FFFDCFE0E02F
:1053F800EEBDEDB5E7FFFDCF3EB5129A31FF3BC0DC
:10540800EE81EF77A0E8AE1B2A2FFA01B0E0EA1789
:10541800FB0708F4242F1298EDB5E093820DE2E023
:10542800EEBDEDB5E7FFFDCFEF81F070EEBDEDB558
:10543800E7FFFDCFEE81EEBDEDB5E7FFFDCF00E064
:10544800021758F4EDB5E093820DE0E0EEBDEDB53E
:10545800E7FFFDCF0F5F1F5FF3CF129AA22FBB2785
:105468004A1B5B0BE22FF0E0AE81BF81EA0FFB1F06
:10547800EE83FF8302C0E0E002C080CFE1E00E943B
:1054880096CA289608951A93EFE7F7E0FA93EA93F5
:10549800E0E0EA93A4E1B0E00E948EC310E015308A
:1054A800D0F5E12FAFE7B7E0F0E00E940DCBEA0FAF
:1054B800FB1F0F01AAE8B6E0E12FF0E00E940DCB38
:1054C800AE0FBF1F0E9486CCD001EC93E12FAFE74F
:1054D800B7E0F0E00E940DCBEA0FFB1F33960F01F7
:1054E800AAE8B6E0E12FF0E00E940DCBAE0FBF1F97
:1054F80013960E9486CCEE1FE0E0EE1FE170D0010B
:10550800E170EE0FEE0FEE0F0E2EEC91E77FE02923
:10551800EC931F5FC4CF199108950E9491CA2A2F56
:1055280010E0153008F0CFC1E12FAFE7B7E0F0E0A9
:105538000E940DCBAE0FBF1FAC91A03081F0E12FC0
:10554800AFE7B7E0F0E00E940DCBAE0FBF1F139698
:10555800EC91E695E695E695E1702E1709F0B1C154
:10556800E12FAFE7B7E0F0E00E940DCBAE0FBF1F11
:10557800AC910E947A3BE03009F479C0E12FAFE7A3
:10558800B7E0F0E00E940DCBAE0FBF1F1396EC9171
:10559800E47009F06BC0E12FAFE7B7E0F0E00E94DC
:1055A8000DCBAE0FBF1F1396EC91E160EC93E12F8A
:1055B800AFE7B7E0F0E00E940DCBAE0FBF1F139628
:1055C800EC91E460EC93E12FAFE7B7E0F0E00E94E4
:1055D8000DCBEA0FFB1F33960F01AAE8B6E0E12FC7
:1055E800F0E00E940DCBAE0FBF1F13960E9486CC31
:1055F800EF77E13010F0E1E001C0E0E0D001E170C8
:10560800EE0F0E2EEC91ED7FE029EC93E12FAFE742
:10561800B7E0F0E00E940DCBEA0FFB1F32960F01B6
:10562800AAE8B6E0E12FF0E00E940DCBAE0FBF1F55
:1056380013960E9486CCEF77D001EC93E12FAFE769
:10564800B7E0F0E00E940DCBEA0FFB1F31960F0187
:10565800AAE8B6E0E12FF0E00E940DCBAE0FBF1F25
:1056680011960E9486CCD001EC932BC12FC0E12F5C
:10567800AFE7B7E0F0E00E940DCBAE0FBF1F139667
:10568800EC91EB7FEC93E12FAFE7B7E0F0E00E94FD
:105698000DCBAE0FBF1F1396EC91E270B9F4E12F5A
:1056A800AFE7B7E0F0E00E940DCBAE0FBF1F139637
:1056B800EC91EE7FEC93E12FAFE7B7E0F0E00E94CA
:1056C8000DCBAE0FBF1F1196E0E0EC93E12FAFE7D3
:1056D800B7E0F0E00E940DCBAE0FBF1F1196AC9162
:1056E800A13008F4EEC0E12FAFE7B7E0F0E00E9488
:1056F8000DCBAE0FBF1F1196EC91E150EC93E12F4B
:10570800AFE7B7E0F0E00E940DCBAE0FBF1F1196D8
:10571800EC91E03009F0D5C0E12FAFE7B7E0F0E059
:105728000E940DCBAE0FBF1F1396EC91E17009F4E8
:105738008CC0E6E7F2E060E070E00E9418CCE12F50
:10574800F0E031966F2F660F660B762F0E9418CC0B
:1057580084E00E9416CA2896E12FAFE7B7E0F0E090
:105768000E940DCBAE0FBF1F1396EC91EE7FEC930A
:10577800E12FAFE7B7E0F0E00E940DCBAE0FBF1FFF
:105788001396EC91E27009F442C0E12FAFE7B7E05D
:10579800F0E00E940DCBAE0FBF1F1296AC91A13066
:1057A800A8F1E12FAFE7B7E0F0E00E940DCBAE0F14
:1057B800BF1F1296EC91E150EC93E12FAFE7B7E0F1
:1057C800F0E00E940DCBAE0FBF1F1296AC91A13036
:1057D800E8F0AAE8B6E0E12FF0E00E940DCBAE0FAA
:1057E800BF1F12960E9486CC0E2FE295EF70E695A9
:1057F800E6953E2F031BE6950E1BE12FAFE7B7E0BA
:10580800F0E00E940DCBEA0FFB1F01831DC0AAE840
:10581800B6E0E12FF0E00E940DCBAE0FBF1F12964D
:105828000E9486CC0E2FE295EF70E695E6953E2F06
:10583800031BE6950E1BE12FAFE7B7E0F0E00E94EF
:105848000DCBEA0FFB1F01833CC0EEE7F2E060E0FE
:1058580070E00E9418CCE12FF0E031966F2F660FB0
:10586800660B762F0E9418CC84E00E9416CA2896F0
:10587800E12FAFE7B7E0F0E00E940DCBAE0FBF1FFE
:105888001396EC91E160EC93AAE8B6E0E12FF0E022
:105898000E940DCBAE0FBF1F11960E9486CC0E2F13
:1058A800E295EF70E695E6953E2F031BE6950E1BF5
:1058B800E12FAFE7B7E0F0E00E940DCBEA0FFB1F46
:1058C80001831F5F2ECEC5C160971A93FE013196E2
:1058D800FA93EA93E0E0EA93A0E1B0E00E948EC375
:1058E80010E0153008F069C0AAE8B6E0E12FF0E052
:1058F8000E940DCBAE0FBF1FE0E00E94A2CCAAE829
:10590800B6E0E12FF0E00E940DCBAE0FBF1F11965D
:10591800E5E00E94A2CCAAE8B6E0E12FF0E00E9400
:105928000DCBAE0FBF1F1296E5E00E94A2CCAAE8ED
:10593800B6E0E12FF0E00E940DCBAE0FBF1F13962B
:105948000E9486CCE0780E94A2CCAAE8B6E0E12FBB
:10595800F0E00E940DCBAE0FBF1F13960E9486CCBD
:10596800EF770E94A2CCFE013196FA93EA93E5E81C
:10597800F2E060E070E00E9418CCE12FF0E0319690
:105988006F2F660F660B762F0E9418CC84E00E945A
:10599800DBC92A96E12FF0E0A0E4B0E40E9409CB2D
:1059A800EA0FFB1FFA93EA93FE013396FA93EA9300
:1059B800A0E10E94B4281F5F94CF65DD22C1E0E01A
:1059C800E2B9EFEFE1B9E1E0E5B9E7EFE4B9E8E121
:1059D800E8B9EFE9E7B9E0E2EBB9E8EBEAB9E2E008
:1059E800EEB9EEE3EDB9E0E0E1BBEFE0E0937E0075
:1059F800E0EFE0BBE0E0E4BBEFE1E3BBE1E5ECBDF9
:105A0800E1E0EDBDE6E0E093C200E8E9E093C10023
:105A1800E0E0E093C500E3E0E093C400EDE0E4BD1E
:105A2800E0E0E6BDEFE4E7BDE2E0E0936E00089554
:105A3800E0E0E093900D0E9498350E947B600E9400
:105A4800747A0E94A63A0E941D170E94F80A1BDD6C
:105A58000E947A220E94BEC00E9438B90E9423BBCD
:105A68000E94F80A0E94067F0E94EF4408956097FA
:105A78001A9310E01A3048F4A8E1B1E0EE27A10F1C
:105A8800BE1F0E94A2CC1F5FF5CFA6E2B1E00E9424
:105A980086CCE07F0E94A2CCA6E2B1E00E9486CC30
:105AA800EF7E0E94A2CCA6E2B1E00E9486CCE06222
:105AB8000E94A2CCA5E2B1E0E0E00E94A2CCA7E25D
:105AC800B1E00E94A2CCA8E2B1E00E94A2CCA9E277
:105AD800B1E00E94A2CCAAE2B1E00E94A2CCABE263
:105AE800B1E00E94A2CCACE2B1E00E94A2CCADE24F
:105AF800B1E0E4E10E94A2CCAEE2B1E0E0E00E94B5
:105B0800A2CCAFE2B1E00E94A2CCA0E3B1E00E9437
:105B1800A2CCA1E3B1E00E94A2CCFE013196FA9397
:105B2800EA93E0E0EA93A0E1B0E00E948EC3FE01B0
:105B38003196FA93EA93A3ECB3E00E94C9C3E0E07C
:105B4800F8E3FA93EA93FE013396FA93EA93A0E115
:105B58000E94B428E0E0E983E0E9F4E4FA93EA93E8
:105B6800FE013396FA93EA93A1E00E94B428A2E3D7
:105B7800B1E0EEE1F0E0FF700F010E9482CCE0702E
:105B8800F07FE029F1290E949ACCA4E3B1E0E0E09B
:105B98000E94A2CCA5E3B1E0EAE00E94A2CCA6E371
:105BA800B1E0E0E80E94A2CCA7E3B1E00E94A2CC59
:105BB800E9E3F1E0FA93EA93A7E00E941E260E9427
:105BC80040790E94B77A0E94F7430E94E5200E941C
:105BD80095167ADE0E9457250E943EC30E94A3BAFA
:105BE8000E94BBBF0E94528E0E9427780E947C466A
:105BF8000E94CB271DDFA8E0B0E0E3E00E94A2CC22
:105C08006BD11881619608950E9491CAA89522E2E5
:105C180031E000E010E02D37E9E03E0748F4D90113
:105C28000E9486CCF0E00E0F1F1F2F5F3F4FF3CF6F
:105C3800EBE9F2E060E070E00E9418CCF80166271A
:105C480077270E9418CC84E00E9416CA2896A89547
:105C5800F8010E9498CA24960895EF97EF9726971F
:105C68000E948FCAE091910DED7FE093910DEB7F3B
:105C7800E093910DE77FE093910DE0E0E093930DC1
:105C8800A8E0B0E00E9486CCE330B1F5E091910D38
:105C9800E260E093910DA2E2B1E00E9486CCE1308F
:105CA80039F5E091910DE460E093910DADDFAF011E
:105CB800A3E2B1E00E9482CCE887F987E985F0E0A9
:105CC800F0E04E1B5F0BE885F985F0E0F0E04E1B35
:105CD8005F0BE885F985E417F50731F4E091910D3C
:105CE800E860E093910D03C0E4E0E093930D03C0F6
:105CF800E2E0E093930D03C0E1E0E093930D30E020
:105D080040E050E0E2E2F1E0EE83FF83AE81BF8144
:105D1800AD37E9E0BE0708F04BC0EDE7F9E0EA1B54
:105D2800FB0BE138A0E0FA0710F010E804C0AE81E0
:105D3800EDE7EA1B1E2FFE013A96FA93EA93E2E298
:105D4800F1E0A0E0B8E20E9428CCEA1BFB0BA88592
:105D5800B985EA0FFB1FFA93EA93A12FBB270E948C
:105D68000128303071F4AA85A13031F0E091930D0B
:105D7800E061E093930D1CC0EB85FC85E887F9870B
:105D880031E000E0011760F4E02FF0E0DE011A9640
:105D9800AE0FBF1FEC91F0E04E0F5F1F0F5FF2CF09
:105DA800A895EE81FF81E058FF4FEE83FF83AECFC9
:105DB800313009F08BC0E985F0E0F0E04E1B5F0B55
:105DC800E885F985F0704E1B5F0BE885F985E417C7
:105DD800F50709F076C0E091910DE87009F070C000
:105DE800AFEFBFE00E9486CCEF5F0E94A2CCE091AB
:105DF800930DE064E093930DE2E2F1E0EE83FF831C
:105E0800AE81BF81AD37E9E0BE07B8F5EDE7F9E04F
:105E1800EA1BFB0BE138A0E0FA0710F010E804C019
:105E2800AE81EDE7EA1B1E2FFE013A96FA93EA933C
:105E3800E2E2F1E0A0E0B8E20E9428CCEA1BFB0B0A
:105E4800A885B985EA0FFB1FFA93EA93A12FBB2710
:105E58000E940128EE81FF81FA93EA93FE013C96A5
:105E6800FA93EA93A12F0E940426A895EE81FF8158
:105E7800E058FF4FEE83FF83C3CFC6DEAF01A3E236
:105E8800B1E00E9482CCE887F987E985F0E0F0E08C
:105E98004E1B5F0BE885F985F0E0F0E04E1B5F0BC9
:105EA800E885F985E417F50731F4E091910DE8608C
:105EB800E093910D05C0E091930DE068E093930D98
:105EC80005C0E091930DE062E093930D0E9496CA9D
:105ED800EF96EF962C960895EF97EF9724970E94E8
:105EE8008FCAE8EAF2E060E070E00E9418CC80E037
:105EF8000E9416CA2496A2E2B1E0E1E00E94A2CC78
:105F0800A3E2B1E0E0E0F0E00E949ACC7DDEAF01D0
:105F1800A3E2B1E00E9482CCEE83FF83EF81F0E040
:105F2800F0E04E1B5F0BEE81FF81F0E0F0E04E1BCE
:105F38005F0BA3E2B1E0FA010E949ACC22E231E0C1
:105F48002D37E9E03E0760F5EDE7F9E0E21BF30BDA
:105F5800E138A0E0FA0710F010E803C0EDE7E21B13
:105F68001E2FFE013896FA93EA933A932A93A12FAB
:105F78000E94E925E2E2F1E0A0E0B8E20E9428CC24
:105F8800EA1BFB0BE20FF31FFA93EA93FE013A9622
:105F9800FA93EA93A12F0E94B42820583F4FD0CFFC
:105FA800E091910DE460E093910DE860E093910D2C
:105FB800E0E0E093930DE091910DE07129F0E0911C
:105FC800910DE160E093910D0E9496CAEF96EF96CD
:105FD8002A960895EF97EF9722970E948FCA4A2F23
:105FE800403039F5A4E1B0E0E3E70E94A2CCA3E297
:105FF800B0E0E1E00E94A2CCA4E2B0E0E0E0F0E092
:106008000E949ACC20E030E004E110E0E8E1F1E001
:106018000E171F0748F4D8010E9486CCF0E02E0F17
:106028003F1F0F5F1F4FF2CFA4E2B0E0F9010E94BB
:106038009ACC00E010E00430E1E01E0748F5E4E007
:10604800F1E0E01BF10BE138A0E0FA0710F050E8AE
:1060580003C0E4E0E01B5E2FFE013696FA93EA9354
:10606800E4E1F0E0E00FF11FFA93EA93A52F0E9414
:10607800E925F801E058F140FA93EA93FE013896D1
:10608800FA93EA93A52F0E94B42800581F4FD3CF44
:106098000E9496CAEF96EF96289608950E948FCA96
:1060A80020E030E004E110E0E8E1F1E00E171F071E
:1060B80048F4D8010E9486CCF0E02E0F3F1F0F5FF6
:1060C8001F4FF2CFA4E2B0E00E9482CCAF01E52FCF
:1060D800F0E0F0E02E1B3F0BFA01F0E0F0E02E1BA1
:1060E8003F0B4217530711F4E1E001C0E0E00E94C2
:1060F80096CA26960895EF97EF9725970E948FCA1C
:10610800E0E0DE01A957BF4FEC93DE01A957BF4F6E
:10611800AC91AA3020F5A8E1B1E0FE01E957FF4FA4
:10612800E081F0E0AE0FBF1F0E9486CCDE01A857C9
:10613800BF4FEC93DE01A857BF4FAC91A03210F0CF
:10614800AB3730F0A8E1B1E0E0E00E94A2CC07C094
:10615800DE01A957BF4FEC91EF5FEC93D6CFE091EA
:10616800910DEF7EE093910DE0E0DE01A957BF4F5E
:10617800EC93DE01A957BF4FAC91A53038F5A0E0EC
:10618800B0E00E9486CCE035C1F4A1E0B0E00E9406
:1061980086CCE33491F4A2E0B0E00E9486CCED34E2
:1061A80061F4A3E0B0E00E9486CCE03531F4A4E0CD
:1061B800B0E00E9486CCE03009F001C007C0DE01E3
:1061C800A957BF4FEC91EF5FEC93D3CFDE01A957EE
:1061D800BF4FAC91A53039F40E94B125E091920DE2
:1061E800E160E093920DA3E2B0E00E9486CCE0303B
:1061F80061F4A4E2B0E00E9482CC309731F4A2E2CC
:10620800B0E00E9486CCEF3109F008C0E091920D11
:10621800E260E093920DA0E0DDDE0EC03FDFE030EB
:1062280031F0E091910DE061E093910D05C0E091AE
:10623800920DE460E093920DE0E0DE01AA57BF4FB3
:10624800EC93E0E0F0E08F019F010430E1E01E07ED
:1062580008F061C0E4E0F1E0E01BF10BE138A0E0F8
:10626800FA0710F0E0E802C0E4E0E01BDE01A857FE
:10627800BF4FEC93FE013696FA93EA93F801E05883
:10628800F140FA93EA93DE01A457BF4FAC91BB27C4
:106298000E940128FE01EA57FF4FE081E030A9F48F
:1062A800AE81A33719F4AD89A13009F008C04E8931
:1062B8005F89E1E0DE01AA57BF4FEC9306C0E09189
:1062C800920DE860E093920D26C0E0E0DE01A95748
:1062D800BF4FEC93FE01E857FF4FE081DE01A9575D
:1062E800BF4FAC91AE17A0F4FE01E957FF4FE08114
:1062F800F0E0DE011696AE0FBF1FEC91F0E02E0F16
:106308003F1FDE01A957BF4FEC91EF5FEC93E2CF3F
:1063180000581F4F9ACFE52FF0E0F0E02E1B3F0BFF
:10632800FA01F0E0F0E02E1B3F0BDE01AA57BF4F49
:10633800AC91A13019F44217530709F059C0E09104
:10634800910DE07109F053C0E091920DE061E09386
:10635800920D00E010E00430E1E01E0798F5EDE74B
:10636800F9E0E01BF10BE138A0E0FA0710F0E0E8F3
:1063780002C0EDE7E01BDE01A857BF4FEC93FE011A
:106388003696FA93EA93F801E058F140FA93EA93C3
:10639800DE01A457BF4FAC91BB270E940128E4E15E
:1063A800F0E0E00FF11FFA93EA93FE013896FA93B2
:1063B800EA93DE01A457BF4FAC910E94042600580F
:1063C8001F4FC9CF6BDEE03069F0E091910DE061BD
:1063D800E093910DAEEFBFE00E9486CCEF5F0E9484
:1063E800A2CC05C0E091920DE062E093920D17C037
:1063F800E091920DE064E093920DE091910DE071CF
:1064080071F0A1E0E7DDADEFBFE00E9486CCEF5F61
:106418000E94A2CCE091920DE068E093920D0E9458
:1064280096CAEF96EF962B960895E2EBF2E060E0BD
:1064380070E00E9418CCE2E0F0E060E070E00E94BA
:1064480018CCECE0F0E060E070E00E9418CCE8E0E6
:10645800F0E060E070E00E9418CC8CE00E9416CA60
:106468006096EDEDF2E060E070E00E9418CCA5E1E6
:10647800B0E00E9482CC662777270E9418CC84E07F
:106488000E9416CA2896E9EEF2E060E070E00E94E9
:1064980018CCA7E1B0E00E9486CCFF2766277727B3
:1064A8000E9418CCA8E1B0E00E9486CCFF2766279E
:1064B80077270E9418CC88E00E9416CA2C96E1E043
:1064C800F3E060E070E00E9418CCE0918D0DFF27AA
:1064D800662777270E9418CCE0918E0DFF27662744
:1064E80077270E9418CCAAE1B0E00E9486CCFF274B
:1064F800662777270E9418CC8CE00E9416CA6096FF
:10650800EFE1F3E060E070E00E9418CCE091F41055
:10651800F091F5106091F6107091F7100E9418CC68
:1065280084E00E9416CA2896E091910DE27009F461
:1065380044C0E091910DE47031F1EDE2F3E060E0E8
:1065480070E00E9418CCA3E2B1E00E9482CC6627DA
:1065580077270E9418CC84E00E9416CA2896E091FA
:10656800910DE87029F0EEE3F3E060E070E004C01C
:10657800E2E4F3E060E070E00E9418CC80E00E9462
:1065880016CA249619C0E9E4F3E060E070E00E94BE
:1065980018CCA2E2B1E00E9486CCFF2766277727B5
:1065A8000E9418CCE1E0F0E060E070E00E9418CCB6
:1065B80088E00E9416CA2C9619C0EEE5F3E060E068
:1065C80070E00E9418CCA8E0B0E00E9486CCFF27BB
:1065D800662777270E9418CCE3E0F0E060E070E0DF
:1065E8000E9418CC88E00E9416CA2C96E3E7F3E0D4
:1065F80060E070E00E9418CCAFEFBFE00E9486CC4C
:10660800FF27662777270E9418CCADEFBFE00E94CE
:1066180086CCFF27662777270E9418CCAEEFBFE00D
:106628000E9486CCFF27662777270E9418CC8CE02B
:106638000E9416CA6096E8E8F3E060E070E00E9405
:1066480018CCE091920DFF27662777270E9418CC77
:10665800E091930DFF27662777270E9418CC88E0E2
:106668000E9416CA2C960895ABE0B0E00E9486CC32
:10667800E0938D0DACE0B0E00E9486CCE0938E0DE7
:106688009ED90E94DF8F7894A1E00E942D370E9446
:106698008226A89530DDE1DAE091910DE07121F0D4
:1066A800E091910DE87009F405C0E091910DE16069
:1066B800E093910DBDD9A091F010B091F1108091A7
:1066C800F2109091F310AA3AE5E5BE07E0E08E07D4
:1066D800EFEF9E0719F4E4B7E0FF1AC0EAEAF5E520
:1066E80060E07FEFE093F010F093F1106093F21008
:1066F8007093F310E0E0F0E060E070E8E093F410ED
:10670800F093F5106093F6107093F710E093F8107B
:10671800A2E3B1E00E9482CCFF70A4E8BDE0FF7064
:106728000F01ED91FD91E070F07FE029F129FE93D2
:10673800EE93E091840DF091850DFF703A9758F42F
:10674800E091840DF091850DE070F07FEA60E093B0
:10675800840DF093850DE4B7E3FF04C0A091F81011
:10676800A03009F002C0A4E006C0E4B7E2FF02C00E
:10677800A5E001C0A2E00E944C27E0E0E4BFE0935E
:10678800F810EBE9F3E060E070E00E9418CC80E0DC
:106798000E9416CA2496F09A0ED2E091EF08E87F7C
:1067A800E260E093EF08E0916304EF7CE062E0933D
:1067B8006304E2E0E093D50CE0E0E093880DA2E307
:1067C800B1E00E9482CCFF70339770F4A2E3B1E08D
:1067D800E3E0F0E0FF700F010E9482CCE070F07FF0
:1067E800E029F1290E949ACCE091920DE03049F01D
:1067F800EAE0EA93E0E0EA93A091920DBB270E94B9
:106808005527E091930DE03049F0EBE0EA93E0E0A2
:10681800EA93A091930DBB270E945527A091E30905
:10682800A03071F4A091CE0AE091CF0AEA1741F4A2
:10683800A0917A00A03021F4A091880DA03009F031
:1068480005C0E1E0E3BF8895E0E0E3BFA091950DC6
:10685800A13060F0E091950DE150E093950DEF5F68
:10686800E091910DE07211F40E94A60B0E9482053E
:10687800A0913608A43028F00E94BA3DE0E0E093E9
:106888003608A091880DA13008F43AC1E091880D2E
:10689800E150E093880DEF5FE5E0E093950DA0E00F
:1068A800F799A1E0E1E0EA2711F4F79801C0F79A17
:1068B800F79BE5C00E94C4BD0E94D4C1E091910D30
:1068C800E072D9F4E091AB07F0E0E130A0E0FA071C
:1068D80019F40E943A4811C0E230A0E0FA0721F00A
:1068E800E330A0E0FA0719F40E94CB5406C0E43064
:1068F800A0E0FA0711F40E943C5BA1E00E94912AF3
:10690800A0E020FCA1E0E1E0EA27E894EE2309F00A
:10691800689420F820FE0FC00E9497B90E94CB22ED
:10692800E091760DE07439F0E091760DEF7BE0931D
:10693800760D0E940084A091B50DA43030F4E0914A
:10694800B50DEF5FE093B50D91C0E0E0E093B50DB4
:10695800A0E021FCA1E0E1E0EA27E894EE2309F0B9
:10696800689421F821FE82C0A895A091900DAF3FB0
:1069780030F4E091900DEF5FE093900DE150A0911D
:10698800940DA13060F0E091940DE150E093940DE6
:10699800EF5FE091940DE03011F4A0E01BDBA091D3
:1069A800830DA13030F0E091830DE150E093830D29
:1069B80016C0E4E0E093830DA5EEB8E00A2EEC9152
:1069C800E695E170A1E0EA27A02DE170EE0F0E2E0A
:1069D800EC91ED7FE029EC93E0E0E093E208A091F0
:1069E8003508A03131F4E0D00E9400840E94136D74
:1069F80011C0E0913308EF70E13060F0A3E3B8E034
:106A080080E0EFE00E944CCCE0913308E061E09335
:106A1800330801C0D0D00E94D0BC0E946A420E94B4
:106A280025200E9400C3A0E00E94912A0E946512BE
:106A38000E94E724E091AB07F0E0E130A0E0FA071C
:106A480011F40E943E4F0E94EA8F0E94E40AA0912E
:106A5800B60DA93030F4E091B60DEF5FE093B60DB6
:106A680005C0E0E0E093B60D0E944ABDE091760DC6
:106A7800EF7BE093760D0E94E06A0E949537E091E3
:106A8800890DF0918A0D7096E093890DF0938A0D27
:106A9800A091890DB0918A0DA533ECE0BE07F0F006
:106AA800E091890DF0918A0DE553FC40E093890D42
:106AB800F0938A0DA4EFB0E1ED91FD916D917D9178
:106AC800EF5FFF4F6F4F7F4F7E936E93FE93EE9372
:106AD8000E94F97A0E9498770E94C438E09133089E
:106AE800E07121F0A0913508A03109F009C0E091CA
:106AF8003308EF7EE093330857D00E94136D5BD0C4
:106B08000E9448908BCEFFCFEA93EFB7EA93E1E07B
:106B1800E093870DE091880DEF5FE093880DE150D9
:106B2800E991EFBFE99118950E9491CA10E01031E0
:106B3800B8F5A2E3B0E0E12FF0E0BD01AAE0B0E0D3
:106B48000E9444CBDB01AE0FBF1F0E9482CC0E9483
:106B58001DCB9F012030E1E03E0788F0E4EAF3E036
:106B680060E070E00E9418CCF901662777270E9440
:106B780018CC84E00E9416CA28962FEF30E0ADEAC0
:106B8800B8E0E12FFF2766277727E054FF4F6F4FC4
:106B98006BBFE691F0E0EA0FFB1F20831F5FC7CFB2
:106BA8000E9498CA24960895E6E8E0937A00E0E007
:106BB800E09332080895E6E8E0937A00E0E9E8B95E
:106BC800E0E0E0937C00E0933408E0933508E1E0EE
:106BD800E0933208E1E4F8E0FA93EA93E0E0EA931C
:106BE800A4E3B0E00E948EC3E9E7F8E0FA93EA93E1
:106BF800E0E0EA93AAE1B0E00E948EC3E3E9F8E09E
:106C0800FA93EA93E0E0EA93AAE1B0E00E948EC327
:106C1800E7ECF8E0FA93EA93E0E0EA93AAE1B0E05F
:106C28000E948EC3EEEDE0937A00E0913308E07F96
:106C3800E560E093330808950A921A928A93AA931A
:106C4800BA93EA93FA93EFB7EA93E0913208F0E047
:106C5800E130A0E0FA0739F4EFECE0937A00E2E0E3
:106C6800E0933208ECC0E230A0E0FA0709F0E7C090
:106C780046B0E0913408EF5FE0933408E150A0910A
:106C88003408A731D0F4E0913408E770E869E8B92E
:106C9800A83010F443980AC0A0913408A03110F429
:106CA800449804C0E3E0E0937C004798EEECE0935E
:106CB8007A00E1E0E093320835C0A0913408A731AA
:106CC80061F4E1E0E0937C00E8E9E8B980E58A95C1
:106CD800F1F7EFECE0937A0025C0A0913408A831D1
:106CE80051F4E2E0E0937C0080E58A95F1F7EFEC5F
:106CF800E0937A0017C0E0E9E8B9E0E0E0933408EF
:106D0800E0937C00EEECE0937A00E1E0E093320857
:106D1800A0913508A03130F4E0913508EF5FE09399
:106D28003508E150A0913408A13010F0A83108F0DE
:106D38002DC0E0913408E770E093B70DA7E3B8E001
:106D4800F0E0EA0FFB1F4082E091B70DE03031F42C
:106D5800E0913608EF5FE0933608E150A9E7B8E024
:106D6800E0913408F0E0AE0FBF1FEC91E429EC93FA
:106D7800A3E9B8E0E0913408F0E0EA0FFB1F0F0147
:106D8800A081E42DE095EA2BD001EC93A091350881
:106D9800A03108F054C0ADEAB8E0E0913408F0E062
:106DA800AE0FBF1FEC91E093B70DE0917800F09122
:106DB8007900A091B70DB0E0AE17BF0798F4A1E431
:106DC800B8E0E0913408F0E0EE0FFF1FEA0FFB1F78
:106DD8000F01DF01ED91FD91DF01E0917800F09165
:106DE800790011C0A1E4B8E0E0913408F0E0EE0FBA
:106DF800FF1FEA0FFB1F0F01DF01ED91FD91DF017E
:106E0800E091B70DF0E0EA0FFB1FD001ED93FC9382
:106E1800A0913408A13140F4A0917800B091790094
:106E2800A03FE3E0BE0708F40AC0A7ECB8E0E09191
:106E38003408F0E0AE0FBF1FEC91EF5FEC93E991DF
:106E4800EFBFF991E991B991A991899119900990A8
:106E580018951A931A2F103041F05C988BE08A9598
:106E6800F1F75C9A8BE08A95F1F72898EDB5E093F5
:106E7800820DE0E4EEBDEDB5E7FFFDCFE5E0EEBD48
:106E8800EDB5E7FFFDCFE8E0EEBDEDB5E7FFFDCFDF
:106E9800289AE091E508EF7BE093E508A5E7B2E0E2
:106EA8000E9486CCE170A5EEB8E0E170E795E0E0DD
:106EB800E7950E2EEC91EF77E029EC93E091E50849
:106EC800E860E093E508E460E093E5082898EDB50C
:106ED800E093820DE0E4EEBDEDB5E7FFFDCFEAE01B
:106EE800EEBDEDB5E7FFFDCFE091E508EEBDEDB5F0
:106EF800E7FFFDCF289A2898EDB5E093820DE0E4EE
:106F0800EEBDEDB5E7FFFDCFE0E0EEBDEDB5E7FF87
:106F1800FDCFE4E0EEBDEDB5E7FFFDCF289A0C9478
:106F2800783BA091E208A13030F0E091E208E1500E
:106F3800E093E20818C0E3E6E093E2082898EDB58C
:106F4800E093820DE0E4EEBDEDB5E7FFFDCFEAE0AA
:106F5800EEBDEDB5E7FFFDCFE091E508EEBDEDB57F
:106F6800E7FFFDCF289AA091E308A13038F0E0911F
:106F7800E308E150E093E308EF5F2DC0E3E6E09318
:106F8800E3082898EDB5E093820DE2E4EEBDEDB597
:106F9800E7FFFDCFEAE0EEBDEDB5E7FFFDCFE091FD
:106FA800E708EEBDEDB5E7FFFDCF289A2898EDB5C7
:106FB800E093820DE2E4EEBDEDB5E7FFFDCFE0E042
:106FC800EEBDEDB5E7FFFDCFE091E608EEBDEDB50E
:106FD800E7FFFDCF289AA091E408A13038F0E091AE
:106FE800E408E150E093E408EF5F2DC0E3E6E093A6
:106FF800E4082898EDB5E093820DE4E4EEBDEDB524
:10700800E7FFFDCFEAE0EEBDEDB5E7FFFDCFE0918C
:10701800E908EEBDEDB5E7FFFDCF289A2898EDB554
:10702800E093820DE4E4EEBDEDB5E7FFFDCFE0E0CF
:10703800EEBDEDB5E7FFFDCFE091E808EEBDEDB59B
:10704800E7FFFDCF289A08950E9491CA589A509A4E
:10705800E091EA08E07CE093EA08E9B1E370E33004
:10706800A9F0E0E0E093BC0010E0E9B1E370E330A0
:1070780011F01A3008F00AC058988BE08A95F1F799
:10708800589A8BE08A95F1F71F5FEFCFEFE0E09316
:10709800B800E4EAE093BC0020E030E0E091BC00F6
:1070A800E07821F42436E0E03E0708F003C02F5FC3
:1070B8003F4FF4CFE091B900E87FE83009F052C0C3
:1070C800E0E9E093BB00E4E8E093BC0020E030E0B6
:1070D800E091BC00E07821F42436E0E03E0708F0B7
:1070E80003C02F5F3F4FF4CFE091B900E87FE8314C
:1070F800C9F5E1E0E093BB00E4E8E093BC0020E0E0
:1071080030E0E091BC00E07821F42436E0E03E076E
:1071180008F003C02F5F3F4FF4CFE091B900E87F3C
:10712800E83201F5E1E6E093BB00E4E9E093BC0056
:1071380020E030E0E091BC00E07821F42436E0E083
:107148003E0708F003C02F5F3F4FF4CFE091B9002E
:10715800E87FE83239F4E0E0E093BC0058985098B2
:107168000C94B63DE4E9E093BC00A2E0B0E00E94D4
:107178005ACEE0E0E093BC00589850980C94B63D85
:107188000E948FCAE091EA08EF73E13030F0AAEE6E
:10719800B8E080E0EFE30E944CCC589A509AE9B1ED
:1071A800E370E330A9F0E0E0E093BC0010E0E9B15F
:1071B800E370E33011F01A3008F00AC058988BE0F9
:1071C8008A95F1F7589A8BE08A95F1F71F5FEFCF10
:1071D800E091EA08EF7309F0D1C0E091EA08E07C99
:1071E800E560E093EA08EFE0E093B800E4EAE093B2
:1071F800BC0020E030E0E091BC00E07821F42436C7
:10720800E0E03E0708F003C02F5F3F4FF4CFE09166
:10721800B900E87FE83009F088C1E0E9E093BB00F5
:10722800E4E8E093BC0020E030E0E091BC00E078C6
:1072380021F42436E0E03E0708F003C02F5F3F4FFB
:10724800F4CFE091B900E87FE83109F06EC1E1E0E0
:10725800E093BB00E4E8E093BC0020E030E0E0917C
:10726800BC00E07821F42436E0E03E0708F003C0D3
:107278002F5F3F4FF4CFE091B900E87FE83209F083
:1072880054C1E0E6E093BB00E4E8E093BC0020E0F2
:1072980030E0E091BC00E07821F42436E0E03E07DD
:1072A80008F003C02F5F3F4FF4CFE091B900E87FAB
:1072B800E83209F03AC1E4EAE093BC0020E030E0AB
:1072C800E091BC00E07821F42436E0E03E0708F0C5
:1072D80003C02F5F3F4FF4CFE091B900E87FE03162
:1072E80009F023C1E0E9E093BB00E4E8E093BC00C7
:1072F80020E030E0E091BC00E07821F42436E0E0C2
:107308003E0708F003C02F5F3F4FF4CFE091B9006C
:10731800E87FE83109F009C1E0E0E093BB00E4E868
:10732800E093BC0020E030E0E091BC00E07821F47C
:107338002436E0E03E0708F003C02F5F3F4FF4CF4C
:10734800E091B900E87FE83209F0EFC0E4E9E093A2
:10735800BC0020E030E0E091BC00E07821F4243665
:10736800E0E03E0708F003C02F5F3F4FF4CFE09105
:10737800EA08E07CEE61E093EA08D6C0E4EAE0932C
:10738800BC0020E030E0E091BC00E07821F4243635
:10739800E0E03E0708F003C02F5F3F4FF4CFE091D5
:1073A800B900E87FE83009F0C0C0E1E9E093BB002C
:1073B800E4E8E093BC0020E030E0E091BC00E07835
:1073C80021F42436E0E03E0708F003C02F5F3F4F6A
:1073D800F4CFE091B900E87FE03409F0A6C0E4EC0E
:1073E800E093BC0020E030E0E091BC00E07821F4BC
:1073F8002436E0E03E0708F003C02F5F3F4FF4CF8C
:10740800E091B900E87FE03509F08FC04091BB00FA
:107418005527E4E8E093BC00FA010E9409CBAF01CC
:1074280020E030E0E091BC00E07821F42436E0E090
:107438003E0708F003C02F5F3F4FF4CFE091B9003B
:10744800E87FE83509F071C0E091BB00F0E00E94E8
:1074580012CB4E2B5F2BE4E9E093BC0053FD506F39
:1074680020E030E0E091BC00E07821F42436E0E050
:107478003E0708F003C02F5F3F4FF4CF4093EC085E
:107488005093ED08A091EC08B091ED08E0E1F0E030
:107498000E949DCBE0938F0DA6E3B1E00E9486CCBD
:1074A8000E2FE2EEE017E4F4E0919C0DE03089F055
:1074B800A0918F0DE02FF0E0E7FDFFEF3197B0E0EE
:1074C800A7FDBFEFAE17BF071CF4E0E0E0939C0DEB
:1074D80007C0A0918F0DA0171CF0E1E0E0939C0D70
:1074E800A7E3B1E00E9486CC0E2FE2EEE017E4F4A9
:1074F800E0919D0DE03089F0A0918F0DE02FF0E034
:10750800E7FDFFEF3197B0E0A7FDBFEFAE17BF076C
:107518001CF4E0E0E0939D0D07C0A0918F0DA0172B
:107528001CF0E1E0E0939D0D09C0E091EA08E07CE1
:10753800E560E093EA08E4E9E093BC000E9496CA9B
:10754800269608951A93F298F398F498F598E0918E
:107558007E00E97FE0937E00E3E9F7E0FA93EA939F
:10756800E0E0EA93ACE0B0E00E948EC310E01C308B
:1075780008F04EC0E12FF0E0ED56F84F0F01AAEBEE
:10758800B1E0EE27A10FBE1F0E9486CCE370D001A8
:10759800E370EE0FEE0F0E2EEC91E37FE029EC93F3
:1075A800E12FF0E0ED56F84F0F01AAEBB1E0EE271E
:1075B800A10FBE1F0E9486CCE695E695E170D0012A
:1075C800E170EE0F0E2EEC91ED7FE029EC93E12FA8
:1075D800F0E0ED56F84FE081F0E00E941FCBE37039
:1075E800F070309741F4123011F0133011F4F49A1E
:1075F80001C0F29A0BC0E130A0E0FA0739F412306A
:1076080011F0133011F4F59A01C0F39A1F5FAFCF50
:10761800E0919507EC70E83031F0AEECB1E00E94F3
:1076280086CCE37051F0E0917E00E260E0937E004A
:10763800E1E0E0933F08F59AF498E0919607EC7042
:10764800E83031F0AEECB1E00E9486CCEC7051F03D
:10765800E0917E00E460E0937E00E1E0E093400882
:10766800F59AF498F29B02C0F39B01C002C0169AE7
:1076780001C01698F49B02C0F59B01C002C0159A80
:1076880001C0159831C01A93ECEBF3E060E070E0AC
:107698000E9418CC80E00E9416CA249610E01C3084
:1076A80000F5E4ECF3E060E070E00E9418CCE12F14
:1076B800F0E031966F2F660F660B762F0E9418CC7C
:1076C800E12FF0E0ED56F84FE081E170FF276627E3
:1076D80077270E9418CC88E00E9416CA2C961F5F54
:1076E800DECFAAE00E942590199108950E9491CAC0
:1076F8003A2FE091910DE17009F433C2373310F05D
:107708003C3308F006C0E32FF0E0F797E957F64F4F
:107718003081313059F4A091990DB0919A0DA0376C
:10772800E7E1BE0710F0E1E01DC21BC2333010F0E4
:107738003F3008F008C0E32FF0E03397ED56F84FDC
:10774800E081E1700FC23F3010F03F3108F020C0F7
:107758003F31E8F4E32FF0E03F97A9E0B0E00E9462
:1077680044CBE950F74FE081E17079F0E32FF0E086
:107778003F97A9E0B0E00E9444CBE950F74FE08181
:10778800E077E03410F4E1E001C0E0E0EBC1E9C1EA
:107798003C3310F0303708F014C0ABE6B4E0E32F08
:1077A800F0E0FC97BD01AEE0B0E00E9444CBDB0105
:1077B800AE0FBF1F1C96EC91EE1FE0E0EE1FE170CC
:1077C800D1C1303710F0343808F011C0A6EDBCE054
:1077D800E32FF0E0E057F0400E940BCBAE0FBF1F45
:1077E800EC91E295EF70E695E695E170BBC134380F
:1077F80010F0383908F00EC0E32FF0E0E458F040FC
:10780800A3E0B0E00E9444CBED5BF84FE081E69541
:10781800E170A8C1383910F03D3908F00EC0E32FE7
:10782800F0E0E859F040AFE7B7E00E940DCBAE0FAB
:10783800BF1F1396EC91E17095C13D39B9F4E09101
:10784800760DEF70E33079F0E091760DEF70E4306B
:1078580051F0E091760DEF70E13029F0E091760D6E
:10786800EF70E63011F4E1E07DC17BC13E3969F487
:10787800E091760DEF70E53029F0E091760DEF702C
:10788800E23011F4E1E06EC16CC13F3910F0373BD2
:1078980008F06FC0E32FEF591E2FFF2766277727C1
:1078A800EA5DFE4F6F4F6BBF0691E12FFF276627FA
:1078B8007727E25CFE4F6F4F6BBF1691113449F585
:1078C800A3E00A9FF001E453F64FE081E07FE03146
:1078D80011F4E1E047C1A3E00A9FF001E453F64F39
:1078E800E081E07FE03288F00A9FF001E453F64F30
:1078F800E081E770E33041F00A9FF001E453F64F6E
:10790800E081E770E43009F401C002C0E1E02AC177
:107918002FC0123401F5A3E00A9FF001E453F64F9B
:10792800E081E07FE03211F4E1E01CC1A3E00A9FAE
:10793800F001E453F64FE081E07FE03340F00A9F26
:10794800F001E453F64FE081E770E43009F002C03B
:10795800E1E008C10DC0133459F4A3E00A9FF00117
:10796800E453F64FE081E07FE03311F4E1E0FAC040
:10797800F8C03A3B10F0363C08F009C0E32FEA5B48
:107988000E2FF0E0E156F84FE081E170EBC0373C94
:1079980010F03F3D08F0BEC0E091AB07F0E0E130E9
:1079A800A0E0FA0709F04CC03F3C88F4E32FE75CFD
:1079B8001E2FA1E0B0E00E94B9CAA091B507B0E0BF
:1079C800EA23FB23309711F0E1E0CCC038C0333D07
:1079D80088F4E32FEF5C1E2FA1E0B0E00E94B9CA43
:1079E800A091B607B0E0EA23FB23309711F0E1E05D
:1079F800B9C025C03B3D88F4E32FE35D1E2FA1E00D
:107A0800B0E00E94B9CAA091CE07B0E0EA23FB23F8
:107A1800309711F0E1E0A6C012C03F3D80F4E32F9B
:107A2800EB5D1E2FA1E0B0E00E94B9CAA091CF077C
:107A3800B0E0EA23FB23309711F0E1E093C069C07E
:107A4800E230A0E0FA0721F0E330A0E0FA0789F479
:107A5800A2EDB7E0E32FF0E0E75CF0400E940DCB29
:107A6800AE0FBF1F1296EC91E17011F0E1E07AC001
:107A780050C0E430A0E0FA0709F04BC03F3C88F45E
:107A8800E32FE75C1E2FA1E0B0E00E94B9CAA091E5
:107A9800B307B0E0EA23FB23309711F0E1E062C0BE
:107AA80038C0333D88F4E32FEF5C1E2FA1E0B0E02F
:107AB8000E94B9CAA091B607B0E0EA23FB23309729
:107AC80011F0E1E04FC025C03B3D88F4E32FE35DB2
:107AD8001E2FA1E0B0E00E94B9CAA091DB07B0E078
:107AE800EA23FB23309711F0E1E03CC012C03F3D90
:107AF80080F4E32FEB5D1E2FA1E0B0E00E94B9CA2D
:107B0800A091DE07B0E0EA23FB23309711F0E1E013
:107B180029C027C03F3D39F4E0919C0DE03011F0B9
:107B2800E1E020C01EC0303E39F4E0919D0DE03008
:107B380011F0E1E017C015C0323059F4A5E3B1E007
:107B48000E9486CCA091900DAE1710F0E1E00AC01B
:107B580008C0313E31F4E0916404E87011F0E1E0CE
:107B680001C0E0E00E9498CA2496089523970E94D5
:107B78008FCAF39904C0F59902C022FE01C003C060
:107B8800689422F89FC4F09B10C0E0919307E170BD
:107B98004E2FE0919407E170E887E0919507E17036
:107BA800EF83E0919607E170EE8322FE48C0E091F2
:107BB8009307EC7009F042C0E0919307E295EF70EB
:107BC8001E2F669B02C0F19B01C01FC0123010F42B
:107BD8001F5F1AC01230B9F4E0919307E27071F098
:107BE800E0919307E17021F0E0919307EE7F03C0E5
:107BF800E0919307E160E093930705C0E091930754
:107C0800E160E09393071FE00EC01B3010F01150A5
:107C18000AC0E0919307E27029F4E0919307EE7FA0
:107C2800E093930710E0E12FEF70E295E07F0E2ECE
:107C3800E0919307EF70E029E093930745C0E09146
:107C48009307EC70E43009F03FC0E0919307E295A8
:107C5800EF701E2F669B0FC01B3010F011500AC02A
:107C6800E0919307E27029F4E0919307EE7FE093A7
:107C7800930710E01EC0123010F41F5F1AC01230B4
:107C8800B9F4E0919307E27071F0E0919307E17025
:107C980021F0E0919307EE7F03C0E0919307E16044
:107CA800E093930705C0E0919307E160E0939307A1
:107CB8001FE0E12FEF70E295E07F0E2EE091930731
:107CC800EF70E029E093930722FE4AC0E091940701
:107CD800EC7009F044C0E0919407E295EF701E2F14
:107CE800679B02C0F19B01C021C0123010F41F5FD6
:107CF8001CC01230C9F4E0919407E27081F0E09161
:107D08009407E17031F0A4E9B7E0EC91EE7FEC93D1
:107D180005C0E0919407E160E093940705C0E09105
:107D28009407E160E09394071FE00EC01B3010F049
:107D380011500AC0E0919407E27029F4A4E9B7E071
:107D4800EC91EE7FEC9310E0A4E9B7E0E12FEF703F
:107D5800E295E07F0E2EEC91EF70E029EC9347C09E
:107D6800E0919407EC70E43009F041C0E091940789
:107D7800E295EF701E2F679B0FC01B3010F011505B
:107D88000AC0E0919407E27029F4A4E9B7E0EC9105
:107D9800EE7FEC9310E020C0123010F41F5F1CC07F
:107DA8001230C9F4E0919407E27081F0E0919407F1
:107DB800E17031F0A4E9B7E0EC91EE7FEC9305C0F7
:107DC800E0919407E160E093940705C0E09194077F
:107DD800E160E09394071FE0A4E9B7E0E12FEF70BA
:107DE800E295E07F0E2EEC91EF70E029EC93E091A4
:107DF8009507EC70E83009F03FC0E0917508F09104
:107E0800760834960E941DCB5E2FE0919507E29587
:107E1800EF701E2FA8ECB1E00E9486CC3E2FA9EC93
:107E2800B1E00E9486CC2E2F321728F5E0919507F5
:107E3800E17089F0351768F0143010F41F5F08C03E
:107E4800143031F4A5E9B7E0EC91EE7FEC9310E043
:107E580001C010E010C0521768F0123010F41F5F14
:107E680008C0123031F4E0919507E160E09395077E
:107E780010E001C010E085C022FE47C0E0919507E0
:107E8800EC7009F041C0E0919507E295EF701E2F64
:107E9800799B0FC01B3010F011500AC0E091950774
:107EA800E27029F4A5E9B7E0EC91EE7FEC9310E0DD
:107EB80020C0123010F41F5F1CC01230C9F4E091CA
:107EC8009507E27081F0E0919507E17031F0A5E93E
:107ED800B7E0EC91EE7FEC9305C0E0919507E16087
:107EE800E093950705C0E0919507E160E093950759
:107EF8001FE0A5E9B7E0E12FEF70E295E07F0E2ED5
:107F0800EC91EF70E029EC9347C0E0919507EC7095
:107F1800E43009F041C0E0919507E295EF701E2F1B
:107F2800799B21C0123010F41F5F1CC01230C9F4B5
:107F3800E0919507E27081F0E0919507E17031F0EA
:107F4800A5E9B7E0EC91EE7FEC9305C0E0919507C9
:107F5800E160E093950705C0E0919507E160E09343
:107F680095071FE00EC01B3010F011500AC0E091B9
:107F78009507E27029F4A5E9B7E0EC91EE7FEC9360
:107F880010E0A5E9B7E0E12FEF70E295E07F0E2E53
:107F9800EC91EF70E029EC93E0919607EC70E830F3
:107FA80009F03FC0E0917708F091780834960E9474
:107FB8001DCB5E2FE0919607E295EF701E2FACEC7B
:107FC800B1E00E9486CC3E2FADECB1E00E9486CC99
:107FD8002E2F321728F5E0919607E17089F03517B2
:107FE80068F0143010F41F5F08C0143031F4A6E9AB
:107FF800B7E0EC91EE7FEC9310E001C010E010C008
:10800800521768F0123010F41F5F08C0123031F4B4
:10801800E0919607E160E093960710E001C010E058
:1080280085C022FE47C0E0919607EC7009F041C078
:10803800E0919607E295EF701E2F7A9B0FC01B30D8
:1080480010F011500AC0E0919607E27029F4A6E9F1
:10805800B7E0EC91EE7FEC9310E020C0123010F402
:108068001F5F1CC01230C9F4E0919607E27081F0DE
:10807800E0919607E17031F0A6E9B7E0EC91EE7F68
:10808800EC9305C0E0919607E160E093960705C080
:10809800E0919607E160E09396071FE0A6E9B7E054
:1080A800E12FEF70E295E07F0E2EEC91EF70E02962
:1080B800EC9347C0E0919607EC70E43009F041C0BA
:1080C800E0919607E295EF701E2F7A9B21C012303F
:1080D80010F41F5F1CC01230C9F4E0919607E270DB
:1080E80081F0E0919607E17031F0A6E9B7E0EC91F4
:1080F800EE7FEC9305C0E0919607E160E093960768
:1081080005C0E0919607E160E09396071FE00EC076
:108118001B3010F011500AC0E0919607E27029F464
:10812800A6E9B7E0EC91EE7FEC9310E0A6E9B7E0A2
:10813800E12FEF70E295E07F0E2EEC91EF70E029D1
:10814800EC93F09B5FC0E0919307E170E41791F026
:10815800EBECF3E060E070E00E9418CCE09193074C
:10816800E170FF27662777270E9418CC84E00E94D9
:1081780016CA2896E0919407E170A885EA1791F04D
:10818800E5EDF3E060E070E00E9418CCE091940720
:10819800E170FF27662777270E9418CC84E00E94A9
:1081A80016CA2896E0919507E170AF81EA1791F019
:1081B800EFEDF3E060E070E00E9418CCE0919507E5
:1081C800E170FF27662777270E9418CC84E00E9479
:1081D80016CA2896E0919607E170AE81EA1791F0E9
:1081E800E9EEF3E060E070E00E9418CCE0919607B9
:1081F800E170FF27662777270E9418CC84E00E9449
:1082080016CA289654E05C3008F028C1E52FF0E043
:10821800ED56F84FE081E1704E2F22FE85C0E52F24
:10822800F0E0ED56F84FE081EC7009F07CC0A7E370
:10823800B8E0E52FFF2766277727EC56FF4F6F4FEB
:108248006BBFE691F0E0AE0FBF1FEC91E0720E2F0E
:10825800F19B02C000E011C0A7E3B8E0E52FFF27BB
:1082680066277727EC56FF4F6F4F6BBFE691F0E01C
:10827800AE0FBF1FEC91E0720E2FE52FF0E0ED5628
:10828800F84FE081E295EF701E2F003061F1123057
:1082980010F41F5F27C0123021F5E52FF0E0ED56EE
:1082A800F84FE081E270B1F0E52FF0E0ED56F84FBD
:1082B800E081E17039F0A52FB0E0AD56B84FEC91F0
:1082C800EE7F06C0A52FB0E0AD56B84FEC91E16047
:1082D800EC9307C0A52FB0E0AD56B84FEC91E16024
:1082E800EC931FE013C01B3010F011500FC0E52FA6
:1082F800F0E0ED56F84FE081E27039F4A52FB0E0D8
:10830800AD56B84FEC91EE7FEC9310E0A52FB0E09E
:10831800AD56B84FE12FEF70E295E07F0E2EEC914D
:10832800EF70E029EC9370C0E52FF0E0ED56F84FC0
:10833800E081EC70E43009F067C0A7E3B8E0E52F0E
:10834800FF2766277727EC56FF4F6F4F6BBFE691E5
:10835800F0E0AE0FBF1FEC91E0720E2FE52FF0E0BA
:10836800ED56F84FE081E295EF701E2F0030A1F036
:108378001B3010F011500FC0E52FF0E0ED56F84F0C
:10838800E081E27039F4A52FB0E0AD56B84FEC911A
:10839800EE7FEC9310E02BC0123010F41F5F27C063
:1083A800123021F5E52FF0E0ED56F84FE081E2704C
:1083B800B1F0E52FF0E0ED56F84FE081E17039F0CB
:1083C800A52FB0E0AD56B84FEC91EE7F06C0A52FB3
:1083D800B0E0AD56B84FEC91E160EC9307C0A52F23
:1083E800B0E0AD56B84FEC91E160EC931FE0A52FDB
:1083F800B0E0AD56B84FE12FEF70E295E07F0E2E5A
:10840800EC91EF70E029EC93F09B26C0E52FF0E0AB
:10841800ED56F84FE081E170E417F1F0E3EFF3E097
:1084280060E070E00E9418CCE52FF0E031966F2FE5
:10843800660F660B762F0E9418CCE52FF0E0ED56FC
:10844800F84FE081E170FF27662777270E9418CC54
:1084580088E00E9416CA2C965F5FD5CEF39B06C0B3
:10846800F29904C0F59B02C0F49B01C002C0E894D5
:1084780014C0F39906C0F29B04C0F59902C0F499A0
:1084880001C002C0689409C0A0E022FCA1E0E1E0BC
:10849800EA27E894EE2309F0689422F8F39B02C0D7
:1084A800F29901C005C022FE02C0169A01C01698B2
:1084B800F59B02C0F49901C005C022FE02C0159ABE
:1084C80001C015980E9496CA2996089524970E947B
:1084D8008FCAAEECB1E00E9486CCE3703E2F3030FC
:1084E80009F4B9C0AFECB1E00E9486CC2E2FA0ED04
:1084F800B1E00E9486CC5E2F313029F4E0917508F6
:10850800F091760804C0E0917708F09178083496E5
:108518000E941FCBE887F98710E0163008F09BC04F
:10852800A1EDB1E0EE27A10FBE1F0E9486CC0E2F51
:10853800013008F48EC0F0E0EE83FF83EE0FFF1FDA
:10854800EE83FF83E12FF0E0E156F84FE081E17020
:1085580009F443C0E22FF0E0A885B985AE0FBF1F2C
:10856800EE27A50FBE1FEE81FF81AE17BF0778F07B
:10857800E22FF0E0AE81BF81AE0FBF1FE52FF0E024
:10858800EA0FFB1FA885B985EA17FB0728F5F09BBA
:108598001CC0EEEFF3E060E070E00E9418CCE12F21
:1085A800F0E031966F2F660F660B762F0E9418CC7D
:1085B800A889B989EAE00E946CCB662777270E94D0
:1085C80018CC88E00E9416CA2C96A12FB0E0A156BC
:1085D800B84FEC91EE7FEC933CC0E22FF0E0A88519
:1085E800B985AE0FBF1FEE81FF81AE17BF0758F0E8
:1085F800E22FF0E0AE81BF81EA0FFB1FA885B985A5
:10860800EA17FB0708F425C0F09B1CC0E2E1F4E080
:1086180060E070E00E9418CCE12FF0E031966F2FF7
:10862800660F660B762F0E9418CCA889B989EAE0F4
:108638000E946CCB662777270E9418CC88E00E949E
:1086480016CA2C96A12FB0E0A156B84FEC91E16064
:10865800EC931F5F62CFAEECB1E00E9486CCE6954A
:10866800E695E3703E2F303009F4B9C0AFECB1E0C5
:108678000E9486CC2E2FA0EDB1E00E9486CC5E2F02
:10868800313029F4E0917508F091760804C0E09142
:108698007708F091780834960E941FCBE887F9870D
:1086A80016E01C3008F09BC0A1EDB1E0EE27A10F49
:1086B800BE1F0E9486CC0E2F013008F48EC0F0E059
:1086C800EE83FF83EE0FFF1FEE83FF83E12FF0E0C1
:1086D800E156F84FE081E17009F443C0E22FF0E081
:1086E800A885B985AE0FBF1FEE27A50FBE1FEE8167
:1086F800FF81AE17BF0778F0E22FF0E0AE81BF81AF
:10870800AE0FBF1FE52FF0E0EA0FFB1FA885B98564
:10871800EA17FB0728F5F09B1CC0EEEFF3E060E0DA
:1087280070E00E9418CCE12FF0E031966F2F660FB1
:10873800660B762F0E9418CCA889B989EAE00E94B6
:108748006CCB662777270E9418CC88E00E9416CA4F
:108758002C96A12FB0E0A156B84FEC91EE7FEC9388
:108768003CC0E22FF0E0A885B985AE0FBF1FEE81AF
:10877800FF81AE17BF0758F0E22FF0E0AE81BF814E
:10878800EA0FFB1FA885B985EA17FB0708F425C07F
:10879800F09B1CC0E2E1F4E060E070E00E9418CCBD
:1087A800E12FF0E031966F2F660F660B762F0E944F
:1087B80018CCA889B989EAE00E946CCB662777278C
:1087C8000E9418CC88E00E9416CA2C96A12FB0E00F
:1087D800A156B84FEC91E160EC931F5F62CF0E9405
:1087E80096CA2A96089560971A93FE013196FA93CD
:1087F800EA93E0E0EA93A0E1B0E00E948EC310E0C3
:108808001C3008F03FC0AAEBB1E0EE27A10FBE1F55
:108818000E9486CCEC7F0E94A2CCAAEBB1E0EE27A6
:10882800A10FBE1F0E9486CCEB7F0E94A2CCFE0146
:108838003196FA93EA93E5E2F4E060E070E00E9492
:1088480018CCE12FF0E031966F2F660F660B762F6C
:108858000E9418CC84E00E94DBC92A96E12FF0E040
:10886800A0E6B9E30E9409CBEA0FFB1FFA93EA934B
:10887800FE013396FA93EA93A0E10E94B428A895E2
:108888001F5FBECFA6ECB1E0E0E00E94A2CCA7EC4F
:10889800B1E0EAEF0E94A2CCA8ECB1E0E4E60E94C5
:1088A800A2CCA9ECB1E0E6E90E94A2CCAAECB1E026
:1088B800E0E00E94A2CCABECB1E0EAEF0E94A2CCCF
:1088C800ACECB1E0E4E60E94A2CCADECB1E0E6E9A4
:1088D8000E94A2CCAEECB1E00E9486CCEC7F0E9454
:1088E800A2CCAEECB1E00E9486CCE37F0E94A2CC81
:1088F800AEECB1E00E9486CCEF700E94A2CCAFEC47
:10890800B1E0E8E10E94A2CCA0EDB1E0E2E00E9473
:10891800A2CCE1EDF1E0FA93EA93ACE00E941E26C6
:1089280010E0163008F054C0FE013196FA93EA932D
:10893800EFE2F4E060E070E00E9418CCE12FF0E094
:1089480031966F2F660F660B762F0E9418CC84E045
:108958000E94DBC92A96E12FF0E0A0EDB3E40E9463
:1089680009CBEA0FFB1FFA93EA93FE013396FA93B9
:10897800EA93A0E10E94B428FE013196FA93EA93A3
:10898800EBE3F4E060E070E00E9418CCE12FF0E047
:1089980031966F2F660F660B762F0E9418CC84E0F5
:1089A8000E94DBC92A96E12FF0E03696A0EDB3E4E9
:1089B8000E9409CBEA0FFB1FFA93EA93FE01339654
:1089C800FA93EA93A0E10E94B428A8951F5FA9CF63
:1089D8001881619608950E948FCAEBEAF7E0FA932E
:1089E800EA93E0E0EA93A7E8B0E00E948EC3A8E328
:1089F800B1E00E9486CCE093AB07E8E4F4E060E0E5
:108A080070E00E9418CC80E00E9416CA2496E0917B
:108A1800AB07F0E0E130A0E0FA0709F028C100E078
:108A2800023008F007C1A9E2B8E0E02FF0E0BD018C
:108A3800A1E7B0E00E9444CBDB01AE0FBF1F0E944C
:108A480086CCE03009F4F4C0ACEAB7E0E02FF0E0FF
:108A5800BD01A9E1B0E00E9444CBE60FF71FFF93E8
:108A6800EF93A9E2B8E0E02FF0E0BD01A1E7B0E0A4
:108A78000E9444CBDB01AE0FBF1F11960E9486CC2B
:108A8800E295EF70AF91BF91EF770E2EEC91E07801
:108A9800E029EC93ACEAB7E0E02FF0E0BD01A9E1F2
:108AA800B0E00E9444CBDB01AE0FBF1F1296E5E099
:108AB800EC9331E0E0E01E2F5E2F2E2F183008F0E7
:108AC80040C0A9E2B8E0E02FF0E0BD01A1E7B0E0C6
:108AD8000E9444CBDB01AE0FBF1F1E96E12FF0E0D2
:108AE8000E940BCBAE0FBF1F16960E9486CCF0E0FB
:108AF800F695E795E370F070E130A0E0FA0721F011
:108B0800E330A0E0FA0709F4232BA9E2B8E0E02F4C
:108B1800F0E0BD01A1E7B0E00E9444CBDB01AE0F5D
:108B2800BF1F1E96E12FF0E00E940BCBAE0FBF1FB8
:108B380016960E9486CCE17009F0532B1F5F330F05
:108B4800BDCFACEAB7E0E02FF0E0BD01A9E1B0E0AD
:108B58000E9444CBE60FF71F2187ACEAB7E0E02F6D
:108B6800F0E0BD01A9E1B0E00E9444CBE60FF71F99
:108B7800558331E0E0E05E2F2E2F1C3008F040C016
:108B8800A9E2B8E0E02FF0E0BD01A1E7B0E00E9463
:108B980044CBDB01AE0FBF1F1E96E12FF0E00E9411
:108BA8000BCBAE0FBF1F16960E9486CCF0E0F69551
:108BB800E795E370F070E130A0E0FA0721F0E330C8
:108BC800A0E0FA0709F4232BA9E2B8E0E02FF0E0CF
:108BD800BD01A1E7B0E00E9444CBDB01AE0FBF1F8F
:108BE8001E96E12FF0E00E940BCBAE0FBF1F16962A
:108BF8000E9486CCE17009F0532B1F5F330FBDCF65
:108C0800ACEAB7E0E02FF0E0BD01A9E1B0E00E94D6
:108C180044CBE60FF71F2287ACEAB7E0E02FF0E07D
:108C2800BD01A9E1B0E00E9444CBE60FF71F5683CF
:108C38000F5FF6CEE0E5F4E060E070E00E9418CC4B
:108C4800A9E2B8E00E9486CCFF27662777270E9412
:108C580018CCAAE9B8E00E9486CCFF2766277727B8
:108C68000E9418CC88E00E9416CA2C963DC0E230BB
:108C7800A0E0FA0769F4E1E6F4E060E070E00E9441
:108C880018CC80E00E9416CA24960E94F2502CC08C
:108C9800E330A0E0FA0769F4E3E7F4E060E070E0AD
:108CA8000E9418CC80E00E9416CA24960E94F250B6
:108CB8001BC0E430A0E0FA0769F4E3E8F4E060E000
:108CC80070E00E9418CC80E00E9416CA24960E9488
:108CD80052590AC0EBE8F4E060E070E00E9418CC5A
:108CE80080E00E9416CA24960E9496CA2696089585
:108CF800E0E0E093AB07A8E3B1E00E94A2CC0895BE
:108D0800BA93AA9323970E948FCAA985BA85EC9132
:108D1800E07109F0A7C1E985FA85A181EFE7EA23A7
:108D28003E2F303009F49EC100E0023008F09AC1AD
:108D3800A9E2B8E0E02FF0E0BD01A1E7B0E00E94B1
:108D480044CBDB01AE0FBF1F0E9486CC3E1709F053
:108D580087C1ACEAB7E0E02FF0E0BD01A9E1B0E0DF
:108D68000E9444CBDB01AE0FBF1F1296EAE0EC93E2
:108D7800E985FA85A181B281E7E00E94CACAEE833B
:108D8800F0E0EE30A0E0FA0709F46AC1E330A0E0B1
:108D9800FA0709F065C1ACEAB7E0E02FF0E0BD01E1
:108DA800A9E1B0E00E9444CBDB01AE0FBF1FEC91FC
:108DB800E07889F5ACEAB7E0E02FF0E0BD01A9E181
:108DC800B0E00E9444CBDB01AE0FBF1FEC91E0681E
:108DD800EC93ACEAB7E0E02FF0E0BD01A9E1B0E028
:108DE8000E9444CBDB01AE0FBF1F1196E0E0EC936D
:108DF800E2E9F4E060E070E00E9418CCE02FF0E0D7
:108E080031966F2F660F660B762F0E9418CC84E080
:108E18000E9416CA2896ACEAB7E0E02FF0E0BD0140
:108E2800A9E1B0E00E9444CBDB01AE0FBF1F129650
:108E3800E1E1EC93ACEAB7E0E02FF0E0BD01A9E195
:108E4800B0E00E9444CBE60FF71F4185ACEAB7E0DB
:108E5800E02FF0E0BD01A9E1B0E00E9444CBDB01C6
:108E6800AE0FBF1F1796EC91E887ACEAB7E0E02F8A
:108E7800F0E0BD01A9E1B0E00E9444CBDB01AE0FF8
:108E8800BF1F1596EC91EF83E985FA85258110E0DF
:108E980051E0183008F5E52FAF81EA2391F0E52F6E
:108EA800E22349F0E52FA885EA2321F44527E52F99
:108EB800EA2BE88705C0E52FE095A885EA23E8872F
:108EC80008C0E52FE22311F0452B03C0E52FE095FC
:108ED8004E231F5F550FDDCFACEAB7E0E02FF0E07F
:108EE800BD01A9E1B0E00E9444CBDB01AE0FBF1F7A
:108EF8001996AC914A17D9F0ACEAB7E0E02FF0E048
:108F0800BD01A9E1B0E00E9444CBE60FF71F4187FD
:108F1800ACEAB7E0E02FF0E0BD01A9E1B0E00E94C3
:108F280044CBDB01AE0FBF1F1396E0E0EC93ACEA35
:108F3800B7E0E02FF0E0BD01A9E1B0E00E9444CB2A
:108F4800E60FF71F3796A885A083ACEAB7E0E02FB5
:108F5800F0E0BD01A9E1B0E00E9444CBE60FF71FA5
:108F68004285ACEAB7E0E02FF0E0BD01A9E1B0E04E
:108F78000E9444CBDB01AE0FBF1F1896EC91E88727
:108F8800ACEAB7E0E02FF0E0BD01A9E1B0E00E9453
:108F980044CBDB01AE0FBF1F1696EC91EF83E9853A
:108FA800FA85268110E051E0143008F5E52FAF81ED
:108FB800EA2391F0E52FE22349F0E52FA885EA237B
:108FC80021F44527E52FEA2BE88705C0E52FE09532
:108FD800A885EA23E88708C0E52FE22311F0452B8E
:108FE80003C0E52FE0954E231F5F550FDDCFACEA98
:108FF800B7E0E02FF0E0BD01A9E1B0E00E9444CB6A
:10900800DB01AE0FBF1F1A96AC914A17D9F0ACEA34
:10901800B7E0E02FF0E0BD01A9E1B0E00E9444CB49
:10902800E60FF71F4287ACEAB7E0E02FF0E0BD019A
:10903800A9E1B0E00E9444CBDB01AE0FBF1F13963D
:10904800E0E0EC93ACEAB7E0E02FF0E0BD01A9E185
:10905800B0E00E9444CBE60FF71F3896A885A0839E
:109068000F5F63CE0E9496CA2B9608956F970E9451
:109078008FCAE0916304E07409F4F8C640E0423016
:1090880008F0F4C6ACEAB7E0E42FF0E0BD01A9E1CE
:10909800B0E00E9444CBDB01AE0FBF1F1296AC912B
:1090A800A13008F4E1C6ACEAB7E0E42FF0E0BD0176
:1090B800A9E1B0E00E9444CBDB01AE0FBF1FEC91E9
:1090C800EF775E2FACEAB7E0E42FF0E0BD01A9E14D
:1090D800B0E00E9444CBDB01AE0FBF1F1396AC91EA
:1090E800A13080F0ACEAB7E0E42FF0E0BD01A9E1DF
:1090F800B0E00E9444CBDB01AE0FBF1F1396EC918A
:10910800E150A7C4ACEAB7E0E42FF0E0BD01A9E163
:10911800B0E00E9444CBDB01AE0FBF1F1396E4E022
:10912800EC93FE013C96FA93EA93E0E0EA93A6E01A
:10913800B0E00E948EC3FE013696FA93EA93E0E00F
:10914800EA93A6E0B0E00E948EC320E0E1E0EE8B57
:10915800E0E1ED8B251708F003C400E030E0A9E258
:10916800B8E0E42FF0E0BD01A1E7B0E00E9444CBF5
:10917800DB01AE0FBF1F1E96E22FF0E00E940BCB63
:10918800AE0FBF1F15960E9486CC1E2FA12F0E94DE
:1091980087783E2F3030E9F4A9E2B8E0E42FF0E018
:1091A800BD01A1E7B0E00E9444CBDB01AE0FBF1FB9
:1091B8001E96E22FF0E00E940BCBAE0FBF1F149655
:1091C8000E9486CC1E2F103021F0A12F0E94877894
:1091D8003E2F3030E9F4A9E2B8E0E42FF0E0BD0119
:1091E800A1E7B0E00E9444CBDB01AE0FBF1F1E9683
:1091F800E22FF0E00E940BCBAE0FBF1F13960E9428
:1092080086CC1E2F103021F0A12F0E9487783E2F88
:10921800303009F4C4C0E32FF0E0E130A0E0FA07F1
:1092280029F5A9E2B8E0E42FF0E0BD01A1E7B0E03C
:109238000E9444CBDB01AE0FBF1F1C960E9486CC58
:10924800E295E7700E2FA9E2B8E0E42FF0E0BD0147
:10925800A1E7B0E00E9444CBDB01AE0FBF1F1C9614
:109268000E9486CCEE1FE0E0EE1F96C0E230A0E040
:10927800FA07F9F4A9E2B8E0E42FF0E0BD01A1E7AC
:10928800B0E00E9444CBDB01AE0FBF1F1C960E94CA
:1092980086CCE7700E2FA9E2B8E0E42FF0E0BD011C
:1092A800A1E7B0E00E9444CBDB01AE0FBF1F1C96C4
:1092B8006EC0E330A0E0FA0729F5A9E2B8E0E42F90
:1092C800F0E0BD01A1E7B0E00E9444CBDB01AE0FA6
:1092D800BF1F1B960E9486CCE295E7700E2FA9E26D
:1092E800B8E0E42FF0E0BD01A1E7B0E00E9444CB74
:1092F800DB01AE0FBF1F1B960E9486CCEE1FE0E07D
:10930800EE1F4AC0E430A0E0FA07F9F4A9E2B8E099
:10931800E42FF0E0BD01A1E7B0E00E9444CBDB01FF
:10932800AE0FBF1F1B960E9486CCE7700E2FA9E2D6
:10933800B8E0E42FF0E0BD01A1E7B0E00E9444CB23
:10934800DB01AE0FBF1F1B9622C0E530A0E0FA0775
:1093580029F5A9E2B8E0E42FF0E0BD01A1E7B0E00B
:109368000E9444CBDB01AE0FBF1F1D960E9486CC26
:10937800E7700E2FA9E2B8E0E42FF0E0BD01A1E705
:10938800B0E00E9444CBDB01AE0FBF1F1D960E94C8
:1093980086CCE695E695E695E170EF8BF0C0A9E2FC
:1093A800B8E0E42FF0E0BD01A1E7B0E00E9444CBB3
:1093B800DB01AE0FBF1F1E96E22FF0E00E940BCB21
:1093C800AE0FBF1F12960E9486CC1E2F103029F0B8
:1093D800A12F0E947A3BE03009F42EC0A9E2B8E040
:1093E800E42FF0E0BD01A1E7B0E00E9444CBDB012F
:1093F800AE0FBF1F1E96E22FF0E00E940BCBAE0F00
:10940800BF1F17960E9486CCE295E7700E2FA9E23F
:10941800B8E0E42FF0E0BD01A1E7B0E00E9444CB42
:10942800DB01AE0FBF1F1E96E22FF0E00E940BCBB0
:10943800AE0FBF1F17969CC0A9E2B8E0E42FF0E07A
:10944800BD01A1E7B0E00E9444CBDB01AE0FBF1F16
:109458001E96E22FF0E00E940BCBAE0FBF1F1196B5
:109468000E9486CC1E2F103029F0A12F0E947A3B33
:10947800E03009F432C0A9E2B8E0E42FF0E0BD0121
:10948800A1E7B0E00E9444CBDB01AE0FBF1F1E96E0
:10949800E22FF0E00E940BCBAE0FBF1F17960E9481
:1094A80086CCE7700E2FA9E2B8E0E42FF0E0BD010A
:1094B800A1E7B0E00E9444CBDB01AE0FBF1F1E96B0
:1094C800E22FF0E00E940BCBAE0FBF1F17960E9451
:1094D80086CCE695E695E69550C0A9E2B8E0E42F7B
:1094E800F0E0BD01A1E7B0E00E9444CBDB01AE0F84
:1094F800BF1F1E96E22FF0E00E940BCBAE0FBF1FDE
:109508000E9486CC1E2F103029F0A12F0E947A3B92
:10951800E03009F434C0A9E2B8E0E42FF0E0BD017E
:10952800A1E7B0E00E9444CBDB01AE0FBF1F1E963F
:10953800E22FF0E00E940BCBAE0FBF1F16960E94E1
:1095480086CCE295E7700E2FA9E2B8E0E42FF0E0B0
:10955800BD01A1E7B0E00E9444CBDB01AE0FBF1F05
:109568001E96E22FF0E00E940BCBAE0FBF1F16969F
:109578000E9486CCEE1FE0E0EE1FE170EF8BEF89D2
:10958800E03009F4C9C0E02FF0E0E130A0E0FA07CC
:1095980081F4283028F4EE89AE81EA2BEE8308C0E6
:1095A800FE0137960F01E081AE89EA2BD001EC93DA
:1095B800B2C0E230A0E0FA0771F4243018F4FE01DA
:1095C800379602C0FE0138960F01E081AD89EA2B7B
:1095D800D001EC93A0C0E330A0E0FA0771F4283082
:1095E80018F4FE01399602C0FE013A960F01E08197
:1095F800AE89EA2BD001EC938EC0E430A0E0FA07E4
:10960800E9F4283028F4EE89AE81EA2BEE8308C00D
:10961800FE0137960F01E081AE89EA2BD001EC9369
:10962800243018F4FE01379602C0FE0138960F0167
:10963800E081AD89EA2BD001EC936DC0E530A0E064
:10964800FA07D9F4243018F4FE01379602C0FE0157
:1096580038960F01E081AD89EA2BD001EC932830D0
:1096680018F4FE01399602C0FE013A960F01E08116
:10967800AE89EA2BD001EC934EC0E630A0E0FA07A1
:10968800E9F4283028F4EE89AE81EA2BEE8308C08D
:10969800FE0137960F01E081AE89EA2BD001EC93E9
:1096A800283018F4FE01399602C0FE013A960F01DF
:1096B800E081AE89EA2BD001EC932DC0E730A0E021
:1096C800FA0749F5283028F4EE89AE81EA2BEE83B3
:1096D80008C0FE0137960F01E081AE89EA2BD00160
:1096E800EC93243018F4FE01379602C0FE01389638
:1096F8000F01E081AD89EA2BD001EC93283018F4F2
:10970800FE01399602C0FE013A960F01E081AE894A
:10971800EA2BD001EC9312C1593008F047C0E02F72
:10972800F0E0E130A0E0FA0729F4EE89AC85EA2BF5
:10973800EC873BC0E230A0E0FA0719F4FE013D9641
:109748002EC0E330A0E0FA0741F1E430A0E0FA07C8
:1097580039F4EE89AC85EA2BEC87FE013D961FC0F3
:10976800E530A0E0FA0789F0E630A0E0FA0729F42E
:10977800EE89AC85EA2BEC8710C0E730A0E0FA0749
:10978800A1F4EE89AC85EA2BEC87FE013D960F012A
:10979800E081AE89EA2BD001EC93FE013E960F01E1
:1097A800E081AE89EA2BD001EC93C8C0E02FF0E04D
:1097B800E130A0E0FA0781F4283028F4EE89AC857E
:1097C800EA2BEC8708C0FE013D960F01E081AE89C7
:1097D800EA2BD001EC93B2C0E230A0E0FA0771F4B2
:1097E800243018F4FE013D9602C0FE013E960F019A
:1097F800E081AD89EA2BD001EC93A0C0E330A0E072
:10980800FA0771F4283018F4FE013F9602C0FE01F1
:1098180070960F01E081AE89EA2BD001EC938EC0DF
:10982800E430A0E0FA07E9F4283028F4EE89AC85A2
:10983800EA2BEC8708C0FE013D960F01E081AE8956
:10984800EA2BD001EC93243018F4FE013D9602C0B7
:10985800FE013E960F01E081AD89EA2BD001EC9321
:109868006DC0E530A0E0FA07D9F4243018F4FE0101
:109878003D9602C0FE013E960F01E081AD89EA2BBC
:10988800D001EC93283018F4FE013F9602C0FE0187
:1098980070960F01E081AE89EA2BD001EC934EC09F
:1098A800E630A0E0FA07E9F4283028F4EE89AC8520
:1098B800EA2BEC8708C0FE013D960F01E081AE89D6
:1098C800EA2BD001EC93283018F4FE013F9602C031
:1098D800FE0170960F01E081AE89EA2BD001EC936E
:1098E8002DC0E730A0E0FA0749F5283028F4EE89C2
:1098F800AC85EA2BEC8708C0FE013D960F01E0819C
:10990800AE89EA2BD001EC93243018F4FE013D9681
:1099180002C0FE013E960F01E081AD89EA2BD0011D
:10992800EC93283018F4FE013F9602C0FE017096B1
:109938000F01E081AE89EA2BD001EC93EE89EE0F9E
:10994800EE8BED89EE0FED8BEE89E03011F4E1E05E
:10995800EE8BED89E03011F4E1E0ED8B2F5FFACB6F
:10996800ACEAB7E0E42FF0E0BD01A9E1B0E00E9465
:1099780044CBE60FF71F3B96FA93EA93FE013E9617
:10998800FA93EA93A6E0B0E00E9463C3E03029F1BD
:10999800ACEAB7E0E42FF0E0BD01A9E1B0E00E9435
:1099A80044CBE60FF71F3B96FA93EA93FE013E96E7
:1099B800FA93EA93A6E0B0E00E947CC3ACEAB7E071
:1099C800E42FF0E0BD01A9E1B0E00E9444CBDB0147
:1099D800AE0FBF1F5796E0E0EC93ACEAB7E0E42F78
:1099E800F0E0BD01A9E1B0E00E9444CBE60FF71F0B
:1099F8007196FA93EA93FE013896FA93EA93A6E0F1
:109A0800B0E00E9463C3E03029F1ACEAB7E0E42F8C
:109A1800F0E0BD01A9E1B0E00E9444CBE60FF71FDA
:109A28007196FA93EA93FE013896FA93EA93A6E0C0
:109A3800B0E00E947CC3ACEAB7E0E42FF0E0BD01DF
:109A4800A9E1B0E00E9444CBDB01AE0FBF1F5896DE
:109A5800E0E0EC93ACEAB7E0E42FF0E0BD01A9E167
:109A6800B0E00E9444CBDB01AE0FBF1F1496AC914F
:109A7800A13088F0ACEAB7E0E42FF0E0BD01A9E13D
:109A8800B0E00E9444CBDB01AE0FBF1F1496EC91EF
:109A9800E150EC9324C1ACEAB7E0E42FF0E0BD015B
:109AA800A9E1B0E00E9444CBDB01AE0FBF1F57967F
:109AB800AC91A13080F0ACEAB7E0E42FF0E0BD0152
:109AC800A9E1B0E00E9444CBDB01AE0FBF1F58965E
:109AD800AC91A13008F403C1ACEAB7E0E42FF0E0A0
:109AE800BD01A9E1B0E00E9444CBDB01AE0FBF1F6E
:109AF8001496E4E6EC93A9E2B8E0E42FF0E0BD01A7
:109B0800A1E7B0E00E9444CBDB01AE0FBF1F179660
:109B18000E9486CCAE2F0E947A3BE03081F1A9E208
:109B2800B8E0E42FF0E0BD01A1E7B0E00E9444CB2B
:109B3800DB01AE0FBF1F18960E9486CCEC8BA9E202
:109B4800B8E0E42FF0E0BD01A1E7B0E00E9444CB0B
:109B5800DB01AE0FBF1F1A960E9486CCE295EF700C
:109B6800EB8BA9E2B8E0E42FF0E0BD01A1E7B0E09B
:109B78000E9444CBDB01AE0FBF1F199671C0A9E24A
:109B8800B8E0E42FF0E0BD01A1E7B0E00E9444CBCB
:109B9800DB01AE0FBF1F14960E9486CCAE2F0E9429
:109BA8007A3BE03079F1A9E2B8E0E42FF0E0BD01BA
:109BB800A1E7B0E00E9444CBDB01AE0FBF1F1596B2
:109BC8000E9486CCEC8BA9E2B8E0E42FF0E0BD015E
:109BD800A1E7B0E00E9444CBDB01AE0FBF1F1A968D
:109BE8000E9486CCEF70EB8BA9E2B8E0E42FF0E09E
:109BF800BD01A1E7B0E00E9444CBDB01AE0FBF1F5F
:109C080016962EC0A9E2B8E0E42FF0E0BD01A1E766
:109C1800B0E00E9444CBDB01AE0FBF1F12960E943A
:109C280086CCEC8BA9E2B8E0E42FF0E0BD01A1E717
:109C3800B0E00E9444CBDB01AE0FBF1F11960E941B
:109C480086CCEF70EB8BA9E2B8E0E42FF0E0BD0121
:109C5800A1E7B0E00E9444CBDB01AE0FBF1F139613
:109C68000E9486CCEA8BE88DE07FE160E88FEF7E8A
:109C7800E88FA9E2B8E0E42FF0E0BD01A1E7B0E089
:109C88000E9444CBDB01AE0FBF1F0E9486CCF0E0E0
:109C9800F460E98FFA8FEA89ED8FDE0158960E9409
:109CA8002D09E88DE07FE260E88FA9E2B8E0E42FB3
:109CB800F0E0BD01A1E7B0E00E9444CBDB01AE0FAC
:109CC800BF1F0E9486CCF0E0F560E98FFA8FEC891F
:109CD800ED8FEB89EE8FDE0158960E942D095930E1
:109CE80010F0E6E001C0E3E0EF700E2EE88DE07FB3
:109CF800E029E88FEF7EE88FACEAB7E0E42FF0E0E8
:109D0800BD01A9E1B0E00E9444CBDB01AE0FBF1F4B
:109D18005796AC91A13088F0ACEAB7E0E42FF0E0B8
:109D2800BD01A9E1B0E00E9444CBDB01AE0FBF1F2B
:109D38005796EC91E150EC933BC0ACEAB7E0E42FC6
:109D4800F0E0BD01A9E1B0E00E9444CBDB01AE0F19
:109D5800BF1F5796EAEFEC93A9E2B8E0E42FF0E0D2
:109D6800BD01A1E7B0E00E9444CBDB01AE0FBF1FED
:109D78000E9486CCF0E0F260E98FFA8FFE017D96B2
:109D8800FA93EA93ACEAB7E0E42FF0E0BD01A9E169
:109D9800B0E00E9444CBE60FF71F3B96FA93EA9394
:109DA800A6E0B0E00E947CC3DE0158960E942D090F
:109DB800ACEAB7E0E42FF0E0BD01A9E1B0E00E9411
:109DC80044CBDB01AE0FBF1F5896AC91A13088F091
:109DD800ACEAB7E0E42FF0E0BD01A9E1B0E00E94F1
:109DE80044CBDB01AE0FBF1F5896EC91E150EC93CA
:109DF8003BC0ACEAB7E0E42FF0E0BD01A9E1B0E078
:109E08000E9444CBDB01AE0FBF1F5896EAEFEC93DC
:109E1800A9E2B8E0E42FF0E0BD01A1E7B0E00E94BC
:109E280044CBDB01AE0FBF1F0E9486CCF0E0F3608D
:109E3800E98FFA8FFE017D96FA93EA93ACEAB7E0D0
:109E4800E42FF0E0BD01A9E1B0E00E9444CBE60FA9
:109E5800F71F7196FA93EA93A6E0B0E00E947CC3DC
:109E6800DE0158960E942D094F5F09C90E9496CAC3
:109E7800A59608952D970E9491CAE0916304E07415
:109E880009F4A8C100E0023008F0A4C1A9E2B8E0D2
:109E9800E02FF0E0BD01A1E7B0E00E9444CBDB0178
:109EA800AE0FBF1F0E9486CCE03081F4ACEAB7E069
:109EB800E02FF0E0BD01A9E1B0E00E9444CBDB0156
:109EC800AE0FBF1F1296E0E0EC9382C1ACEAB7E098
:109ED800E02FF0E0BD01A9E1B0E00E9444CBDB0136
:109EE800AE0FBF1F1296AC91A13008F46CC0ACEA5B
:109EF800B7E0E02FF0E0BD01A9E1B0E00E9444CB5B
:109F0800DB01AE0FBF1F1296EC91E150EC93ACEA67
:109F1800B7E0E02FF0E0BD01A9E1B0E00E9444CB3A
:109F2800DB01AE0FBF1F1196AC91A13088F0ACEAEF
:109F3800B7E0E02FF0E0BD01A9E1B0E00E9444CB1A
:109F4800DB01AE0FBF1F1196EC91E150EC933AC0C4
:109F5800ACEAB7E0E02FF0E0BD01A9E1B0E00E9473
:109F680044CBDB01AE0FBF1F1196E2E3EC93EC810B
:109F7800E07FE860EC83EF7EEC83A9E2B8E0E02FB5
:109F8800F0E0BD01A1E7B0E00E9444CBDB01AE0FD9
:109F9800BF1F0E9486CCF0E0F660ED83FE83EBE203
:109FA800E987E0E0EA87E8E1EB87E5E0EC87E4EFC2
:109FB800ED87E1E0EE87E0E0EF87E88BDE011496BD
:109FC8000E942D0905C1ACEAB7E0E02FF0E0BD0121
:109FD800A9E1B0E00E9444CBDB01AE0FBF1FEC91BA
:109FE800E07809F4C8C0ACEAB7E0E02FF0E0BD01C2
:109FF800A9E1B0E00E9444CBDB01AE0FBF1FEC919A
:10A00800EF773E2FACEAB7E0E02FF0E0BD01A9E121
:10A01800B0E00E9444CBDB01AE0FBF1FEC91EF779D
:10A02800EC93E2EAF4E060E070E00E9418CCE02FE4
:10A03800F0E031966F2F660F660B762F0E9418CCD2
:10A0480084E00E9416CA289621E010E0131708F051
:10A0580047C0A9E2B8E0E02FF0E0BD01A1E7B0E019
:10A068000E9444CBDB01AE0FBF1F1E96E12FF0E02C
:10A078000E940BCBAE0FBF1F16960E9486CCF0E055
:10A08800F695E795E370F070309799F4ACEAB7E08D
:10A09800E02FF0E0BD01A9E1B0E00E9444CBE60F5B
:10A0A800F71F39960F01A081E22FE095EA23D0012E
:10A0B80013C0E130A0E0FA0781F4ACEAB7E0E02F82
:10A0C800F0E0BD01A9E1B0E00E9444CBDB01AE0F96
:10A0D800BF1F1996EC91E22BEC931F5F220FB6CFAE
:10A0E80021E0131708F047C0A9E2B8E0E02FF0E03C
:10A0F800BD01A1E7B0E00E9444CBDB01AE0FBF1F5A
:10A108001E96E12FF0E00E940BCBAE0FBF1F1696F4
:10A118000E9486CCF0E0F695E795E370F0703097F2
:10A1280099F4ACEAB7E0E02FF0E0BD01A9E1B0E0B6
:10A138000E9444CBE60FF71F3A960F01A081E22F49
:10A14800E095EA23D00113C0E130A0E0FA0781F4DA
:10A15800ACEAB7E0E02FF0E0BD01A9E1B0E00E9471
:10A1680044CBDB01AE0FBF1F1A96EC91E22BEC93A8
:10A178001F5F220FB6CFACEAB7E0E02FF0E0BD01D9
:10A18800A9E1B0E00E9444CBDB01AE0FBF1F1296DD
:10A19800EAE0EC93EC81E07FE260EC83EF7EEC8315
:10A1A800E0E0ED83EE83E1E0E987A9E2B8E0E02FA3
:10A1B800F0E0BD01A1E7B0E00E9444CBDB01AE0FA7
:10A1C800BF1F0E9486CCEA87DE0114960E942D09E3
:10A1D8000F5F59CE0E9498CA619608950E9491CA4D
:10A1E80010E0133008F081C0AEEAB7E0E12FF0E0EC
:10A1F800BD01ACE0B0E00E9444CBE60FF71F3196FA
:10A20800FF93EF93A9E2B8E0E12FF0E0BD01AAE0E7
:10A21800B0E00E9444CBDB01AE0FBF1F0E9486CC8A
:10A22800AF91BF91EC93AEEAB7E0E12FF0E0BD014A
:10A23800ACE0B0E00E9444CBE60FF71F3296FF93E4
:10A24800EF93A9E2B8E0E12FF0E0BD01AAE0B0E0A9
:10A258000E9444CBDB01AE0FBF1F11960E9486CC33
:10A26800AF91BF91EC93AEEAB7E0E12FF0E0BD010A
:10A27800ACE0B0E00E9444CBE60FF71F3596FF93A1
:10A28800EF93A9E2B8E0E12FF0E0BD01AAE0B0E069
:10A298000E9444CBDB01AE0FBF1F12960E9486CCF2
:10A2A800AF91BF91EC93AEEAB7E0E12FF0E0BD01CA
:10A2B800ACE0B0E00E9444CBE60FF71F3696FF9360
:10A2C800EF93A9E2B8E0E12FF0E0BD01AAE0B0E029
:10A2D8000E9444CBDB01AE0FBF1F15960E9486CCAF
:10A2E800AF91BF91EC931F5F7CCFE091B007E093F3
:10A2F800BD07A091B007E091BC07EA0FE093C9073A
:10A30800A091C907E091C807EA0FE093AD0710E0F4
:10A31800183108F0E1C0E0E03E2F0E2FA7E4B8E0C6
:10A32800E12FF0E0BD01ACE0B0E00E9444CBDB01DE
:10A33800AE0FBF1F11960E9486CCE03009F031E0C5
:10A34800A7E4B8E0E12FF0E0BD01ACE0B0E00E9486
:10A3580044CBDB01AE0FBF1F12960E9486CCE030C3
:10A3680009F03260A7E4B8E0E12FF0E0BD01ACE00D
:10A37800B0E00E9444CBDB01AE0FBF1F15960E94D0
:10A3880086CCE03009F03460A7E4B8E0E12FF0E0D3
:10A39800BD01ACE0B0E00E9444CBDB01AE0FBF1FB3
:10A3A80016960E9486CCE03009F03860A7E4B8E041
:10A3B800E12FF0E0BD01ACE0B0E00E9444CBDB014E
:10A3C800AE0FBF1F19960E9486CCE03009F03061AD
:10A3D800A7E4B8E0E12FF0E0BD01ACE0B0E00E94F6
:10A3E80044CBDB01AE0FBF1F1A960E9486CCE0302B
:10A3F80009F03062A7E4B8E0E12FF0E0BD01ACE07D
:10A40800B0E00E9444CBDB01AE0FBF1F13960E9441
:10A4180086CCE03009F000E1A7E4B8E0E12FF0E0F5
:10A42800BD01ACE0B0E00E9444CBDB01AE0FBF1F22
:10A4380017960E9486CCE03009F00062A7E4B8E0E5
:10A44800E12FF0E0BD01ACE0B0E00E9444CBDB01BD
:10A45800AE0FBF1F1B960E9486CCE03009F0006447
:10A46800A2EDB7E0E12FF0E00E940DCBEA0FFB1F51
:10A478000283A2EDB7E0E12FF0E00E940DCBEA0FD6
:10A48800FB1F3383A2EDB7E0E12FF0E00E940DCB74
:10A49800EA0FFB1F3296FF93EF93A7E4B8E0E12F92
:10A4A800F0E0BD01ACE0B0E00E9444CBDB01AE0FB0
:10A4B800BF1F0E9486CCE295EF70E695E695E170A5
:10A4C800AF91BF91E170EE0FEE0F0E2EEC91EB7F86
:10A4D800E029EC931F5F1CCF0E9498CA2496089528
:10A4E800BA93AA9325970E948FCAE091AB07F0E030
:10A4F800E230A0E0FA0739F4AB85BC85EC91E07155
:10A5080009F02AC10AC0E330A0E0FA0731F4AB85AC
:10A51800BC85EC91E07109F41FC1E091AB07F0E054
:10A52800E230A0E0FA0729F0E330A0E0FA0709F0EA
:10A5380013C110E0133008F00FC1AEEAB7E0E12F05
:10A54800F0E0BD01ACE0B0E00E9444CBE60FF71F9D
:10A558002281213008F4FDC0AEEAB7E0E12FF0E037
:10A56800BD01ACE0B0E00E9444CBE60FF71F31819B
:10A57800A091AB07A23089F4E32FF0E0E058FE4F3A
:10A588000F01AB85BC851196ED91FC911197E015F3
:10A59800F10509F0DFC0E1E007C0EB85FC85E1814A
:10A5A800E31709F0D7C0E3E0EA87AEEAB7E0E12FA6
:10A5B800F0E0BD01ACE0B0E00E9444CBDB01AE0F9F
:10A5C800BF1FEC91E03079F4AEEAB7E0E12FF0E09C
:10A5D800BD01ACE0B0E00E9444CBDB01AE0FBF1F71
:10A5E8001496EFEFEC93AEEAB7E0E12FF0E0BD018F
:10A5F800ACE0B0E00E9444CBDB01AE0FBF1FECE043
:10A60800EC93AEEAB7E0E12FF0E0BD01ACE0B0E0DA
:10A618000E9444CBE60FF71F5381E0E04E2FE887F6
:10A628000E2F421708F094C0A091AB07A230A1F4F6
:10A63800003069F407E0AB85BC851596E885EF5FC7
:10A64800E887E150F0E0AE0FBF1FEC9103C0015066
:10A65800E985E695E98714C0003069F403E0AB8525
:10A66800BC851596E885EF5FE887E150F0E0AE0F0E
:10A67800BF1FEC9104C00150E985E695E695E9878E
:10A68800A2EDB7E0E52FF0E00E940DCBAE0FBF1FA3
:10A698001296EC91E47009F43FC0A2EDB7E0E52F03
:10A6A800F0E00E940DCBAE0FBF1F1296EC91E17047
:10A6B800EF83A2EDB7E0E52FF0E00E940DCBAE0FDF
:10A6C800BF1F1296EC91E695E170EE83EA85A985A5
:10A6D800EA23E13069F4EE81E03049F4E1E0EE8309
:10A6E800EF81E03011F0E0E001C0E1E0EF8302C06B
:10A6F800E0E0EE83A2EDB7E0E52FF0E00E940DCB9D
:10A70800AE0FBF1F1296EE81E170EE0F0E2EEC9188
:10A71800ED7FE029EC9309C0EA85A985EA23E130B9
:10A7280011F4E1E001C0E0E0EF83A2EDB7E0E52F2E
:10A73800F0E00E940DCBAE0FBF1F1296EF81E170C3
:10A748000E2EEC91EE7FE029EC934F5F5F5F69CFAF
:10A7580003C002C01F5FEECE0E9496CA2D960895D0
:10A768002D970E9491CA1A2F09893A89EC81E061D4
:10A77800EC83E07FE860EC83F32FE0E0662777273F
:10A78800E060F0606F6E7861DF01CB01E0915C04FE
:10A79800FF2766277727EA2BFB2B682B792BED837E
:10A7A800FE836F837887E02FEF5FE987A2EDB7E03C
:10A7B800E12FF0E00E940DCBAE0FBF1FEC91EA87AE
:10A7C800A2EDB7E0E12FF0E00E940DCBAE0FBF1F66
:10A7D8001196EC91EB87C9C02D970E948FCA4A2F1A
:10A7E800EE81EF7EEE83E07FE860EE83EC89F0E0B7
:10A7F800E050FE4FEF83F887FE013B96FA93EA9309
:10A80800E0E0EA93A8E0B0E00E948EC351E020E0C7
:10A8180031E0E0E00E2F1E2F141708F04BC030E097
:10A82800333008F042C0503051F4E02F0F5FF0E0B1
:10A83800DE011B96EA0FFB1F208351E020E0E32F87
:10A84800F0E0309769F4A2EDB7E0EB89F0E00E9400
:10A858000DCBAE0FBF1FEC91EF7009F0252B22C076
:10A86800E130A0E0FA0769F4A2EDB7E0EB89F0E087
:10A878000E940DCBAE0FBF1FEC91E07F09F0252B96
:10A8880011C0E230A0E0FA0769F4A2EDB7E0EB8965
:10A89800F0E00E940DCBAE0FBF1F1196EC91E03097
:10A8A80009F0252B550F3F5FBBCF1F5FEB89EF5F8B
:10A8B800EB8BB2CFE02FF0E0DE011B96EA0FFB1F17
:10A8C8002083DE0116960E942D090E9496CA65967D
:10A8D80008952D970E9491CA1A2F09893A89FE0175
:10A8E8003996FA93EA93E0E0EA93A0E0B0E00E9498
:10A8F8008EC3EC81EF7EEC83E07FE860EC83E32F8E
:10A90800F0E0E050FD4FED83FE831987FE013B9692
:10A91800008335C02D970E9491CA1A2F09893A8958
:10A92800EC81E061EC83E07FE860EC83F32FE0E00A
:10A9380066277727E060F060606D7861DF01CB0102
:10A94800E0915C04FF2766277727EA2BFB2B682B0F
:10A95800792BED83FE836F837887E0E0E987FE013A
:10A968003A960083FE013B961083FE013C96FA93CB
:10A97800EA93EFEFEA93A5E0B0E00E948EC3DE0110
:10A9880014960E942D090E9498CA639608956297AA
:10A998000E948FCAE0916304E07409F47BC4A0911B
:10A9A800AC07A43038F4E091AC07EF5FE093AC0754
:10A9B800E15003C0E0E0E093AC07A091AC07A330FE
:10A9C80008F068C4AEEAB7E0E091AC07F0E0BD017A
:10A9D800ACE0B0E00E9444CBE60FF71F5181AEEA2D
:10A9E800B7E0E091AC07F0E0BD01ACE0B0E00E9458
:10A9F80044CBE60FF71F1281AEEAB7E0E091AC074F
:10AA0800F0E0BD01ACE0B0E00E9444CBE60FF71FD8
:10AA18003381113010F0103108F03CC4E091AB07DD
:10AA2800F0E0E230A0E0FA0729F0E330A0E0FA070E
:10AA380009F030C4AEEAB7E0E091AC07F0E0BD0140
:10AA4800ACE0B0E00E9444CBDB01AE0FBF1FAC917D
:10AA5800A13008F440C0AEEAB7E0E091AC07F0E0FE
:10AA6800BD01ACE0B0E00E9444CBDB01AE0FBF1FDC
:10AA7800EC91E150EC93AEEAB7E0E091AC07F0E07E
:10AA8800BD01ACE0B0E00E9444CBDB01AE0FBF1FBC
:10AA9800EC91E030F9F400E0232F0117D8F4A2ED8F
:10AAA800B7E0E22FF0E00E940DCBAE0FBF1F129669
:10AAB800EC91EE7FEC93A2EDB7E0E22FF0E00E947C
:10AAC8000DCBAE0FBF1F1296EC91E260EC930F5FB7
:10AAD8002F5FE3CF48C0A091AB07A23009F043C075
:10AAE800AEEAB7E0E091AC07F0E0BD01ACE0B0E061
:10AAF8000E9444CBDB01AE0FBF1F1A96AC91A13068
:10AB080088F0AEEAB7E0E091AC07F0E0BD01ACE058
:10AB1800B0E00E9444CBDB01AE0FBF1F1A96EC9148
:10AB2800E15020C0EE81E07FE260EE83EF7EEE83AD
:10AB3800E0E0EF83E887E1E0EB87E0E0EC87DE0127
:10AB480016960E942D09AEEAB7E0E091AC07F0E056
:10AB5800BD01ACE0B0E00E9444CBDB01AE0FBF1FEB
:10AB68001A96E4E1EC93AEEAB7E0E091AC07F0E0C6
:10AB7800BD01ACE0B0E00E9444CBDB01AE0FBF1FCB
:10AB88001696AC910E947A3BE03011F1A9E2B8E048
:10AB9800E091AC07F0E0BD01AAE0B0E00E9444CB30
:10ABA800DB01AE0FBF1F16960E9486CC4E2FA9E27E
:10ABB800B8E0E091AC07F0E0BD01AAE0B0E00E9487
:10ABC80044CBDB01AE0FBF1F17960E9486CC37C05F
:10ABD800AEEAB7E0E091AC07F0E0BD01ACE0B0E070
:10ABE8000E9444CBDB01AE0FBF1F1596AC910E94AB
:10ABF8007A3BE03011F1A9E2B8E0E091AC07F0E06F
:10AC0800BD01AAE0B0E00E9444CBDB01AE0FBF1F3C
:10AC180013960E9486CC4E2FA9E2B8E0E091AC07CB
:10AC2800F0E0BD01AAE0B0E00E9444CBDB01AE0F2A
:10AC3800BF1F14960E9486CC02C040E0E0E0EF8B74
:10AC4800AEEAB7E0E091AC07F0E0BD01ACE0B0E0FF
:10AC58000E9444CBDB01AE0FBF1F1796AC914A1779
:10AC680099F4AEEAB7E0E091AC07F0E0BD01ACE0E2
:10AC7800B0E00E9444CBDB01AE0FBF1F1896AC9129
:10AC8800EF89EA1709F447C0AEEAB7E0E091AC07EC
:10AC9800F0E0BD01ACE0B0E00E9444CBE60FF71F46
:10ACA8004783AEEAB7E0E091AC07F0E0BD01ACE065
:10ACB800B0E00E9444CBE60FF71F3896AF89A08317
:10ACC800A091AB07A23011F55A93AEEAB7E0E09134
:10ACD800AC07F0E0BD01ACE0B0E00E9444CBDB0182
:10ACE800AE0FBF1F1896EC91EA93AEEAB7E0E09179
:10ACF800AC07F0E0BD01ACE0B0E00E9444CBDB0162
:10AD0800AE0FBF1F1796AC91E4DD05C05A93E88DCE
:10AD1800EA93A42FFFDD00E0232F011708F0E8C114
:10AD2800A2EDB7E0E22FF0E00E940DCBAE0FBF1FFF
:10AD38001296EC91EE8BA2EDB7E0E22FF0E00E94C4
:10AD48000DCBAE0FBF1F1396EC91ED8BEE89E07122
:10AD5800A1F0A7E4B8E0E22FF0E0BD01ACE0B0E07C
:10AD68000E9444CBDB01AE0FBF1F13960E9486CC16
:10AD7800AE2F0E945160E03009F412C0A7E4B8E099
:10AD8800E22FF0E0BD01ACE0B0E00E9444CBDB0173
:10AD9800AE0FBF1F0E9486CCE295E370EF5F55C0EF
:10ADA800ED89E270A1F0A7E4B8E0E22FF0E0BD0180
:10ADB800ACE0B0E00E9444CBDB01AE0FBF1F12969F
:10ADC8000E9486CCAE2F0E947A3BE03009F413C073
:10ADD800A7E4B8E0E22FF0E0BD01ACE0B0E00E94EB
:10ADE80044CBDB01AE0FBF1F0E9486CCE695E695EB
:10ADF800E370EF5F2AC0ED89E170A1F0A7E4B8E045
:10AE0800E22FF0E0BD01ACE0B0E00E9444CBDB01F2
:10AE1800AE0FBF1F11960E9486CCAE2F0E947A3BC0
:10AE2800E03009F411C0A7E4B8E0E22FF0E0BD017A
:10AE3800ACE0B0E00E9444CBDB01AE0FBF1F0E9424
:10AE480086CCE370EF5F01C0E0E0EC8BEE89E07246
:10AE5800A1F0A7E4B8E0E22FF0E0BD01ACE0B0E07B
:10AE68000E9444CBDB01AE0FBF1F17960E9486CC11
:10AE7800AE2F0E945160E03009F411C0A7E4B8E099
:10AE8800E22FF0E0BD01ACE0B0E00E9444CBDB0172
:10AE9800AE0FBF1F14960E9486CCE29551C0ED8973
:10AEA800E870A1F0A7E4B8E0E22FF0E0BD01ACE063
:10AEB800B0E00E9444CBDB01AE0FBF1F16960E9484
:10AEC80086CCAE2F0E947A3BE03009F412C0A7E48A
:10AED800B8E0E22FF0E0BD01ACE0B0E00E9444CB66
:10AEE800DB01AE0FBF1F14960E9486CCE695E6954F
:10AEF80027C0ED89E470A1F0A7E4B8E0E22FF0E004
:10AF0800BD01ACE0B0E00E9444CBDB01AE0FBF1F37
:10AF180015960E9486CCAE2F0E947A3BE03009F449
:10AF280016C0A7E4B8E0E22FF0E0BD01ACE0B0E065
:10AF38000E9444CBDB01AE0FBF1F14960E9486CC43
:10AF4800E370EF5FE295E07FAC89EA2BEC8BEE894A
:10AF5800E074A1F0A7E4B8E0E22FF0E0BD01ACE0B6
:10AF6800B0E00E9444CBDB01AE0FBF1F1B960E94CE
:10AF780086CCAE2F0E945160E03009F413C0A7E4DC
:10AF8800B8E0E22FF0E0BD01ACE0B0E00E9444CBB5
:10AF9800DB01AE0FBF1F18960E9486CCE295E370C6
:10AFA800EF5F57C0ED89E072A1F0A7E4B8E0E22FA7
:10AFB800F0E0BD01ACE0B0E00E9444CBDB01AE0F95
:10AFC800BF1F1A960E9486CCAE2F0E947A3BE030B3
:10AFD80009F414C0A7E4B8E0E22FF0E0BD01ACE04A
:10AFE800B0E00E9444CBDB01AE0FBF1F18960E9451
:10AFF80086CCE695E695E370EF5F2BC0ED89E071AE
:10B00800A1F0A7E4B8E0E22FF0E0BD01ACE0B0E0C9
:10B018000E9444CBDB01AE0FBF1F19960E9486CC5D
:10B02800AE2F0E947A3BE03009F412C0A7E4B8E0E2
:10B03800E22FF0E0BD01ACE0B0E00E9444CBDB01C0
:10B04800AE0FBF1F18960E9486CCE370EF5F01C059
:10B05800E0E0EB8BA2EDB7E0E22FF0E00E940DCB31
:10B06800AE0FBF1FAC91EC89EA1769F4A2EDB7E007
:10B07800E22FF0E00E940DCBAE0FBF1F1196AC91EE
:10B08800EB89EA1791F1A2EDB7E0E22FF0E00E9418
:10B098000DCBEA0FFB1FAC89A083A2EDB7E0E22F2E
:10B0A800F0E00E940DCBEA0FFB1F3196AB89A0831D
:10B0B800AEEAB7E0E091AC07F0E0BD01ACE0B0E08B
:10B0C8000E9444CBDB01AE0FBF1F1996E4E1EC935D
:10B0D800A091AB07A23029F45A933A93A12F7CDBB5
:10B0E80004C05A930A93A22F3BDB0F5F2F5F15CE44
:10B0F800AEEAB7E0E091AC07F0E0BD01ACE0B0E04B
:10B108000E9444CBDB01AE0FBF1F1996AC91A13052
:10B1180088F0AEEAB7E0E091AC07F0E0BD01ACE042
:10B12800B0E00E9444CBDB01AE0FBF1F1996EC9133
:10B13800E150AFC0A091AB07A230B1F5AEEAB7E0DD
:10B14800E091AC07F0E0BD01ACE0B0E00E9444CB78
:10B15800DB01AE0FBF1F1996E9E0EC935A933A93BF
:10B16800A12F3ADB5A93AEEAB7E0E091AC07F0E0E2
:10B17800BD01ACE0B0E00E9444CBDB01AE0FBF1FC5
:10B188001896EC91EA93AEEAB7E0E091AC07F0E0EC
:10B19800BD01ACE0B0E00E9444CBDB01AE0FBF1FA5
:10B1A8001796AC9196DB76C0AEEAB7E0E091AC07B3
:10B1B800F0E0BD01ACE0B0E00E9444CBDB01AE0F93
:10B1C800BF1F1996EAE0EC93AEEAB7E0E091AC074E
:10B1D800F0E0BD01ACE0B0E00E9444CBDB01AE0F73
:10B1E800BF1F1496AC91A11790F1AEEAB7E0E091B9
:10B1F800AC07F0E0BD01ACE0B0E00E9444CBDB015D
:10B20800AE0FBF1F1496E0E0EC935A93AEEAB7E096
:10B21800E091AC07F0E0BD01ACE0B0E00E9444CBA7
:10B22800DB01AE0FBF1F1896EC91EA93AEEAB7E0C8
:10B23800E091AC07F0E0BD01ACE0B0E00E9444CB87
:10B24800DB01AE0FBF1F1796AC9164DB23C0AEEADB
:10B25800B7E0E091AC07F0E0BD01ACE0B0E00E94DF
:10B2680044CBE60FF71F04815A930A93A02FA30F2C
:10B2780077DAAEEAB7E0E091AC07F0E0BD01ACE008
:10B28800B0E00E9444CBDB01AE0FBF1F1496EC91D7
:10B29800EF5FEC930E9496CA689608950E9491CA3F
:10B2A800ECEAF7E0FA93EA93E0E0EA93A9E6B0E083
:10B2B8000E948EC3A9E2B8E00E9486CCE093AD0755
:10B2C800AAE2B8E00E9486CCE093D50710E01230DD
:10B2D80008F0A2C0ABE2B8E0E12FF0E0BD01AAE0BF
:10B2E800B0E00E9444CBDB01AE0FBF1F0E9482CCAE
:10B2F8009F01ADEAB7E0E12FF0E0BD01A8E2B0E0C0
:10B308000E9444CBE60FF71F3496FF93EF93ABE20E
:10B31800B8E0E12FF0E0BD01AAE0B0E00E9444CB24
:10B32800DB01AE0FBF1F12960E9486CCAF91BF9172
:10B33800EC93ADEAB7E0E12FF0E0BD01A8E2B0E0A0
:10B348000E9444CBE60FF71F3596FF93EF93ABE2CD
:10B35800B8E0E12FF0E0BD01AAE0B0E00E9444CBE4
:10B36800DB01AE0FBF1F16960E9486CCAF91BF912E
:10B37800EC93ADEAB7E0E12FF0E0BD01A8E2B0E060
:10B388000E9444CBE60FF71F2787308BADEAB7E062
:10B39800E12FF0E0BD01A8E2B0E00E9444CBDB0160
:10B3A800AE0FBF1F1E96EC91E07FE460EC93ADEA10
:10B3B800B7E0E12FF0E0BD01A8E2B0E00E9444CB85
:10B3C800DB01AE0FBF1F1196F9013196ED93FC9387
:10B3D800ADEAB7E0E12FF0E0BD01A8E2B0E00E94DD
:10B3E80044CBDB01AE0FBF1F5C96F9013496ED9399
:10B3F800FC93ADEAB7E0E12FF0E0BD01A8E2B0E0D0
:10B408000E9444CBDB01AE0FBF1F5B96EC91E07F3F
:10B41800E860EC931F5F5BCFAFE3B8E00E9486CC97
:10B42800E093B507A0E4B8E00E9486CCE093B807A3
:10B43800A1E4B8E00E9486CCE093DD07A2E4B8E07E
:10B448000E9486CCE093E00710E01831A0F500E0F8
:10B45800A3E4B8E0E12FF0E00E940DCBAE0FBF1FD0
:10B4680011960E9486CCE03009F001E0A3E4B8E030
:10B47800E12FF0E00E940DCBAE0FBF1F12960E9485
:10B4880086CCE03009F00260A3E4B8E0E12FF0E0F8
:10B498000E940DCBAE0FBF1F13960E9486CCE030E2
:10B4A80009F00460ADEFB7E0E12FF0E0EA0FFB1F11
:10B4B80000831F5FCACF0E9498CA24960895BA9342
:10B4C800AA930E948FCA10E0123008F0CDC0ADEAEE
:10B4D800B7E0E12FF0E0BD01A8E2B0E00E9444CB64
:10B4E800DB01AE0FBF1FEC91E030B1F0ADEAB7E081
:10B4F800E12FF0E0BD01A8E2B0E00E9444CBE60FE6
:10B50800F71F01801280AE81BF811196ED91FC91E9
:10B518001197E015F10509F0A5C0EE81FF810581BD
:10B52800ADEAB7E0E12FF0E0BD01A8E2B0E00E948B
:10B5380044CBE60FF71F2681ADEAB7E0E12FF0E034
:10B54800BD01A8E2B0E00E9444CBE60FF71F50858A
:10B55800ADEAB7E0E12FF0E0BD01A8E2B0E00E945B
:10B5680044CBE60FF71F37812523A02FA523EFEF44
:10B57800E327EA232E27E52FE095E0232E2BADEADB
:10B58800B7E0E12FF0E0BD01A8E2B0E00E9444CBB3
:10B59800E60FF71F2683ADEAB7E0E12FF0E0BD0123
:10B5A800A8E2B0E00E9444CBE60FF71F0783EE81C4
:10B5B800FF81E681EF700E2FADEAB7E0E12FF0E0F2
:10B5C800BD01A8E2B0E00E9444CBE60FF71F218539
:10B5D800ADEAB7E0E12FF0E0BD01A8E2B0E00E94DB
:10B5E80044CBE60FF71F5385ADEAB7E0E12FF0E053
:10B5F800BD01A8E2B0E00E9444CBE60FF71F3285F8
:10B608002523A02FA523EFEFE327EA232E27E52FF5
:10B61800E095E0232E2BADEAB7E0E12FF0E0BD0185
:10B62800A8E2B0E00E9444CBE60FF71F2187ADEAFD
:10B63800B7E0E12FF0E0BD01A8E2B0E00E9444CB02
:10B64800E60FF71F0287ADEAB7E0E12FF0E0BD0192
:10B65800A8E2B0E00E9444CBDB01AE0FBF1F1396F7
:10B66800EAE0EC931F5F30CF0E9496CA28960895AF
:10B6780024970E948FCAE0916304E07409F4BBC365
:10B68800A091AC07A43038F4E091AC07EF5FE093E9
:10B69800AC07E15003C0E0E0E093AC07A091AC0731
:10B6A800A23008F0A8C3ADEAB7E0E091AC07F0E03B
:10B6B800BD01A8E2B0E00E9444CBDB01AE0FBF1F82
:10B6C800EC91E03009F497C3ADEAB7E0E091AC073C
:10B6D800F0E0BD01A8E2B0E00E9444CBDB01AE0F70
:10B6E800BF1F1396AC91A13008F463C0ADEAB7E070
:10B6F800E091AC07F0E0BD01A8E2B0E00E9444CBC5
:10B70800DB01AE0FBF1F1396EC91E150EC93ADEA4D
:10B71800B7E0E091AC07F0E0BD01A8E2B0E00E941C
:10B7280044CBDB01AE0FBF1F1396EC91E03009F05C
:10B7380040C0ADEAB7E0E091AC07F0E0BD01A8E297
:10B74800B0E00E9444CBDB01AE0FBF1F1696E0E0CD
:10B75800EC93ADEAB7E0E091AC07F0E0BD01A8E2F8
:10B76800B0E00E9444CBDB01AE0FBF1F1796E0E0AC
:10B77800EC93ADEAB7E0E091AC07F0E0BD01A8E2D8
:10B78800B0E00E9444CBDB01AE0FBF1F1996E0E08A
:10B79800EC93ADEAB7E0E091AC07F0E0BD01A8E2B8
:10B7A800B0E00E9444CBDB01AE0FBF1F1A96E0E069
:10B7B800EC93E0E02E2F3E2FE091AC07E03011F43F
:10B7C80050E001C05CE040E011E0103009F47DC0B9
:10B7D800ADEFB7E0EE27A50FBE1F0C9102FF10C01A
:10B7E800A3E4B8E0E52FF0E00E940DCBAE0FBF1F39
:10B7F80013960E9486CCAE2F0E945160E03009F467
:10B808000EC0A3E4B8E0E52FF0E00E940DCBAE0F28
:10B81800BF1F0E9486CCE295E370EE8343C001FF10
:10B8280010C0A3E4B8E0E52FF0E00E940DCBAE0F06
:10B83800BF1F12960E9486CCAE2F0E947A3BE03042
:10B8480009F40FC0A3E4B8E0E52FF0E00E940DCBA7
:10B85800AE0FBF1F0E9486CCE695E695E370EE8397
:10B8680021C000FF10C0A3E4B8E0E52FF0E00E947B
:10B878000DCBAE0FBF1F11960E9486CCAE2F0E9433
:10B888007A3BE03009F40DC0A3E4B8E0E52FF0E01E
:10B898000E940DCBAE0FBF1F0E9486CCE370EE83D3
:10B8A80001C010C0EE81F0E0309711F4312B0AC0CE
:10B8B800E130A0E0FA0729F0E230A0E0FA0711F43D
:10B8C800312B212B5F5F110F80CFADEAB7E0E091FC
:10B8D800AC07F0E0BD01A8E2B0E00E9444CBE60F5F
:10B8E800F71FA0A13A1771F0ADEAB7E0E091AC07F5
:10B8F800F0E0BD01A8E2B0E00E9444CBE60FF71FDC
:10B9080030A341E0ADEAB7E0E091AC07F0E0BD015B
:10B91800A8E2B0E00E9444CBE60FF71FA2A12A17C5
:10B9280071F0ADEAB7E0E091AC07F0E0BD01A8E244
:10B93800B0E00E9444CBE60FF71F22A341E0E0E00D
:10B948002E2F3E2F11E0103109F47CC0ADEFB7E087
:10B95800EE27A50FBE1F0C9102FF0FC0A3E4B8E0AD
:10B96800E52FF0E00E940DCBAE0FBF1F13960E948B
:10B9780086CCAE2F92D3E03009F40EC0A3E4B8E031
:10B98800E52FF0E00E940DCBAE0FBF1F0E9486CCC2
:10B99800E295E370EE8343C001FF10C0A3E4B8E072
:10B9A800E52FF0E00E940DCBAE0FBF1F12960E944C
:10B9B80086CCAE2F0E947A3BE03009F40FC0A3E496
:10B9C800B8E0E52FF0E00E940DCBAE0FBF1F0E943C
:10B9D80086CCE695E695E370EE8321C000FF10C0A3
:10B9E800A3E4B8E0E52FF0E00E940DCBAE0FBF1F37
:10B9F80011960E9486CCAE2F0E947A3BE03009F463
:10BA08000DC0A3E4B8E0E52FF0E00E940DCBAE0F27
:10BA1800BF1F0E9486CCE370EE8301C010C0EE8188
:10BA2800F0E0309711F4312B0AC0E130A0E0FA07BA
:10BA380029F0E230A0E0FA0711F4312B212B5F5FE7
:10BA4800110F81CFADEAB7E0E091AC07F0E0BD019E
:10BA5800A8E2B0E00E9444CBE60FF71FA1A13A1775
:10BA680071F0ADEAB7E0E091AC07F0E0BD01A8E203
:10BA7800B0E00E9444CBE60FF71F31A341E0ADEAE6
:10BA8800B7E0E091AC07F0E0BD01A8E2B0E00E94A9
:10BA980044CBE60FF71FA3A12A1771F0ADEAB7E070
:10BAA800E091AC07F0E0BD01A8E2B0E00E9444CB11
:10BAB800E60FF71F23A341E0403089F4ADEAB7E071
:10BAC800E091AC07F0E0BD01A8E2B0E00E9444CBF1
:10BAD800DB01AE0FBF1F1D96AC91A13008F412C058
:10BAE800ADEAB7E0E091AC07F0E0BD01A8E2B0E054
:10BAF8000E9444CBDB01AE0FBF1F1D96EC91E150B5
:10BB0800EC9320C0ADEAB7E0E091AC07F0E0BD01EE
:10BB1800A8E2B0E00E9444CBDB01AE0FBF1F1D9628
:10BB2800E0E1EC93ADEAB7E0E091AC07F0E0BD01ED
:10BB3800A8E2B0E00E9444CBDB01AE0FBF1F5B96CA
:10BB48000E942D09ADEAB7E0E091AC07F0E0BD0135
:10BB5800A8E2B0E00E9444CBDB01AE0FBF1F1496F1
:10BB6800AC91A03091F4ADEAB7E0E091AC07F0E019
:10BB7800BD01A8E2B0E00E9444CBDB01AE0FBF1FBD
:10BB88001596AC91A03009F436C140E0E1E0E987B0
:10BB9800EFE0E887EF83ADEAB7E0E091AC07F0E0CB
:10BBA800BD01A8E2B0E00E9444CBDB01AE0FBF1F8D
:10BBB8001596AC910E947A3BE03089F1ABE2B8E08F
:10BBC800E091AC07F0E0BD01AAE0B0E00E9444CBF0
:10BBD800DB01AE0FBF1F17960E9486CCE987ABE248
:10BBE800B8E0E091AC07F0E0BD01AAE0B0E00E9447
:10BBF80044CBDB01AE0FBF1F18960E9486CCE887A6
:10BC0800ABE2B8E0E091AC07F0E0BD01AAE0B0E03B
:10BC18000E9444CBDB01AE0FBF1F199643C0ADEAAB
:10BC2800B7E0E091AC07F0E0BD01A8E2B0E00E9407
:10BC380044CBDB01AE0FBF1F1496AC910E947A3B38
:10BC4800E03099F1ABE2B8E0E091AC07F0E0BD017B
:10BC5800AAE0B0E00E9444CBDB01AE0FBF1F1396F1
:10BC68000E9486CCE987ABE2B8E0E091AC07F0E04F
:10BC7800BD01AAE0B0E00E9444CBDB01AE0FBF1FBC
:10BC880014960E9486CCE887ABE2B8E0E091AC0756
:10BC9800F0E0BD01AAE0B0E00E9444CBDB01AE0FAA
:10BCA800BF1F15960E9486CCEF83ADEAB7E0E091FE
:10BCB800AC07F0E0BD01A8E2B0E00E9444CBE60F7B
:10BCC800F71FA489E985EA1781F0ADEAB7E0E091AA
:10BCD800AC07F0E0BD01A8E2B0E00E9444CBE60F5B
:10BCE800F71F7496A985A08341E0ADEAB7E0E0911B
:10BCF800AC07F0E0BD01A8E2B0E00E9444CBE60F3B
:10BD0800F71FA589E885EA1781F0ADEAB7E0E09169
:10BD1800AC07F0E0BD01A8E2B0E00E9444CBE60F1A
:10BD2800F71F7596A885A08341E0ADEAB7E0E091DA
:10BD3800AC07F0E0BD01A8E2B0E00E9444CBE60FFA
:10BD4800F71FA689EF81EA1781F0ADEAB7E0E09125
:10BD5800AC07F0E0BD01A8E2B0E00E9444CBE60FDA
:10BD6800F71F7696AF81A08341E0403089F4ADEAB1
:10BD7800B7E0E091AC07F0E0BD01A8E2B0E00E94B6
:10BD880044CBDB01AE0FBF1F1C96AC91A13008F469
:10BD980012C0ADEAB7E0E091AC07F0E0BD01A8E25F
:10BDA800B0E00E9444CBDB01AE0FBF1F1C96EC91A4
:10BDB800E150EC9320C0ADEAB7E0E091AC07F0E0C9
:10BDC800BD01A8E2B0E00E9444CBDB01AE0FBF1F6B
:10BDD8001C96E0E1EC93ADEAB7E0E091AC07F0E047
:10BDE800BD01A8E2B0E00E9444CBDB01AE0FBF1F4B
:10BDF8001E960E942D090E9496CA2A9608950895B3
:10BE08001A931A2FA9E01A9FF001E650F74FA08164
:10BE1800A73B21F4A12F0E9444813DC11730D0F4E3
:10BE2800103011F42D9815C0113011F4109811C06C
:10BE3800123011F42E980DC0133011F4A19809C0D6
:10BE4800143011F4739805C0153011F4A29801C08C
:10BE5800A09825C01D30B0F4173011F45F9811C0B8
:10BE6800183011F42F980DC0193011F4139809C027
:10BE78001A3011F4749805C01B3011F4149801C0DD
:10BE880075980DC0123158F41D3011F48C9807C004
:10BE98001E3011F42C9803C01F3009F48D98FBC094
:10BEA8001A931A2F1730D0F4103011F42D9A15C0A8
:10BEB800113011F4109A11C0123011F42E9A0DC0DD
:10BEC800133011F4A19A09C0143011F4739A05C003
:10BED800153011F4A29A01C0A09A25C01D30B0F403
:10BEE800173011F45F9A11C0183011F42F9A0DC051
:10BEF800193011F4139A09C01A3011F4749A05C054
:10BF08001B3011F4149A01C0759A0DC0123158F4FF
:10BF18001D3011F48C9A07C01E3011F42C9A03C0FE
:10BF28001F3009F48D9AB7C01A931A2F1730D0F41E
:10BF3800103011F42D9815C0113011F4109811C05B
:10BF4800123011F42E980DC0133011F4A19809C0C5
:10BF5800143011F4739805C0153011F4A29801C07B
:10BF6800A09825C01D30B0F4173011F45F9811C0A7
:10BF7800183011F42F980DC0193011F4139809C016
:10BF88001A3011F4749805C01B3011F4149801C0CC
:10BF980075980DC0123158F41D3011F48C9807C0F3
:10BFA8001E3011F42C9803C01F3009F48D9873C00B
:10BFB8001A931A2FE6EBF4E060E070E00E9418CCC8
:10BFC800E12FFF27662777270E9418CC84E00E947C
:10BFD80016CA289611501730A0F4E12FA1E00E944C
:10BFE800B1CA1E2FA091E608E095EA23E093E6087F
:10BFF800E091E708E12BE093E708E0E0E093E3084D
:10C0080016C01830A0F41850E12FA1E00E94B1CA60
:10C018001E2FA091E808E095EA23E093E808E09154
:10C02800E908E12BE093E908E0E0E093E40833C095
:10C038001A931A2FE7ECF4E060E070E00E9418CC45
:10C04800E12FFF27662777270E9418CC84E00E94FB
:10C0580016CA28961150173070F4E12FA1E00E94FB
:10C06800B1CA1E2FE091E608E12BE093E608E0E074
:10C07800E093E30810C0183070F41850E12FA1E0E5
:10C088000E94B1CA1E2FE091E808E12BE093E8086E
:10C09800E0E0E093E408199108950E9491CA3A2FCC
:10C0A8003F3010F03F3108F01EC0E32FEF501E2F35
:10C0B800A9E01A9FF001E950F74FE081E47011F010
:10C0C800E1E074C2A9E01A9FF001E950F74FE0815E
:10C0D800E295E7700E2F013021F0043011F00530A1
:10C0E80011F4E1E063C2A32F0E948A7A5FC20E9422
:10C0F80091CAE091EF08EF7EE093EF08EF7DE093BF
:10C10800EF08E4E1E093F308E091EF08EF7BE093B8
:10C11800EF08E091F008EE7FE093F008ED7FE09300
:10C12800F008E7EFF8E0FA93EA93E0E0EA93A0E991
:10C13800B0E00E948EC3089A999A9A9A989A0B9A94
:10C148006C9A859AE2B1E67EE2B9E5B1EF70E5B99D
:10C158005F98EEB1E77CEEB9E1B3EF7CE1BBE4B305
:10C16800E87FE4BBEFEFE093E608E093E80810E02F
:10C17800103108F008C2A9E01A9FF001E650F74F05
:10C18800FF93EF93A5E4B1E0E12FF0E0BD01A7E054
:10C19800B0E00E9444CBDB01AE0FBF1F0E9486CCEB
:10C1A800AF91BF91EC93A9E01A9FF001E950F74FC6
:10C1B800FF93EF93A5E4B1E0E12FF0E0BD01A7E024
:10C1C800B0E00E9444CBDB01AE0FBF1F12960E9465
:10C1D80086CCE07121F5A5E4B1E0E12FF0E0BD01E6
:10C1E800A7E0B0E00E9444CBDB01AE0FBF1F129660
:10C1F8000E9486CCE07299F4A5E4B1E0E12FF0E06A
:10C20800BD01A7E0B0E00E9444CBDB01AE0FBF1F29
:10C2180012960E9486CCE07411F4E0E001C0E1E0DF
:10C22800AF91BF91E170EE0F0E2EEC91ED7FE029FA
:10C23800EC93A5E4B1E0E12FF0E0BD01A7E0B0E0A8
:10C248000E9444CBDB01AE0FBF1F15960E9486CC1F
:10C25800E07249F0A9E01A9FF001E850F74FDF01BA
:10C26800EC91E061EC93A5E4B1E0E12FF0E0BD01D1
:10C27800A7E0B0E00E9444CBDB01AE0FBF1F1596CC
:10C288000E9486CCE07449F0A9E01A9FF001E850BA
:10C29800F74FDF01EC91E062EC93A5E4B1E0E12F08
:10C2A800F0E0BD01A7E0B0E00E9444CBDB01AE0F97
:10C2B800BF1F12960E9486CCE07859F0183020F4FF
:10C2C800E091EF08E06103C0E091EF08E062E093DD
:10C2D800EF08A7E6B9E0E12FF0E0F595E795AE0F96
:10C2E800BF1F0E9486CC0E2F10FF0DC0E02FE07FED
:10C2F80049F0A9E01A9FF001E950F74FDF01EC91EE
:10C30800E068EC930CC0E02FEF7049F0A9E01A9FA9
:10C31800F001E950F74FDF01EC91E068EC93A9E0F8
:10C328001A9FF001E650F74FA081A63309F03FC0ED
:10C33800E12FFF2766277727E056FF4F6F4F6BBF28
:10C348003691303148F4A9E03A9FF001E850F74FB0
:10C35800DF01EC91E064EC93E12FF0E0E130A0E044
:10C36800FA0711F4089823C0E330A0E0FA0711F4A3
:10C3780099981DC0E530A0E0FA0711F49A9817C003
:10C38800E630A0E0FA0711F4989811C0E930A0E06F
:10C39800FA0711F40B980BC0EA30A0E0FA0711F481
:10C3A8006C9805C0EF30A0E0FA0709F48598A5E479
:10C3B800B1E0E12FF0E0BD01A7E0B0E00E9444CB7E
:10C3C800DB01AE0FBF1F15960E9486CCE07409F4FE
:10C3D800D8C0183008F06AC0E12FF0E0309749F46F
:10C3E800E091E608EE7FE093E608E091E708E16077
:10C3F8005AC0E130A0E0FA0749F4E091E608ED7F81
:10C40800E093E608E091E708E2604DC0E230A0E082
:10C41800FA0749F4E091E608EF7EE093E608E09138
:10C42800E708E06140C0E330A0E0FA0749F4E09192
:10C43800E608EF77E093E608E091E708E06833C0A4
:10C44800E430A0E0FA0749F4E091E608EB7FE093D6
:10C45800E608E091E708E46026C0E530A0E0FA07C6
:10C4680049F4E091E608EF7DE093E608E091E708FB
:10C47800E06219C0E630A0E0FA0749F4E091E60866
:10C48800EF7BE093E608E091E708E0640CC0E73052
:10C49800A0E0FA0751F4E091E608E77FE093E608A8
:10C4A800E091E708E860E093E7086BC0E12FF0E06F
:10C4B800E830A0E0FA0749F4E091E808EE7FE0935D
:10C4C800E808E091E908E1605AC0E930A0E0FA071D
:10C4D80049F4E091E808EF77E093E808E091E9088B
:10C4E800E0684DC0EA30A0E0FA0749F4E091E808B6
:10C4F800EF7BE093E808E091E908E06440C0EB30A6
:10C50800A0E0FA0749F4E091E808EF7DE093E80835
:10C51800E091E908E06233C0EC30A0E0FA0749F4A2
:10C52800E091E808EF7EE093E808E091E908E0612F
:10C5380026C0ED30A0E0FA0749F4E091E808E77F6B
:10C54800E093E808E091E908E86019C0EE30A0E05F
:10C55800FA0749F4E091E808EB7FE093E808E091F6
:10C56800E908E4600CC0EF30A0E0FA0751F4E0916C
:10C57800E808ED7FE093E808E091E908E260E093DD
:10C58800E9081F5FF5CDE0E0E093E308E093E408F5
:10C59800E091EF08E07111F0A39A01C0A398E0912F
:10C5A800EF08E07211F0A49A01C0A4980E9498CAFA
:10C5B8002496089527970E948FCAE091F108EF7397
:10C5C800E03100F1A398A498E091F108E07CE093B1
:10C5D800F108E091EE08E770E063E093EE08E2B15D
:10C5E800E67EE2B9E5B1EF70E5B95F98EEB1E77CB8
:10C5F800EEB9E1B3EF7CE1BBE4B3E87FE4BBA0E0D4
:10C608004FDCB6C2E091EE08E87FE83008F4B0C22B
:10C61800AEEEB8E083E0EFE10E944CCCE091EE088A
:10C62800E87FE830D1F4A1E4B8E0E091F108EF73D5
:10C63800FF2766277727E054FF4F6F4F6BBFE691C0
:10C64800F0E0EE0FFF1FAE0FBF1FED91FC911197A9
:10C65800E093F508F093F6088BC2E091EE08E87FC6
:10C6680009F086C2A1E4B8E0E091F108EF73FF2772
:10C6780066277727E054FF4F6F4F6BBFE691F0E0D6
:10C68800EE0FFF1FAE0FBF1FED91FD91A091F508B2
:10C69800B091F608EA0FFB1FE093F508F093F6084F
:10C6A800A091F508B091F608E091F608F070EA0F4D
:10C6B800FB1FE093F508F093F6080E941FCBE09368
:10C6C800F508F093F608E091EE08F0E0E770F070F6
:10C6D800E230A0E0FA07E1F5A2E3B0E0E091F1086A
:10C6E800EF73F0E0BD01AAE0B0E00E9444CBDB01AB
:10C6F800AE0FBF1FE091F508F091F6080E949ACCA2
:10C70800E091F108EF73FF2766277727E053FF4F83
:10C718006F4F6BBFE691E03061F4E6E5F1E060E071
:10C7280070E00E9407CC9F01E6E7F1E060E070E06E
:10C738000BC0E6E9F1E060E070E00E9407CC9F01E1
:10C74800E6EBF1E060E070E00E9407CCAF0103C1C6
:10C75800E330A0E0FA07E9F5A2E3B0E0E091F108E0
:10C76800EF73F0E0BD01AAE0B0E00E9444CBDB012A
:10C77800AE0FBF1F1296E091F508F091F6080E94DF
:10C788009ACCE091F108EF73FF2766277727E053EB
:10C79800FF4F6F4F6BBFE691E03061F4E8E5F1E0E1
:10C7A80060E070E00E9407CC9F01E8E7F1E060E0FC
:10C7B80070E00BC0E8E9F1E060E070E00E9407CCAF
:10C7C8009F01E8EBF1E060E070E00E9407CCAF0168
:10C7D800C2C0E430A0E0FA07E9F5A2E3B0E0E091D6
:10C7E800F108EF73F0E0BD01AAE0B0E00E9444CB8D
:10C7F800DB01AE0FBF1F1496E091F508F091F60823
:10C808000E949ACCE091F108EF73FF2766277727FB
:10C81800E053FF4F6F4F6BBFE691E03061F4EAE5FC
:10C82800F1E060E070E00E9407CC9F01EAE7F1E0E8
:10C8380060E070E00BC0EAE9F1E060E070E00E94BF
:10C8480007CC9F01EAEBF1E060E070E00E9407CCC2
:10C85800AF0181C0E530A0E0FA07E9F5A2E3B0E056
:10C86800E091F108EF73F0E0BD01AAE0B0E00E94AA
:10C8780044CBDB01AE0FBF1F1696E091F508F0918F
:10C88800F6080E949ACCE091F108EF73FF2766271B
:10C898007727E053FF4F6F4F6BBFE691E03061F4AD
:10C8A800ECE5F1E060E070E00E9407CC9F01ECE766
:10C8B800F1E060E070E00BC0ECE9F1E060E070E00E
:10C8C8000E9407CC9F01ECEBF1E060E070E00E9471
:10C8D80007CCAF0140C0E630A0E0FA07E1F5A2E3DB
:10C8E800B0E0E091F108EF73F0E0BD01AAE0B0E03C
:10C8F8000E9444CBDB01AE0FBF1F1896E091F508EC
:10C90800F091F6080E949ACCE091F108EF73FF27A6
:10C9180066277727E053FF4F6F4F6BBFE691E030F4
:10C9280061F4EEE5F1E060E070E00E9407CC9F0161
:10C93800EEE7F1E060E070E00BC0EEE9F1E060E006
:10C9480070E00E9407CC9F01EEEBF1E060E070E040
:10C958000E9407CCAF01ECEDF4E060E070E00E94CB
:10C9680018CCE091F108EF73F0E031966F2F660F65
:10C97800660B762F0E9418CCE091F508F091F60826
:10C98800662777270E9418CC88E00E9416CA2C9642
:10C99800A091F508B091F608A217B30718F04A1746
:10C9A8005B0708F402C011E013C010E0E091F20840
:10C9B800EC7771F4A2EFB8E0E091F108EF73EF5F64
:10C9C800EF71EE0FEE0F0E2EEC91E378E029EC9369
:10C9D800A12F0E940EBBE7E0EF83E9EFE887E98526
:10C9E800E160E987E12FE170EE0F0E2EE985ED7F1A
:10C9F800E029E987E091F108EF73EF5FEF73EE0F3D
:10CA0800EE0F0E2EE985E370E029E987E091F5083D
:10CA1800F091F608EB87FC87E091EE08F0E0E7700C
:10CA2800F070E230A0E0FA0711F4E1E019C0E33059
:10CA3800A0E0FA0711F4E2E013C0E430A0E0FA073E
:10CA480011F4E3E00DC0E530A0E0FA0711F4E4E0EA
:10CA580007C0E630A0E0FA0711F4E5E001C0E0E025
:10CA6800EA87E2B1E67EE2B9E5B1EF70E5B95F9831
:10CA7800EEB1E77CEEB9E1B3EF7CE1BBE4B3E87F6C
:10CA8800E4BBDE0116960E94E790E091F108EF738F
:10CA9800EF3090F4A1EFB8E080E0EFE30E9448CCDB
:10CAA800E091EE08E770E062E093EE08E091F108AB
:10CAB800EF73AE2FF5D95CC0A2E2B0E00E9486CC3D
:10CAC8001E2EE091EE08E770E250A1E00E94B1CA84
:10CAD800E129A2E2B0E00E94A2CCE7EEF4E060E037
:10CAE80070E00E9418CC80E00E9416CA2496E0915B
:10CAF800F208EC7791F4E2EFF4E060E070E00E9475
:10CB080018CC80E00E9416CA2496E091EE08E770DF
:10CB1800E23011F40E94983514C0E6EFF4E060E0CA
:10CB280070E00E9418CCE091F208E695E695EF7166
:10CB3800FF27662777270E9418CC84E00E9416CA30
:10CB48002896E091EF08E07111F0A39A01C0A3982C
:10CB5800E091EF08E07211F0A49A01C0A498E09166
:10CB6800EE08E87FE160E093EE08E6E0E093940DDC
:10CB78000E9496CA2D9608952F970E948FCAE09119
:10CB8800F108EF73E03100F1E091F108E07CE09307
:10CB9800F108E091EE08E770E062E093EE08A398F0
:10CBA800A498E2B1E67EE2B9E5B1EF70E5B95F9825
:10CBB800EEB1E77CEEB9E1B3EF7CE1BBE4B3E87F2B
:10CBC800E4BBA0E06DD938C2E091EE08E87FE83018
:10CBD80008F432C2E091F108EF730E2FAEEEB8E020
:10CBE80083E0EFE10E944CCCE091EE08E87FE8306A
:10CBF800D1F40031B8F4A1E4B8E0E02FFF276627AC
:10CC08007727E054FF4F6F4F6BBFE691F0E0EE0FD0
:10CC1800FF1FAE0FBF1FED91FC911197E093F50830
:10CC2800F093F60809C2E091EE08E87F09F004C223
:10CC3800E7E0EF83E9EFE887E6E0EA87E985E16086
:10CC4800E987E260E987E091F108EF73EF5FEF733E
:10CC5800EE0FEE0F0E2EE985E370E029E987E0E09C
:10CC6800EB87EC87003108F0AAC1A1E4B8E0E02F17
:10CC7800FF2766277727E054FF4F6F4F6BBFE6917A
:10CC8800F0E0EE0FFF1FAE0FBF1FED91FD91A091D9
:10CC9800F508B091F608AE0FBF1FFD010E941FCB2B
:10CCA8009F01A2E3B0E0E02FF0E0BD01AAE0B0E010
:10CCB8000E9444CBDB01AE0FBF1F0E9482CCAF01A4
:10CCC8004217530718F020E030E0E1C0A2E3B0E0DB
:10CCD800E02FF0E0BD01AAE0B0E00E9444CBDB0108
:10CCE800AE0FBF1F12960E9482CCEB8BFC8BE21713
:10CCF800F30708F1241B350BF901662777276E2FF8
:10CD08007F2FE0E0F0E07F936F93FF93EF93EB8941
:10CD1800FC89E41BF50B66277727AFE8B2E080E0D3
:10CD280090E00E944CCBAF91BF918F919F910E9450
:10CD3800A2CB9F01ACC0A2E3B0E0E02FF0E0BD01C0
:10CD4800AAE0B0E00E9444CBDB01AE0FBF1F1496EF
:10CD58000E9482CCE98BFA8BE217F30730F1AB899A
:10CD6800BC892A1B3B0BD90188279927E1E10E943E
:10CD7800DBCA7F936F93FF93EF93AB89BC89E989F3
:10CD8800FA89EA1BFB0B66277727AFE8B2E080E059
:10CD980090E00E944CCBAF91BF918F919F910E94E0
:10CDA800A2CB9F012C593F4F72C0A2E3B0E0E02F05
:10CDB800F0E0BD01AAE0B0E00E9444CBDB01AE0F79
:10CDC800BF1F16960E9482CCEF87F88BE217F307F5
:10CDD80030F1A989BA892A1B3B0BD90188279927E1
:10CDE800E1E10E94DBCA7F936F93FF93EF93A989D8
:10CDF800BA89EF85F889EA1BFB0B66277727A4EB2E
:10CE0800B1E080E090E00E944CCBAF91BF918F9150
:10CE18009F910E94A2CB9F01245D3E4F38C0A2E3A0
:10CE2800B0E0E02FF0E0BD01AAE0B0E00E9444CB02
:10CE3800DB01AE0FBF1F18960E9482CCED87FE87DC
:10CE4800AF85B8892A1B3B0BD90188279927E3E1CD
:10CE58000E94DBCA7F936F93FF93EF93AF85B889E6
:10CE6800ED85FE85EA1BFB0BF695E7956627772788
:10CE7800ACEEB2E080E090E00E944CCBAF91BF9165
:10CE88008F919F910E94A2CB9F01285A3D4FEBE0C2
:10CE9800F5E060E070E00E9418CCE02FF0E03196F9
:10CEA8006F2F660F660B762F0E9418CCF901662744
:10CEB80077270E941FCDDF01CB01E0E0F0E068ECAE
:10CEC80072E40E94F6CD0E9418CC88E00E9416CA2F
:10CED8002C96F6982B873C8710E0103108F06FC02D
:10CEE8000117B1F5A3E9B8E0E12FFF2766277727F7
:10CEF800E055FF4F6F4F6BBFE691F0E0AE0FBF1FDD
:10CF0800EC91E07421F5EAE1F5E060E070E00E9460
:10CF180018CCE02FF0E031966F2F660F660B762F56
:10CF28000E9418CCE12FF0E031966F2F660F660B48
:10CF3800762F0E9418CC88E00E9416CA2C96E091A1
:10CF4800F208E260E093F208E985ED7FE98735C0F1
:10CF5800A3E9B8E0E12FFF2766277727E055FF4FC1
:10CF68006F4F6BBFE691F0E0AE0FBF1FEC91E0741E
:10CF780021F1E4E3F5E060E070E00E9418CCE02FD6
:10CF8800F0E031966F2F660F660B762F0E9418CC53
:10CF9800E12FF0E031966F2F660F660B762F0E9417
:10CFA80018CC88E00E9416CA2C96E091F208E2603C
:10CFB800E093F208E985ED7FE9871F5F8ECFE09166
:10CFC800F108EF730E2FA02F0E94985FDE011696CE
:10CFD8000E94E7900F3098F4A1EFB8E080E0EFE30B
:10CFE8000E9448CCE091F108EF73AE2F0E94545F85
:10CFF800E091EE08E770E062E093EE081DC0E1E51D
:10D00800F5E060E070E00E9418CC80E00E9416CA4B
:10D018002496E091F208E695E170A0E0EA17E1E0D5
:10D0280009F0EE27AE2F0E940EBBE091EE08E87FD4
:10D03800E093EE08A398A4980E9496CA659608956E
:10D0480026970E948FCAEDE5F5E060E070E00E9447
:10D0580018CCABE1B0E00E9482CC662777270E940B
:10D0680018CC84E00E9416CA2896ABE1B0E00E9472
:10D0780082CCE03CA3E3FA0740F0ABE1B0E00E94C9
:10D0880082CCE134AFE3FA0708F002C021E001C026
:10D0980020E0A22F0E940EBBEEE6F5E060E070E013
:10D0A8000E9418CCADE1B0E00E9482CC66277727B9
:10D0B8000E9418CCAFE1B0E00E9482CC66277727A7
:10D0C8000E9418CC88E00E9416CA2C96ADE1B0E008
:10D0D8000E9482CCE53AA7E1FA07C0F0ADE1B0E0E2
:10D0E8000E9482CCE73EACE1FA0780F4AFE1B0E001
:10D0F8000E9482CCE53AA7E1FA0740F0AFE1B0E040
:10D108000E9482CCE73EACE1FA0708F002C051E089
:10D1180001C050E0A52F0E940EBBE7E8F5E060E0F3
:10D1280070E00E9418CCA2E2B0E00E9486CCFF27F3
:10D13800662777270E9418CC84E00E9416CA289692
:10D14800E0E01E2F3E2F103108F03FC1ECE9F5E07A
:10D1580060E070E00E9418CCE12FF0E031966F2F6C
:10D16800660F660B762F0E9418CCA2E3B0E0E12F81
:10D17800F0E0BD01AAE0B0E00E9444CBDB01AE0FB5
:10D18800BF1F0E9482CC662777270E9418CCA2E393
:10D19800B0E0E12FF0E0BD01AAE0B0E00E9444CB8E
:10D1A800DB01AE0FBF1F12960E9482CC662777273D
:10D1B8000E9418CCA2E3B0E0E12FF0E0BD01AAE0A4
:10D1C800B0E00E9444CBDB01AE0FBF1F14960E9453
:10D1D80082CC662777270E9418CCA2E3B0E0E12F23
:10D1E800F0E0BD01AAE0B0E00E9444CBDB01AE0F45
:10D1F800BF1F16960E9482CC662777270E9418CCFC
:10D20800A2E3B0E0E12FF0E0BD01AAE0B0E00E94A7
:10D2180044CBDB01AE0FBF1F18960E9482CC662755
:10D2280077270E9418CC88E10E9416CA6C9600E005
:10D2380000E0053008F0B6C0E02FF0E0309769F460
:10D24800A2E3B0E0E12FF0E0BD01AAE0B0E00E9467
:10D2580044CBDB01AE0FBF1F47C0E130A0E0FA07A7
:10D2680071F4A2E3B0E0E12FF0E0BD01AAE0B0E084
:10D278000E9444CBDB01AE0FBF1F129635C0E230CF
:10D28800A0E0FA0771F4A2E3B0E0E12FF0E0BD01FD
:10D29800AAE0B0E00E9444CBDB01AE0FBF1F14969A
:10D2A80023C0E330A0E0FA0771F4A2E3B0E0E12F75
:10D2B800F0E0BD01AAE0B0E00E9444CBDB01AE0F74
:10D2C800BF1F169611C0E430A0E0FA0789F4A2E364
:10D2D800B0E0E12FF0E0BD01AAE0B0E00E9444CB4D
:10D2E800DB01AE0FBF1F18960E9482CCEE83FF832E
:10D2F800E12FFF2766277727E053FF4F6F4F6BBF5C
:10D30800E691E030C1F4E02FA6E5B1E080E0FF2728
:10D3180066277727EE0FFF1F661F771FEA0FFB1F91
:10D32800681F791F0E9407CCEA87FB87E02FA6E7D2
:10D33800B1E080E017C0E02FA6E9B1E080E0FF2768
:10D3480066277727EE0FFF1F661F771FEA0FFB1F61
:10D35800681F791F0E9407CCEA87FB87E02FA6EB9E
:10D36800B1E080E0FF2766277727EE0FFF1F661FD3
:10D37800771FEA0FFB1F681F791F0E9407CCE887F9
:10D38800F987EE81FF81AA85BB85EA17FB0738F08C
:10D39800E885F985AE81BF81EA17FB0708F402C06A
:10D3A8000F5F47CFA02FE5E0EA17E1E009F0EE278D
:10D3B800AE2F0E940EBB053010F4303009F003C0C8
:10D3C800E12FEF5F3E2F1F5FBECEE7EEF4E060E097
:10D3D80070E00E9418CC80E00E9416CA2496A2E24F
:10D3E800B0E00E9486CCEF3181F5203029F4EBEBD8
:10D3F800F5E060E070E022C0503029F4EEECF5E092
:10D4080060E070E01BC03130A8F0E6EFF4E060E0C7
:10D4180070E00E9418CCE091F208E695E695EF716D
:10D42800FF27662777270E9418CC84E00E9416CA37
:10D4380028960AC0E2EFF4E060E070E00E9418CCA1
:10D4480080E00E9416CA24960AC0E0EEF5E060E08B
:10D4580070E00E9418CC80E00E9416CA24960E94B0
:10D4680096CA2C9608950E9491CA0A2F3C813031A1
:10D4780008F03FC0A9E03A9FF001E950F74FDF01FB
:10D48800EC91E068EC9330FF1CC03695A7E6B9E054
:10D49800EE27A30FBE1F0E9486CC1E2F023019F460
:10D4A800E07FE03169F01F70E02FE295E07F1E2BEE
:10D4B800A7E6B9E0EE27A30FBE1FE12F0E94A2CC7A
:10D4C80018C03695A7E6B9E0EE27A30FBE1F0E9445
:10D4D80086CC1E2F023019F4EF70E13051F0107F26
:10D4E800102BA7E6B9E0EE27A30FBE1FE12F0E947D
:10D4F800A2CC0E9498CA259608951A930A930A2FD7
:10D50800E3EFF5E060E070E00E9418CCE02FFF2721
:10D51800662777270E9418CC84E00E9416CA2896AE
:10D52800003108F046C0A9E00A9FF001E950F74F22
:10D53800DF01EC91EF77EC93A9E00A9FF001E75047
:10D54800F74FDF01EC91E07FEC9300FF02C01FE092
:10D5580001C010EFA7E6B9E0E02FF0E0F595E795F8
:10D56800AE0FBF1F0E9486CCE1230E94A2CCA9E087
:10D578000A9FF001E950F74FE081E17089F00A9FB6
:10D58800F001E950F74FE081E077E03440F00A9F7E
:10D59800F001E950F74FDF01EC91EF78EC9309C007
:10D5A800A9E00A9FF001E950F74FDF01EC91EF780D
:10D5B800EC930991199108950E948FCAE091EE08A1
:10D5C800E770E23008F0F6C1A7E2B1E00E9486CC2D
:10D5D800E03079F0A7E2B1E00E9486CCAE2F0E943D
:10D5E8007A3BA0EFB8E0E1700E2EEC91EE7FE029D7
:10D5F800EC93A8E2B1E00E9486CCE03081F0A8E28A
:10D60800B1E00E9486CCAE2F0E947A3BA0EFB8E032
:10D61800E170EE0F0E2EEC91ED7FE029EC931FE008
:10D62800103108F0C7C1A9E01A9FF001E650F74F82
:10D638002081263309F4BCC1A9E01A9FF001E95002
:10D64800F74FE081E295E7705E2F40E0E091EE0849
:10D65800E770E13041F41A9FF001E950F74FE0819B
:10D66800E1703E2F73C0273B09F4A2C1A9E01A9FBD
:10D67800F001E950F74FE081E27009F441C0A5E4F8
:10D68800B1E0E12FF0E0BD01A7E0B0E00E9444CB9B
:10D69800DB01AE0FBF1F12960E9486CCE07121F00D
:10D6A800E091F008E17059F5A5E4B1E0E12FF0E070
:10D6B800BD01A7E0B0E00E9444CBDB01AE0FBF1F65
:10D6C80012960E9486CCE07221F0E091F008E27098
:10D6D800B1F4A5E4B1E0E12FF0E0BD01A7E0B0E0CE
:10D6E8000E9444CBDB01AE0FBF1F12960E9486CC6E
:10D6F800E07421F0E091EF08E07809F401C001C07E
:10D7080002C030E016C0A22F0E947A3B3E2FA9E04B
:10D718001A9FF001E850F74FE081E07121F0E091A5
:10D72800910DE17009F405C0303011F030E001C00E
:10D7380031E0A9E01A9FF001E950F74FDF01E32F2C
:10D74800E1700E2EEC91EE7FE029EC93303069F118
:10D75800E52FF0E0309721F0E130A0E0FA07D9F4A6
:10D76800E091EF08E770E23098F0E2E0F6E060E080
:10D7780070E00E9418CCE12FF0E031966F2F660F11
:10D78800660B762F0E9418CC84E00E9416CA289651
:10D7980041E052E009C0E430A0E0FA0721F0E530AA
:10D7A800A0E0FA0709F442E029C0503011F05130E6
:10D7B80009F424C042E050E0A9E01A9FF001E950C2
:10D7C800F74FDF01EC91EB7FEC93A9E01A9FF00192
:10D7D800E250F74FA0E0B0E0A083B183A9E01A9F20
:10D7E800F001E550F74FA0E0A083A9E01A9FF001EF
:10D7F800E750F74FDF01EC91E07FEC93E42FF0E086
:10D80800309709F484C0E130A0E0FA0709F05CC061
:10D81800A12F0E94545FA9E01A9FF001E850F74F2A
:10D82800DF01EC91E068EC93A9E01A9FF001E55064
:10D83800F74FA0E0A083A9E01A9FF001E750F74F47
:10D84800DF01EC91E07FEC93A9E01A9FF001E8502A
:10D85800F74FE081E074B9F1E12FFF2766277727BA
:10D86800E056FF4F6F4F6BBF06910A9FF001E950DA
:10D87800F74FDF01EC91E160EC93A9E00A9FF0011A
:10D88800E950F74FDF01EC91EF78E062EC93A9E003
:10D898000A9FF001E850F74FDF01EC91E068EC9344
:10D8A800A9E00A9FF001E550F74FA0E0A083A9E0A6
:10D8B8000A9FF001E750F74FDF01EC91E07FEC930E
:10D8C800A02F0E94545F23C0E230A0E0FA07F9F4C9
:10D8D800A12F0E94045FA9E01A9FF001E850F74FBA
:10D8E800E081E074A1F0E12FFF2766277727E05653
:10D8F800FF4F6F4F6BBF06910A9FF001E950F74F3A
:10D90800DF01EC91EE7FEC93A02F0E94045FE09181
:10D91800EF08E770E23050F0A9E01A9FF001E950F3
:10D92800F74FE081E295E7705E1709F432C0EEE048
:10D93800F6E060E070E00E9418CCE12FF0E031964C
:10D948006F2F660F660B762F0E9418CCA9E01A9FDE
:10D95800F001E950F74FE081E295E770FF2766276D
:10D9680077270E9418CCE52FFF27662777270E9484
:10D9780018CCE32FFF27662777270E9418CCE42FBF
:10D98800FF27662777270E9418CC84E10E9416CAD1
:10D998006896A9E01A9FF001E950F74FDF01E52FDB
:10D9A800E770E295E07F0E2EEC91EF78E029EC939A
:10D9B800115036CE0E9496CA2696089527970E943F
:10D9C80091CA8D013B852C85E7E0ED83E9EFEE8375
:10D9D800EF81E160EF83E32FE170EE0F0E2EEF8110
:10D9E800ED7FE029EF83203011F4E7E001C0E8E0A3
:10D9F800E887E22FEF73EE0FEE0F0E2EEF81E37044
:10DA0800E029EF8309871A87DE0114960E94E790C0
:10DA1800A32F0E940EBB0E9498CA2D960895629764
:10DA28000E948FCAE091EE08E770E23080F0E09142
:10DA3800EE08E770E73011F49FD802C00E94DE625A
:10DA4800E4E1E093F3080E9496CA68960895E0E03E
:10DA5800F0E0E093F508F093F608E091F208E17041
:10DA6800C9F1E091F208EE7FE093F208EEE2F6E009
:10DA780060E070E00E9418CC80E00E9416CA2496EC
:10DA8800E0E0EB8BAB89A03210F5E3E3F6E060E071
:10DA980070E00E9418CCEF89FF27662777270E943D
:10DAA80018CCA1E4B8E0EB8DF0E0EE0FFF1FAE0F4D
:10DAB800BF1FED91FD91662777270E9418CC88E05B
:10DAC8000E9416CA2C96EB89EF5FEB8BDBCFAAE09E
:10DAD8000E942590ABE1B0E00E9482CCED87FE87E2
:10DAE800A091970DB091980DE0916308F0916408AA
:10DAF8000E941FCBEA0FFB1FE093970DF093980D40
:10DB0800E091960DEF70E93038F4A6E9BDE080E0C9
:10DB1800EFE00E9448CC6BC0E091960DE071D1F126
:10DB2800E091960DEF7EE093960DABE1B0E0E091C9
:10DB3800970DF091980D0E949ACCE6E0E093940D31
:10DB4800EAE3F6E060E070E00E9418CCE091970DFF
:10DB5800F091980D662777270E9418CC84E00E94E0
:10DB680016CA2896E0E0EA93A091970DB091980D17
:10DB7800A03CE3E3BE0730F0A134EFE3BE0710F4A6
:10DB8800E1E001C0E0E0EA93A091970DB091980D13
:10DB980015DF22C0E091970DF091980D6627772741
:10DBA800E987FA876B877C87A0EEBEE280E090E089
:10DBB8000E944CCBE987FA876B877C87ED85FE85C9
:10DBC800A985BA858B859C85662777270E94A2CB75
:10DBD800E093990DF0939A0DE091960DE07FE09314
:10DBE800960DE0E0F0E0E093970DF093980DE0914A
:10DBF8006308F091640866277727E987FA876B87B7
:10DC08007C87ACE2B1E080E090E00E944CCBE987F1
:10DC1800FA876B877C87ED85FE85F695E795A9855C
:10DC2800BA858B859C8566277727EA0FFB1F681FB7
:10DC3800791FE987FA876B877C87ED85FE85A9853B
:10DC4800BA858B859C85662777270E94A2CBE093AF
:10DC58009B0DAAE2B1E00E9486CCE13008F4A1C095
:10DC6800E091EF08E07809F443C0A091990DB091D4
:10DC78009A0DE4E6F0E00E948ACB0F01ACE2B1E035
:10DC88000E9486CCD001F0E0AE17BF0768F1ADE284
:10DC9800B1E00E9486CCA091F408AE1738F4E09168
:10DCA800F408EF5FE093F408E1501DC0E4E4F6E007
:10DCB80060E070E00E9418CCE091990DF0919A0D07
:10DCC800662777270E9418CC84E00E9416CA2896F7
:10DCD800A9E00E944C27E091EF08EF77E093EF0866
:10DCE800E0E0E093F40803C0E0E0E093F40859C0F2
:10DCF800E0E0EA8BABE2B1E00E9486CCEA3058F46F
:10DD0800AAE2B1E00E9486CCA0919B0DAE1710F458
:10DD1800E1E0EA8B14C0A091990DB0919A0DE4E668
:10DD2800F0E00E948ACB0F01AAE2B1E00E9486CC03
:10DD3800D001F0E0AE17BF0710F4E1E0EA8BEA8902
:10DD4800E03061F1ABE2B1E00E9486CCA091F4082A
:10DD5800AE1738F4E091F408EF5FE093F408E1506F
:10DD68001CC0E4E5F6E060E070E00E9418CCE091A9
:10DD78009B0DFF27662777270E9418CC84E00E9416
:10DD880016CA2896A8E00E944C27E091EF08E068A0
:10DD9800E093EF08E0E0E093F40803C0E0E0E093EC
:10DDA800F408A0919B0DA83330F5E091F308E0301A
:10DDB800E9F4E5E6F6E060E070E00E9418CCE09156
:10DDC8009B0DF0E06F2F660F660B762F0E941FCD1C
:10DDD800DF01CB01E0E0F0E060E271E40E94F6CD03
:10DDE8000E9418CC84E00E9416CA2896EAE0E093C4
:10DDF800F308F19A35C0A091F308A13088F1E091B9
:10DE0800F308E150E093F308EF5FE091F308E030A6
:10DE180039F5E091EF08E07411F1E091EF08EF7B3C
:10DE2800E093EF08EDE7F6E060E070E00E9418CCC0
:10DE3800E0919B0DF0E06F2F660F660B762F0E9426
:10DE48001FCDDF01CB01E0E0F0E060E271E40E9469
:10DE5800F6CD0E9418CC84E00E9416CA2896F19844
:10DE6800A091F308E0E0EA17E1E008F0EE27E88B7C
:10DE7800A0913F08A13008F490C0E0913F08F0E07D
:10DE8800E130A0E0FA07C1F5E0917108F09172085D
:10DE980066277727A8EEB3E080E090E00E944CCB9D
:10DEA8007F936F93FF93EF93ADE1B0E00E9482CC34
:10DEB800AF91BF918F919F91662777270E94A2CB40
:10DEC800E0937508F0937608A0917508B0917608EC
:10DED800139718F4E0E0F0E00AC0A0917508B0913B
:10DEE8007608A93FE7E0BE0730F0E8EFF7E0E093F7
:10DEF8007508F093760851C0E230A0E0FA0721F4E3
:10DF0800E3E0E0933F0849C0E330A0E0FA0709F0F6
:10DF180044C0E1E0E0933F08E0917108F091720895
:10DF2800F695E795ED87FE87ADE1B0E00E949ACCC3
:10DF3800E4E9F6E060E070E00E9418CCE989FA892B
:10DF4800662777270E9418CC84E00E9416CA289674
:10DF5800E3E0EA93EE85FF85E53AA7E1FA0740F0AA
:10DF6800AE85BF85A73EECE1BE0710F4E1E001C035
:10DF7800E0E0EA93AF85B88921DDE1E0E0933F086E
:10DF8800E6E0E093940DA0914008A23020F4F49BC1
:10DF980002C0F59B01C001C0159AA0914008A130AC
:10DFA80008F490C0E0914008F0E0E130A0E0FA0702
:10DFB800C1F5A0914108B091420888279927E8EE59
:10DFC800F3E060E070E00E944CCB7F936F93FF9387
:10DFD800EF93AFE1B0E00E9482CCAF91BF918F91F7
:10DFE8009F91662777270E94A2CBE0937708F0934A
:10DFF8007808A0917708B0917808139718F4E0E0B2
:10E00800F0E00AC0A0917708B0917808A93FE7E04E
:10E01800BE0730F0E8EFF7E0E0937708F093780870
:10E0280051C0E230A0E0FA0721F4E3E0E0934008B1
:10E0380049C0E330A0E0FA0709F044C0E1E0E0930A
:10E048004008E0914108F0914208F695E795ED8780
:10E05800FE87AFE1B0E00E949ACCE6E0E093940D31
:10E06800E0EAF6E060E070E00E9418CCE989FA89FD
:10E07800662777270E9418CC84E00E9416CA289643
:10E08800E4E0EA93EE85FF85E53AA7E1FA0740F078
:10E09800AE85BF85A73EECE1BE0710F4E1E001C004
:10E0A800E0E0EA93AF85B88989DCE1E0E0934008D5
:10E0B800A0913F08A23020F4F49B02C0F59B01C058
:10E0C80001C0159AEFE0EB8BAB89A03108F0AEC622
:10E0D800EB89A9E0EA9FF001E850F74FE081E0788A
:10E0E80049F0EB89EA9FF001E850F74FDF01EC9126
:10E0F800EF7797C6EB89A9E0EA9FF001E650F74F62
:10E10800E081E887E0E0EE83EF87A885A633D9F4BD
:10E11800EB89FF2766277727E056FF4F6F4F6BBFC6
:10E12800E691A9E0EA9FF001E950F74FE081E1703C
:10E13800E98BEB89FF2766277727E056FF4F6F4F5C
:10E148006BBFE6910AC0EB89A9E0EA9FF001E950AC
:10E15800F74FE081E170E98BEB89A9E0EA9FF001D4
:10E16800E950F74FE081E295E770EF83E989E03005
:10E1780009F4F5C4A1E4B8E0EB89FF2766277727FF
:10E18800E054FF4F6F4F6BBFE691F0E0EE0FFF1FBB
:10E19800AE0FBF1FED91FD91F695E795ED87FE87D0
:10E1A800A2E3B0E0EB89F0E0BD01AAE0B0E00E9494
:10E1B80044CBDB01AE0FBF1F0E9482CC8F01AD851F
:10E1C800BE850A171B0720F0E0E0ED87EE87F1C057
:10E1D800A2E3B0E0EB89F0E0BD01AAE0B0E00E9464
:10E1E80044CBDB01AE0FBF1F12960E9482CC9F0169
:10E1F800AD85BE852A173B0710F1ED85FE85E01B2E
:10E20800F10BED87FE87662777276E2F7F2FE0E0DB
:10E21800F0E07F936F93FF93EF93F901E01BF10B0D
:10E2280066277727AFE8B2E080E090E00E944CCB09
:10E23800AF91BF918F919F910E94A2CBB8C0A2E3EA
:10E24800B0E0EB89F0E0BD01AAE0B0E00E9444CB69
:10E25800DB01AE0FBF1F14960E9482CCAF01AD85C3
:10E26800BE854A175B0738F1ED85FE85E21BF30B87
:10E27800ED87FE87AD85BE8588279927E1E10E9455
:10E28800DBCA7F936F93FF93EF93FA01E21BF30BC3
:10E2980066277727AFE8B2E080E090E00E944CCB99
:10E2A800AF91BF918F919F910E94A2CBED87FE877E
:10E2B800EC59FF4F7CC0A2E3B0E0EB89F0E0BD0170
:10E2C800AAE0B0E00E9444CBDB01AE0FBF1F169658
:10E2D8000E9482CCEE8BFF8BAD85BE85EA17FB07CB
:10E2E80040F1ED85FE85E41BF50BED87FE87AD85D6
:10E2F800BE8588279927E1E10E94DBCA7F936F9347
:10E30800FF93EF93EE89FF89E41BF50B66277727C8
:10E31800A4EBB1E080E090E00E944CCBAF91BF91BC
:10E328008F919F910E94A2CBED87FE87E45DFE4FFF
:10E338003EC0A2E3B0E0EB89F0E0BD01AAE0B0E0A6
:10E348000E9444CBDB01AE0FBF1F18960E9482CCFF
:10E35800EC8BFD8BAE89BF89ED85FE85EA1BFB0B37
:10E36800ED87FE87AD85BE8588279927E3E10E9462
:10E37800DBCA7F936F93FF93EF93AE89BF89EC89D4
:10E38800FD89EA1BFB0BF695E79566277727ACEE28
:10E39800B2E080E090E00E944CCBAF91BF918F91AA
:10E3A8009F910E94A2CBED87FE87E85AFD4FED872B
:10E3B800FE87A885A73BA1F0A63389F4EB89FF2740
:10E3C80066277727E056FF4F6F4F6BBFE691A9E0AE
:10E3D800EA9FF001E650F74FA081A73B09F06EC015
:10E3E800A885A73B19F4EB89EA8B0AC0EB89FF27BC
:10E3F80066277727E056FF4F6F4F6BBF06900A8A54
:10E40800A2E9B9E0EA89FF2766277727E052FF4F9C
:10E418006F4F6BBFE691F0E00E940BCBAE0FBF1FB2
:10E428001196AC91A83C11F4E0E001C0E1E0EF875F
:10E43800AD85BE85A130E0E4BE0720F0E0E0F0E461
:10E44800ED87FE87EB89A9E0EA9FF001E450F74FDA
:10E45800CF0160817181EB89A9E0EA9FF001E45066
:10E46800F74FDF01ED91FD910E941BCBDF01FB010E
:10E47800EA1BFB0BDC01ED93FC93EB89A9E0EA9F17
:10E48800F001E450F74F0F01DF01ED91FD91DF013D
:10E49800ED85FE850E941FCBEA0FFB1FD001ED938F
:10E4A800FC93EB89A9E0EA9FF001E450F74FDF0104
:10E4B800ED91FD910E941FCBED87FE87E091F50855
:10E4C800F091F608AD85BE85EA0FFB1FE093F508CD
:10E4D800F093F608EB89A9E0EA9FF001E850F74FBE
:10E4E800E081E074B1F0EB89FF2766277727E056D3
:10E4F800FF4F6F4F6BBFE691EA9FF001E250F74F75
:10E50800DF01ED91FD91AD85BE85EA0FFB1FED871B
:10E51800FE87AD85BE85A73FE7E2BE0720F0E6EFA0
:10E52800F7E2ED87FE87EB89A9E0EA9FF001E25068
:10E53800F74FAD85BE85A083B183E091EF08E87001
:10E54800C9F0ECEAF6E060E070E00E9418CCEF89D0
:10E55800F0E031966F2F660F660B762F0E9418CC6D
:10E56800ED89FE89662777270E9418CC88E00E94EB
:10E5780016CA2C96EF81F0E0E230A0E0FA0709F025
:10E58800A3C0A889A03039F5A7ECB8E0EB89FF272C
:10E5980066277727E054FF4F6F4F6BBFE691F0E097
:10E5A800AE0FBF1FAC91A230A8F4AF85A03089F49C
:10E5B800A9E7B8E0EB89FF2766277727E055FF4FE3
:10E5C8006F4F6BBFE691F0E0AE0FBF1FEC91E074A8
:10E5D80009F401C001C04FC0EB89A9E0EA9FF0012E
:10E5E800E750F74FE081EF70E43058F4EB89EA9F89
:10E5F800F001E750F74FDF0180E0EFE00E9448CCE0
:10E608003AC0E5E0EF83E2E0EE83EB89EA93A3E02A
:10E618000E94376AEB89A9E0EA9FF001E850F74FBA
:10E62800E081EF70EA3098F4EB89EA9FF001E85056
:10E63800F74FDF0180E0EFE00E9448CCE6E6EA937E
:10E64800EC89E15FEA93A0E0B0E00E945527E8EB8F
:10E65800F6E060E070E00E9418CCEF89F0E03196B7
:10E668006F2F660F660B762F0E9418CC84E00E94ED
:10E6780016CA289673C2EB89A9E0EA9FF001E55013
:10E68800F74FA081A53058F4EB89A9E0EA9FF00183
:10E69800E550F74FDF01EC91EF5FEC9314C0EB8985
:10E6A800A9E0EA9FF001E550F74FA0E0A083EB89CD
:10E6B800A9E0EA9FF001E750F74FDF01EC91E07F16
:10E6C800EC93E3E0EF834AC2E330A0E0FA0709F0F5
:10E6D80045C2A889A03039F5A7ECB8E0EB89FF2737
:10E6E80066277727E054FF4F6F4F6BBFE691F0E046
:10E6F800AE0FBF1FAC91A230A8F4AF85A03089F44B
:10E70800A9E7B8E0EB89FF2766277727E055FF4F91
:10E718006F4F6BBFE691F0E0AE0FBF1FEC91E07456
:10E7280009F401C001C050C0EB89A9E0EA9FF001DB
:10E73800E750F74FE081EF70E33058F4EB89EA9F38
:10E74800F001E750F74FDF0180E0EFE00E9448CC8E
:10E758003AC0E5E0EF83E2E0EE83EB89EA93A3E0D9
:10E768000E94376AEB89A9E0EA9FF001E850F74F69
:10E77800E081EF70EA3098F4EB89EA9FF001E85005
:10E78800F74FDF0180E0EFE00E9448CCE6E6EA932D
:10E79800EC89E15FEA93A0E0B0E00E945527E7EC3E
:10E7A800F6E060E070E00E9418CCEF89F0E0319666
:10E7B8006F2F660F660B762F0E9418CC84E00E949C
:10E7C80016CA2896CBC114C0EB89A9E0EA9FF001CC
:10E7D800E750F74FE081EF70E13050F0EB89EA9FA6
:10E7E800F001E750F74FDF0180E0EFE00E944CCCEA
:10E7F800A885A63309F4B2C1A5E4B1E0EB89F0E03D
:10E80800BD01A7E0B0E00E9444CBDB01AE0FBF1F03
:10E8180014960E9482CCFF71ED87FE87EB89A9E0F0
:10E82800EA9FF001E650F74FA081A73B79F4E09109
:10E83800EE08E770E13049F4EB89A9E0EA9FF001BE
:10E84800E950F74FE081E17009F401C035C0A2E951
:10E85800B9E0EB89FF2766277727E052FF4F6F4F14
:10E868006BBFE691F0E00E940BCBAE0FBF1F119675
:10E87800EC91EA8BE03029F4ED85FE850E941DCBF2
:10E8880019C0EA89EC5EEA8BAA89A83CA8F4AD8590
:10E89800BE8588279927F0E06F2F660F660B762FC5
:10E8A8000E944CCBDF01CB01E8ECF0E060E070E0C7
:10E8B8000E94A2CBED87FE87EB89A9E0EA9FF001D1
:10E8C800E250F74FDF01ED91FD91DF01ED85FE8507
:10E8D800AE17BF0708F48CC0EB89A9E0EA9FF001E6
:10E8E800E950F74FDF01EC91EB7FEC93EB89A9E05E
:10E8F800EA9FF001E950F74FE081E87091F4EB8965
:10E90800EA9FF001E950F74FDF01EC91E860EC93E2
:10E91800EB89A9E0EA9FF001E550F74FA0E0A0835A
:10E9280066C0EB89A9E0EA9FF001E550F74FDF01E7
:10E93800EC91EF5FEC93EB89A9E0EA9FF001E550D9
:10E94800F74FE081EF93A5E4B1E0EB89F0E0BD017A
:10E95800A7E0B0E00E9444CBDB01AE0FBF1F1696C4
:10E968000E9486CCAF91AE1708F441C0E4E0EF8373
:10E97800E2E0EE83EB89EA93A4E00E94376AEB8930
:10E98800A9E0EA9FF001E850F74FE081EF70EA3024
:10E99800D8F4EB89EA9FF001E850F74FDF0180E0F7
:10E9A800EFE00E9448CCE7E6EA93EC89E15FEA935E
:10E9B800ED89A9E0EA9FF001E250F74FDF01ED9100
:10E9C800FD91DF010E945527E6EDF6E060E070E07A
:10E9D8000E9418CCEF89F0E031966F2F660F660B16
:10E9E800762F0E9418CC84E00E9416CA2896B6C0DA
:10E9F800EB89A9E0EA9FF001E950F74FE081E87060
:10EA080089F0EB89EA9FF001E950F74FDF01EC91BB
:10EA1800E77FEC93EB89A9E0EA9FF001E550F74F17
:10EA2800A0E0A083A5E4B1E0EB89F0E0BD01A7E098
:10EA3800B0E00E9444CBDB01AE0FBF1F11960E94CD
:10EA480082CCFF70ED87FE87AD85BE8500240A164F
:10EA58000B0608F083C0EB89A9E0EA9FF001E250B9
:10EA6800F74FDF01ED91FD91AD85BE85EA17FB07F4
:10EA780008F062C0EB89A9E0EA9FF001E550F74F82
:10EA8800E081EF93A5E4B1E0EB89F0E0BD01A7E0F8
:10EA9800B0E00E9444CBDB01AE0FBF1F13960E946B
:10EAA80086CCAF91AE1758F4EB89A9E0EA9FF00144
:10EAB800E550F74FDF01EC91EF5FEC933CC0EB8939
:10EAC800A9E0EA9FF001E950F74FE081E47099F579
:10EAD800EB89EA9FF001E950F74FDF01EC91E46020
:10EAE800EC93EB89EA93A2E00E94376AEB89A9E0EC
:10EAF800EA9FF001E850F74FE081EF70EA30D8F470
:10EB0800EB89EA9FF001E850F74FDF0180E0EFE082
:10EB18000E9448CCE5E6EA93EC89E15FEA93ED8947
:10EB2800A9E0EA9FF001E250F74FDF01ED91FD9176
:10EB3800DF010E94552712C0EB89A9E0EA9FF00186
:10EB4800E550F74FA0E0A083EB89A9E0EA9FF00128
:10EB5800E950F74FDF01EC91EB7FEC93D0C0EB89E4
:10EB6800A9E0EA9FF001E250F74FA0E0B0E0A083EF
:10EB7800B183EB89A9E0EA9FF001E450F74FA0E0E8
:10EB8800B0E0A083B183A885A63389F0A5E4B1E0FD
:10EB9800EB89F0E0BD01A7E0B0E00E9444CBDB01C7
:10EBA800AE0FBF1F12960E9486CCE07809F4A7C06A
:10EBB800EF81F0E0309709F06CC0E889E03009F0A7
:10EBC8009EC0A3E9B8E0EB89FF2766277727E055C1
:10EBD800FF4F6F4F6BBFE691F0E0AE0FBF1FEC9198
:10EBE800E07459F4EB89A9E0EA9FF001E750F74F88
:10EBF800DF01EC91E07FEC934BC0EB89A9E0EA9F41
:10EC0800F001E750F74FE081EF70EF3058F4EB89EF
:10EC1800EA9FF001E750F74FDF0180E0EFE00E9444
:10EC280048CC36C0E1E0EF83EB89A9E0EA9FF00128
:10EC3800E750F74FDF01EC91E07FEC93EB89EA9323
:10EC4800A1E00E94376AEB89A9E0EA9FF001E85049
:10EC5800F74FE081EF70EA30D8F4EB89EA9FF001D2
:10EC6800E850F74FDF0180E0EFE00E9448CCE4E68F
:10EC7800EA93EC89E15FEA93ED89A9E0EA9FF00164
:10EC8800E250F74FDF01ED91FD91DF010E9455271A
:10EC980036C0E130A0E0FA0791F5A3E9B8E0EB89C6
:10ECA800FF2766277727E055FF4F6F4F6BBFE69129
:10ECB800F0E0AE0FBF1FEC91E07409F5EB89A9E015
:10ECC800EA9FF001E750F74FE081EF70EF3058F41A
:10ECD800EB89EA9FF001E750F74FDF0180E0EFE0B2
:10ECE8000E9448CC0CC0E0E0EF83EB89A9E0EA9FE2
:10ECF800F001E750F74FDF01EC91E07FEC93AE8134
:10ED0800A230B1F5AB890E94045FEB89A9E0EA9FC4
:10ED1800F001E850F74FE081E07419F4A885A633B4
:10ED280039F5EB89FF2766277727E056FF4F6F4FA6
:10ED38006BBF06900A8AEA89A9E0EA9FF001E950C8
:10ED4800F74FDF01EC91EE7FEC93EA89A9E0EA9FA7
:10ED5800F001E950F74FDF01EF81E770E295E07FBE
:10ED68000E2EEC91EF78E029EC93AA890E94045FBB
:10ED7800AE81A23009F046C0E091EF08E770E230BA
:10ED880068F0EB89A9E0EA9FF001E950F74FE081CC
:10ED9800E295E770AE2FEF81EA1709F433C0E5EE8C
:10EDA800F6E060E070E00E9418CCEF89F0E0319660
:10EDB8006F2F660F660B762F0E9418CCEB8DA9E09B
:10EDC800EA9FF001E950F74FE081E295E770FF27ED
:10EDD800662777270E9418CCEB89FF2766277727B5
:10EDE8000E9418CCE9A1FF27662777270E9418CC34
:10EDF800EA8DFF27662777270E9418CC84E10E94B6
:10EE080016CA6896EB89A9E0EA9FF001E950F74F26
:10EE1800DF01EF81E770E295E07F0E2EEC91EF784D
:10EE2800E029EC93EB89E150EB8B4EC9E091EF08B8
:10EE3800E87009F475C0E6E0F7E060E070E00E9471
:10EE480018CC80E00E9416CA2496E0E0EB8BAB89D0
:10EE5800A03108F060C0EB89A9E0EA9FF001E95011
:10EE6800F74FE081E17009F452C0E0E1F7E060E0BB
:10EE780070E00E9418CCEF89F0E031966F2F660F92
:10EE8800660B762F0E9418CCA3E9B8E0EB8DFF271C
:10EE980066277727E055FF4F6F4F6BBFE691F0E08D
:10EEA800AE0FBF1FEC91E07411F0E1E001C0E0E0AB
:10EEB8000E9424CB0E9418CCA1E4B8E0EF8DFF2774
:10EEC80066277727E054FF4F6F4F6BBFE691F0E05E
:10EED800EE0FFF1FAE0FBF1FED91FD91662777273D
:10EEE8000E9418CCEBA1A9E0EA9FF001E250F74F8D
:10EEF800DF01ED91FD91AAE0B0E00E9444CB6627C6
:10EF080077270E9418CC80E10E9416CA6496EB8984
:10EF1800EF5FEB8B9CCFE091EF08E77FE093EF0882
:10EF28000E9496CA689608950E948FCAE0E05E2FF4
:10EF38002E2F3E2F0E2F10E01C3040F5A7E6B9E02B
:10EF4800EE27A10FBE1F0E9486CCE03009F021E019
:10EF5800A9E01A9FF001E950F74FE081F0E00E9424
:10EF68001BCBE770F070E130A0E0FA0711F451E034
:10EF78000BC0E430A0E0FA0711F431E005C0E53039
:10EF8800A0E0FA0709F401E01F5FD6CF10E01830BF
:10EF980040F5A3E7B9E0EE27A10FBE1F0E9486CC7B
:10EFA800E03009F021E0A9E01A9FF001E950F74F9D
:10EFB800E081F0E00E941BCBE770F070E130A0E048
:10EFC800FA0711F451E00BC0E430A0E0FA0711F49D
:10EFD80031E005C0E530A0E0FA0709F401E01F5F61
:10EFE800D6CFA0EFB8E0E02FE170EE0FEE0F0E2EB7
:10EFF800EC91EB7FE029EC93A0EFB8E0E32FE17010
:10F00800EE0FEE0FEE0F0E2EEC91E77FE029EC935A
:10F01800A0EFB8E0E22FE170E295E07FEE0F0E2E50
:10F02800EC91EF7DE029EC93A0EFB8E0E52FE170DB
:10F03800E295E07F0E2EEC91EF7EE029EC930E94A2
:10F0480096CA269608951A93EAE2F7E060E070E01F
:10F058000E9418CC80E00E9416CA2496ABE7B9E05B
:10F06800E0E0F0E00E949ACC10E01031F0F5A9E061
:10F078001A9FF001E850F74FDF01EC91E07FEC9325
:10F08800A9E01A9FF001E950F74FDF01EC91EF7703
:10F09800EC93A9E01A9FF001E750F74FDF01EC91DC
:10F0A800E07FEC93A9E01A9FF001E950F74FE08167
:10F0B800F0E00E941BCBE770F070E130A0E0FA07A7
:10F0C80021F0E430A0E0FA0709F404C0E530A0E03C
:10F0D800FA0749F4A9E01A9FF001E950F74FDF0158
:10F0E800EC91EF78EC931F5FC0CF10E01C3048F430
:10F0F800A7E6B9E0EE27A10FBE1F0E94A2CC1F5FB2
:10F10800F5CF199108950E9491CA3A2F373310F01C
:10F118003C3308F064C000E010E0103108F05DC036
:10F12800A9E01A9FF001E650F74FA0813A1709F0BD
:10F1380052C0A9E01A9FF001E950F74FE081F0E0D2
:10F148000E941BCBE770F070309761F41A9FF001B2
:10F15800E950F74FE081E07811F0003009F001C084
:10F1680005E039C0E230A0E0FA0721F0E330A0E082
:10F17800FA07B9F4A9E01A9FF001E950F74FE081C6
:10F18800E47011F002E00CC0A9E01A9FF001E95008
:10F19800F74FE081E07811F0003009F001C005E098
:10F1A8001AC0E130A0E0FA0751F4A9E01A9FF00173
:10F1B800E950F74FE081E07809F001E00CC0E43055
:10F1C800A0E0FA0711F4E4E0CAC1E530A0E0FA07CC
:10F1D80011F4E3E0C4C11F5FA0CFE02FC0C1E32F4B
:10F1E800EF501E2F103108F046C0A9E01A9FF00119
:10F1F800E950F74FE081F0E00E941BCBE770F07018
:10F20800309751F41A9FF001E950F74FE081E07808
:10F2180011F0E5E0A4C1A2C1E230A0E0FA0721F0B4
:10F22800E330A0E0FA07A9F4A9E01A9FF001E95039
:10F23800F74FE081E47011F0E2E091C1A9E01A9F74
:10F24800F001E950F74FE081E07811F0E5E087C17F
:10F2580085C1E130A0E0FA0711F4E1E080C1E430B3
:10F26800A0E0FA0711F4E4E07AC1E530A0E0FA077B
:10F2780011F4E3E074C172C167971A93FE013896DE
:10F28800FA93EA93E0E0EA93A0E1B0E00E948EC32B
:10F29800FE013196FA93EA93E0E0EA93A7E0B0E042
:10F2A8000E948EC3EAE0EC83EF8310E0103108F08F
:10F2B80058C0E12FFF2766277727E053FF4F6F4F8E
:10F2C8006BBFE691E03039F4ED81FE81E070F07EAD
:10F2D800E062F36006C0ED81FE81E070F07EE46FCD
:10F2E800F160ED83FE83A5E4B1E0E12FF0E0BD011C
:10F2F800A7E0B0E00E9444CBE60FF71FFA93EA9329
:10F30800FE013396FA93EA93A7E00E940426FE01D1
:10F318003896FA93EA93E6E3F7E060E070E00E943B
:10F3280018CCE12FF0E031966F2F660F660B762F21
:10F338000E9418CC84E00E94DBC92A96E12FF0E0F5
:10F34800A0E1B8E30E9409CBEA0FFB1FFA93EA9306
:10F35800FE013A96FA93EA930E94B428A8951F5F93
:10F36800A5CF0E947B6018810C94F87E1A930A93AB
:10F3780010E0103108F0B1C0E12FF0E0309711F43F
:10F38800E5B166C0E130A0E0FA0719F4E2B1E17036
:10F3980060C0E230A0E0FA0719F4E5B1E07459C0A2
:10F3A800E330A0E0FA0719F4E4B3E27052C0E430A5
:10F3B800A0E0FA0719F4EEB1E8704BC0E530A0E020
:10F3C800FA0719F4E4B3E47044C0E630A0E0FA07A1
:10F3D80019F4E4B3E1703DC0E730A0E0FA0719F48E
:10F3E800EBB1E07836C0E830A0E0FA0719F4E5B1EF
:10F3F800E0782FC0E930A0E0FA0719F4E2B1E8702C
:10F4080028C0EA30A0E0FA0719F4EEB1E07121C093
:10F41800EB30A0E0FA0719F4E2B1E0711AC0EC3061
:10F42800A0E0FA0711F4EEB113C0ED30A0E0FA073E
:10F4380019F4E1B3E0710DC0EE30A0E0FA0719F459
:10F44800E5B1E07106C0EF30A0E0FA0719F4E1B3C6
:10F45800E0720E2FE0E4F7E060E070E00E9418CC64
:10F46800E12FF0E031966F2F660F660B762F0E9422
:10F4780018CCA9E01A9FF001E950F74FE081E29516
:10F48800E770FF27662777270E9418CC1A9FF0019C
:10F49800E950F74FE081E170FF27662777270E9440
:10F4A80018CC013010F0E1E301C0E0E3FF27662744
:10F4B80077270E9418CCA9E01A9FF001E250F74F75
:10F4C800DF01ED91FD91662777270E9418CC84E132
:10F4D8000E9416CA68961F5F4CCF0991199108952A
:10F4E8001A9310E0153080F4E12FF0E0E957F64F59
:10F4F8000F01A5EBB1E0EE27A10FBE1F0E9486CC3D
:10F50800D001EC931F5FEECF0C9442810E9491CA08
:10F518003A2F10E0103110F5A9E01A9FF001E650DB
:10F52800F74FA0813A17C1F4A9E01A9FF001E950FA
:10F53800F74FE081E295E7700E2F1A9FF001E9502E
:10F54800F74FE081E47031F4013021F0043011F01C
:10F55800053011F4E1E003C01F5FDCCFE0E00E945A
:10F5680098CA2496089560971A93FE013196FA93E3
:10F57800EA93E0E0EA93A2E0B0E00E948EC310E0D4
:10F58800153080F5A5EBB1E0EE27A10FBE1F0E9454
:10F59800A2CCFE013196FA93EA93E0E6F7E060E048
:10F5A80070E00E9418CCE12FF0E031966F2F660FC3
:10F5B800660B762F0E9418CC84E00E94DBC92A963D
:10F5C800E12FF0E0A0E1B9E30E9409CBEA0FFB1FAD
:10F5D800FA93EA93FE013396FA93EA930E94B428C9
:10F5E8001F5FCECF18816196089562970E948FCAD7
:10F5F800A6E2B1E00E9486CCE07109F4F3C3A5E26B
:10F60800B1E00E9486CC0E2FA6E2B1E00E9486CC23
:10F61800EF70ED8B00FF04C0E0919307E170F1F407
:10F6280001FF04C0E0919407E170C1F402FF04C037
:10F63800E0919507E17091F403FF04C0E09196070B
:10F64800E17061F4AD89A53040F0ED89F0E03197C3
:10F65800ED56F84FE081E17009F412C0A2E3B1E081
:10F668000E9482CCFF70A4E8BDE0FF700F01ED910D
:10F67800FD91E070F07FE029F129FE93EE93B2C38B
:10F68800A1E3B1E00E9486CCEE83E030C1F0AE8108
:10F698000E947A3BE03091F0A2E3B1E00E9482CC74
:10F6A800FF70A4E8BDE0FF700F01ED91FD91E070DF
:10F6B800F07FE029F129FE93EE9394C31BC0E091FB
:10F6C800CF03E27021F0A091CE03A13008F412C05C
:10F6D800A2E3B1E00E9482CCFF70A4E8BDE0FF7015
:10F6E8000F01ED91FD91E070F07FE029F129FE9383
:10F6F800EE9378C3E091840DF091850DFF7000249E
:10F708000E160F0640F4A4E8BDE080E0EFEFFFE03E
:10F718000E9476CC67C3A6E2B1E00E9486CCE2954F
:10F72800EF70E695E170EB8BE03021F0A091CD0A07
:10F73800A13008F401C056C3E0E0E093900D0E94A8
:10F74800E06A0E94D835A6E00E944C27A1E00E94FA
:10F75800C7B8E0E7F7E060E070E00E9418CC80E00E
:10F768000E9416CA249616981598E0E0E093E508DA
:10F77800E460E093E508E064E093E5082898EDB5D7
:10F78800E093820DE0E4EEBDEDB5E7FFFDCFEAE0E2
:10F79800EEBDEDB5E7FFFDCFE091E508EEBDEDB5B7
:10F7A800E7FFFDCF289A07FF3FC0E2B1E67EE2B946
:10F7B800E5B1EF70E5B95F98EEB1E77CEEB9E1B37A
:10F7C800EF7CE1BBE4B3E87FE4BBE0E0E093E7086B
:10F7D800E093E9082898EDB5E093820DE2E4EEBDE8
:10F7E800EDB5E7FFFDCFEAE0EEBDEDB5E7FFFDCFF4
:10F7F800E091E708EEBDEDB5E7FFFDCF289A289820
:10F80800EDB5E093820DE4E4EEBDEDB5E7FFFDCF85
:10F81800EAE0EEBDEDB5E7FFFDCFE091E908EEBD0A
:10F82800EDB5E7FFFDCF289AE0E0E98BEA8B00FF12
:10F838000FC0E0919307EC7021F452E0E1E0EA8B0D
:10F8480006C0E0919307EC70E43009F451E001C080
:10F8580050E001FF0FC0E0919407EC7021F442E002
:10F86800E1E0EA8B06C0E0919407EC70E43009F41B
:10F8780041E001C040E002FF11C0E0919507EC7043
:10F8880029F4E2E0EF8BE1E0E98B07C0E09195070E
:10F89800EC70E43011F4E1E0EF8B02C0E0E0EF8BB4
:10F8A80003FF11C0E0919607EC7029F4E2E0EE8BBB
:10F8B800E1E0E98B07C0E0919607EC70E43011F4C1
:10F8C800E1E0EE8B02C0E0E0EE8BE0E0EC8BAD898E
:10F8D800A530E8F0ED89E1501E2FFF27662777272E
:10F8E800EC56FF4F6F4F6BBFE691E150E8B9E12F3F
:10F8F800F0E0ED56F84FE081EC70E43029F4ED8942
:10F90800EC8BE0E0ED8B02C0E1E0EA8B02C0EFE3B4
:10F91800E8B9E0E0EF87EE87ED87EC87EB8739E120
:10F9280020E0E093B80DEF83EA87A6E2B1E00E94F9
:10F9380086CCE295EF70E695E695E170E88BA4E356
:10F94800B1E00E9486CCE887E987E0E0E093D80040
:10F95800ECBDA4E1B0E00E945ACEE0E0E093C10023
:10F96800E093C2000E942838E1E0E0936900E0E0FB
:10F97800E4BD0E94F780E0E0E0938000E09385001A
:10F98800E0938400E8E1E0938900E9E6E0938800E9
:10F99800E2E0E6BBE0936F00E0E0E0937A00F894E1
:10F9A800E0E8E0936100E6E0E09361007894EAE043
:10F9B800E0938100E1E8ECBBE1E0E3BF8895A8951E
:10F9C800E091B80DAF81EA0FEF83E0E0E093B80D66
:10F9D800AF81A53088F0EF81E550EF83A4EFB0E167
:10F9E800ED91FD916D917D91EF5FFF4F6F4F7F4FCF
:10F9F8007E936E93FE93EE93E0E0EA87513089F4AC
:10FA0800669B03C0E0E0EF870CC0E889E03039F47A
:10FA1800AF85A23020F4EF85EF5FEF8702C0E1E009
:10FA2800EA87413089F4679B03C0E0E0EE870CC0A9
:10FA3800E889E03039F4AE85A23020F4EE85EF5F36
:10FA4800EE8702C0E2E0EA87AF89A13089F4799BAA
:10FA58000DC0E889E03039F4AD85A23020F4ED8599
:10FA6800EF5FED8702C0E3E0EA8702C0E0E0ED87E0
:10FA7800AE89A13089F47A9B0DC0E889E03039F469
:10FA8800AC85A23020F4EC85EF5FEC8702C0E4E09F
:10FA9800EA8702C0E0E0EC87EC89E03089F0359B2A
:10FAA80003C0E0E0EB870CC0E889E03039F4AB85AF
:10FAB800A23020F4EB85EF5FEB8702C0E5E0EA8730
:10FAC800EA89E03019F4E989E030D1F0E0E5ECBDED
:10FAD800E1E0EDBDEA89E03009F0169AE989E03005
:10FAE80009F0159AAD89A03019F4AC89A03029F035
:10FAF80088E592E00197F1F703C085E88A95F1F768
:10FB0800523089F4669B0DC0E889E03039F4AF853E
:10FB1800A23020F4EF85EF5FEF8702C0E1E0EA87CB
:10FB280002C0E0E0EF87423089F4679B0DC0E889A6
:10FB3800E03039F4AE85A23020F4EE85EF5FEE8731
:10FB480002C0E2E0EA8702C0E0E0EE87AF89A230B7
:10FB580089F4799B03C0E0E0ED870CC0E889E030C8
:10FB680039F4AD85A23020F4ED85EF5FED8702C052
:10FB7800E3E0EA87AE89A23089F47A9B03C0E0E02B
:10FB8800EC870CC0E889E03039F4AC85A23020F469
:10FB9800EC85EF5FEC8702C0E4E0EA87AD89A1302D
:10FBA80088F0359B0DC0E889E03039F4AB85A23088
:10FBB80020F4EB85EF5FEB8702C0E5E0EA8702C03F
:10FBC800E0E0EB87EA89E03009F01698E989E0304F
:10FBD80009F01598313018F131502030F9F020E053
:10FBE800E091E508ED7FE093E508E0E5ECBDE1E0B4
:10FBF800EDBD2898EDB5E093820DE0E4EEBDEDB5DE
:10FC0800E7FFFDCFEAE0EEBDEDB5E7FFFDCFE09100
:10FC1800E508EEBDEDB5E7FFFDCF289A20C031E33A
:10FC280021E0E091E508E260E093E508E0E5ECBD5D
:10FC3800E1E0EDBD2898EDB5E093820DE0E4EEBD7E
:10FC4800EDB5E7FFFDCFEAE0EEBDEDB5E7FFFDCF8F
:10FC5800E091E508EEBDEDB5E7FFFDCF289AE0E0BD
:10FC6800ECBDE091CF03E27029F0E09902C0489919
:10FC780001C001C002C0E6E0EA87609902C0E7E07F
:10FC8800EA87EA85E03049F0A985A13020F0E985C6
:10FC9800E150E98701C004C002C0E885E9878CCE3D
:10FCA800F894E0E8E0936100E0E0E0936100789484
:10FCB800EDBBE0938100E0936F00E1E5ECBDE1E08E
:10FCC800EDBD719AE6E0E093C200E8E9E093C10077
:10FCD800E0E0E093C500E3E0E093C400EDE0E4BDBC
:10FCE800E0E0E093900DACE6B2E00E9482CCDF0148
:10FCF8000E94D204A0E00E942D370E94A63A07FF76
:10FD080002C00E947B607ED0A2E3B1E00E9482CC58
:10FD1800FF70A4E8BDE0FF700F01ED91FD91E07068
:10FD2800F07FE029F129FE93EE93AA85A73099F494
:10FD3800E091840DF091850DFF703A9758F4E091A9
:10FD4800840DF091850DE070F07FEA60E093840DFA
:10FD5800F093850D12C0E091840DF091850DFF7030
:10FD6800359758F4E091840DF091850DE070F07F9F
:10FD7800E560E093840DF093850DE0E0E093880D55
:10FD8800EBE7F7E060E070E00E9418CCEE85FF2713
:10FD9800662777270E9418CC84E00E9416CA289606
:10FDA800A0E00E94C7B8A7E00E944C270E94DF3558
:10FDB800E889E03029F0AA85A13010F0A53008F0D4
:10FDC80011C0EA85E150EA87AA85B0E0AD56B84F80
:10FDD800EC91E160EC93AA85B0E0AD56B84FEC9198
:10FDE800E06FEC930E9496CA68960895EA93EFB77D
:10FDF800EA93E091B80DEF5FE093B80DE991EFBF9A
:10FE0800E991189522970E948FCA20E050E030E0CF
:10FE1800EAD1ECE8F9E0FA93EA93E0E0EA93AEE39A
:10FE2800B0E00E948EC310E0173008F0F7C0E12F51
:10FE3800FF2766277727EA52FE4F6F4F6BBF469121
:10FE4800A5E4B1E0E42FF0E0BD01A7E0B0E00E9436
:10FE580044CBDB01AE0FBF1F0E9486CCE73B09F005
:10FE6800DBC0A2E9B9E0E12FF0E00E940BCBAE0FB6
:10FE7800BF1FEC91E160EC93113028F0143010F4BE
:10FE880021E001C051E0ABE3B7E0E12FF0E0BD01B4
:10FE9800A2E2B0E00E9444CBDB01AE0FBF1F0E947C
:10FEA80086CCE03059F0A2E9B9E0E12FF0E00E94F9
:10FEB8000BCBAE0FBF1FEC91E260EC93ABE3B7E066
:10FEC800E12FF0E0BD01A2E2B0E00E9444CBDB01EB
:10FED800AE0FBF1F11960E9486CCE03059F0A2E900
:10FEE800B9E0E12FF0E00E940BCBAE0FBF1FEC9101
:10FEF800E460EC93ABE3B7E0E12FF0E0BD01A2E2F0
:10FF0800B0E00E9444CBDB01AE0FBF1F12960E94E7
:10FF180086CCE03059F0A2E9B9E0E12FF0E00E9488
:10FF28000BCBAE0FBF1FEC91E860EC93ABE3B7E0EF
:10FF3800E12FF0E0BD01A2E2B0E00E9444CBDB017A
:10FF4800AE0FBF1F13960E9486CCE03059F0A2E98D
:10FF5800B9E0E12FF0E00E940BCBAE0FBF1FEC9190
:10FF6800E061EC93ABE3B7E0E12FF0E0BD01A2E282
:10FF7800B0E00E9444CBDB01AE0FBF1F14960E9475
:10FF880086CCE03059F0A2E9B9E0E12FF0E00E9418
:10FF98000BCBAE0FBF1FEC91E062EC93ABE3B7E085
:10FFA800E12FF0E0BD01A2E2B0E00E9444CBDB010A
:10FFB800AE0FBF1F18960E947ECC309760407040ED
:10FFC80061F031E0A2E9B9E0E12FF0E00E940BCB4B
:10FFD800AE0FBF1FEC91E064EC93ABE3B7E0E12F09
:10FFE800F0E0BD01A2E2B0E00E9444CBDB01AE0F1D
:08FFF800BF1F53960E947ECC4E
:020000021000EC
:0800000030976040704061F090
:1000080031E0A2E9B9E0E12FF0E00E940BCBAE0F9E
:10001800BF1FEC91E068EC931F5F06CFE32FE17000
:10002800EE0F0E2EE0918C09ED7FE029E0938C090C
:10003800E0919209E17021F4203011F4503029F058
:10004800E0918C09E160E0938C09E0919209E170FC
:10005800A1F1A6E3B7E00E9486CCF0E0309711F456
:10006800E7E629C0E130A0E0FA0711F4EFE623C083
:10007800E230A0E0FA0711F4E6E61DC0E330A0E0A4
:10008800FA0711F4E5E617C0E430A0E0FA0711F426
:10009800E4E611C0E530A0E0FA0711F4E3E60BC08E
:1000A800E630A0E0FA0711F4EBE605C0E730A0E07F
:1000B800FA0719F4E2E6E0938D09203009F446C006
:1000C800A7E3B7E00E9482CCEE83FF83AE81BF81B5
:1000D800AA3FE0E0BE0760F001E0EE81FF816627FD
:1000E8007727A0E0B4E284EF90E00E94A2CB1BC087
:1000F800AE81BF81939760F002E0EE81FF816627B1
:100108007727A0E8B4E88EE190E00E94A2CB0BC06C
:1001180003E0EE81FF8166277727A0E9B0ED83E051
:1001280090E00E94C6CBEE83FF83E0938E09F093A4
:100138008F09EF81E0938700EE81E0938600E2E08B
:10014800E0938000E02FE85EE0938100503009F4EE
:1001580046C0A9E3B7E00E9482CCEE83FF83AE815C
:10016800BF81AA3FE0E0BE0760F001E0EE81FF81B9
:1001780066277727A0E0B4E284EF90E00E94A2CB44
:100188001BC0AE81BF81939760F002E0EE81FF81D2
:1001980066277727A0E8B4E88EE190E00E94A2CB1A
:1001A8000BC003E0EE81FF8166277727A0E9B0ED59
:1001B80083E090E00E94C6CBEE83FF83E093900932
:1001C800F0939109EF81E0939700EE81E093960018
:1001D800E2E0E0939000E02FE85EE09391000E9457
:1001E80096CA289608951A93E0E0E093B000E0914B
:1001F8008000E370E0938000E0919000E370E0936A
:10020800900010E01730C0F4A2E9B9E0E12FF0E067
:100218000E940BCBAE0FBF1F1196E0E0EC93A2E952
:10022800B9E0E12FF0E00E940BCBAE0FBF1FEC91BD
:10023800ED7FEC931F5FE6CF10E01031F8F4A9E0F2
:100248001A9FF001E650F74FA081A73BA9F4A9E057
:100258001A9FF001E950F74FDF01EC91EE7FEC9324
:10026800A9E01A9FF001E950F74FDF01EC91EF7810
:10027800EC93A12F0E94045F1F5FDFCF19910895AF
:100288001A930A930A2FE02FFF2766277727E05251
:10029800FF4F6F4F6BBF1691183308F0CCC0A2E91F
:1002A800B9E0E12FF0E00E940BCBAE0FBF1F119613
:1002B800E0E0EC93E12FF0E03097B1F4E0E0E09378
:1002C800B000E0919209E47069F0ACE3B7E00E94F5
:1002D80086CCAE2F0E947A3BE03011F02C9A01C0F8
:1002E8002C9801C02C98A7C0E130A0E0FA07C1F40F
:1002F800E0918000EF73E0938000E0919A09E47048
:1003080069F0AEE5B7E00E9486CCAE2F0E947A3B3A
:10031800E03011F02D9A01C02D9801C02D988BC0A6
:10032800E230A0E0FA07C1F4E0918000EF7CE093AE
:100338008000E091A209E47069F0A0E8B7E00E94AB
:1003480086CCAE2F0E947A3BE03011F02E9A01C085
:100358002E9801C02E986FC0E330A0E0FA07C1F4D0
:10036800E0918000E37FE0938000E091AA09E470C7
:1003780069F0A2EAB7E00E9486CCAE2F0E947A3BD1
:10038800E03011F02F9A01C02F9801C02F9853C068
:10039800E430A0E0FA07C1F4E0919000EF73E09335
:1003A8009000E091B209E47069F0A4ECB7E00E9413
:1003B80086CCAE2F0E947A3BE03011F0739A01C0D0
:1003C800739801C0739837C0E530A0E0FA07C1F40C
:1003D800E0919000EF7CE0939000E091BA09E4701E
:1003E80069F0A6EEB7E00E9486CCAE2F0E947A3B59
:1003F800E03011F0749A01C0749801C074981BC061
:10040800E630A0E0FA07B9F4E0919000E37FE093CA
:100418009000E091C209E47069F0A8E0B8E00E9499
:1004280086CCAE2F0E947A3BE03011F0759A01C05D
:10043800759801C07598099119910895BA93AA936E
:1004480026970E948FCAE0918C09E17021F0E09113
:100458008C09E27009F4CCC1AC85BD85EC91E295BC
:10046800E1703E2F303041F011960E9401CCEE83AE
:10047800FF836887798708C0AC85BD851196ED91A3
:10048800FC911197EA87FB8710E0173008F0B0C19C
:10049800A2E9B9E0E12FF0E00E940BCBAE0FBF1F3D
:1004A800EC91E17009F4A2C1A2E9B9E0E12FF0E012
:1004B8000E940BCBAE0FBF1FEC91E07409F4C5C0CE
:1004C8003030B1F0ABE3B7E0E12FF0E0BD01A2E2DC
:1004D800B0E00E9444CBDB01AE0FBF1F18960E940C
:1004E8007ECCAE81BF81888599850E943CCB13C0A4
:1004F800ABE3B7E0E12FF0E0BD01A2E2B0E00E947B
:1005080044CBDB01AE0FBF1F18960E9482CCAA8590
:10051800BB850E942ACB2E2F203009F496C0ABE36E
:10052800B7E0E12FF0E0BD01A2E2B0E00E9444CBC9
:10053800DB01AE0FBF1F1C960E9486CCEF700E2FFA
:10054800013010F0083008F046C0AC85BD8515961E
:10055800E02FF0E03197AE0FBF1F4C915527542F75
:100568004427ABE3B7E0E12FF0E0BD01A2E2B0E041
:100578000E9444CBDB01AE0FBF1F1C960E9486CCA5
:10058800E295EF700E2F013010F0083008F022C00D
:10059800AC85BD851596E02FF0E03197AE0FBF1FF3
:1005A800EC91F0E04E2B5F2BA2E9B9E0E12FF0E0EF
:1005B8000E940BCBEA0FFB1F43835483A2E9B9E0E7
:1005C800E12FF0E00E940BCBAE0FBF1F1296E09117
:1005D8005E04EC933AC0ABE3B7E0E12FF0E0BD0175
:1005E800A2E2B0E00E9444CBDB01AE0FBF1F1C9615
:1005F8000E9486CCE295EF700E2F013010F0083083
:1006080008F023C0A2E9B9E0E12FF0E00E940BCB8B
:10061800EA0FFB1F33960F01AC85BD851596E02FB9
:10062800F0E03197AE0FBF1FEC91D001F0E0ED93F1
:10063800FC93A2E9B9E0E12FF0E00E940BCBAE0FEA
:10064800BF1F1296E0915E04EC93A2E9B9E0E12F96
:10065800F0E00E940BCBAE0FBF1FEC91E07809F4DD
:10066800C5C03030B1F0ABE3B7E0E12FF0E0BD0139
:10067800A2E2B0E00E9444CBDB01AE0FBF1F53964D
:100688000E947ECCAE81BF81888599850E943CCB33
:1006980013C0ABE3B7E0E12FF0E0BD01A2E2B0E0A8
:1006A8000E9444CBDB01AE0FBF1F53960E9482CC41
:1006B800AA85BB850E942ACB2E2F203009F496C02C
:1006C800ABE3B7E0E12FF0E0BD01A2E2B0E00E94A9
:1006D80044CBDB01AE0FBF1F57960E9486CCEF704C
:1006E8000E2F013010F0083008F046C0AC85BD85EB
:1006F8001596E02FF0E03197AE0FBF1F4C915527AC
:10070800542F4427ABE3B7E0E12FF0E0BD01A2E2AC
:10071800B0E00E9444CBDB01AE0FBF1F57960E948A
:1007280086CCE295EF700E2F013010F0083008F0FB
:1007380022C0AC85BD851596E02FF0E03197AE0F4D
:10074800BF1FEC91F0E04E2B5F2BA2E9B9E0E12F3F
:10075800F0E00E940BCBEA0FFB1F46835783A2E908
:10076800B9E0E12FF0E00E940BCBAE0FBF1F15964A
:10077800E0915E04EC933AC0ABE3B7E0E12FF0E020
:10078800BD01A2E2B0E00E9444CBDB01AE0FBF1F67
:1007980057960E9486CCE295EF700E2F013010F02C
:1007A800083008F023C0A2E9B9E0E12FF0E00E9488
:1007B8000BCBEA0FFB1F36960F01AC85BD8515964E
:1007C800E02FF0E03197AE0FBF1FEC91D001F0E0C1
:1007D800ED93FC93A2E9B9E0E12FF0E00E940BCB86
:1007E800AE0FBF1F1596E0915E04EC931F5F4DCED0
:1007F8000E9496CA2E96089563970E948FCAE09128
:100808008C09E17029F0E091EE08E770E13021F4FD
:100818000E9496CA69960895A7E2B1E00E9486CC24
:10082800E03011F4E0E007C0A7E2B1E00E9486CC16
:10083800AE2F0E947A3BEB8BA8E2B1E00E9486CCF7
:10084800E03011F4E0E007C0A8E2B1E00E9486CCF5
:10085800AE2F0E947A3BEA8BA0E023FCA1E0E1E006
:10086800EA27E894EE2309F0689423F810E017309B
:1008780010F00C944E8EA2E9B9E0E12FF0E00E944E
:100888000BCBAE0FBF1FEC91E17011F40C944B8EA3
:10089800E12FFF2766277727EA52FE4F6F4F6BBF7E
:1008A80006900C8AEC89A9E0EA9FF001E950F74F1D
:1008B800E081E295E770E98BA2E9B9E0E12FF0E089
:1008C8000E940BCBAE0FBF1FEC91E270A1F0ABE31F
:1008D800B7E0E12FF0E0BD01A2E2B0E00E9444CB16
:1008E800DB01AE0FBF1F0E9486CCAE2F0E947A3B61
:1008F800E03009F442C0EB89E03089F0A5E4B1E0CA
:10090800EC89F0E0BD01A7E0B0E00E9444CBDB0138
:10091800AE0FBF1F12960E9486CCE07151F5EA898E
:10092800E03089F0A5E4B1E0EC89F0E0BD01A7E092
:10093800B0E00E9444CBDB01AE0FBF1F12960E94AD
:1009480086CCE072B1F4E091F408E03089F0A5E4D7
:10095800B1E0EC89F0E0BD01A7E0B0E00E9444CB33
:10096800DB01AE0FBF1F12960E9486CCE07409F41B
:1009780002C030E001C031E001C030E050E030306A
:1009880009F451C4A2E9B9E0E12FF0E00E940BCBD1
:10099800AE0FBF1FEC91E87009F4BDC0ABE3B7E040
:1009A800E12FF0E0BD01A2E2B0E00E9444CBDB0100
:1009B800AE0FBF1F12960E9486CCE88BA889A83B71
:1009C80009F053C0E0917508F091760834960E94BA
:1009D8001DCB0E2FA6ECB1E00E9486CCEE8BA7ECC7
:1009E800B1E00E9486CCED8BAE89A017E8F50E1712
:1009F80058F5A02FBB27EE89F0E0AE1BBF0BAE87E2
:100A0800BF87ABE3B7E0E12FF0E0BD01A2E2B0E0C1
:100A18000E9444CBDB01AE0FBF1F15960E9486CC07
:100A2800F0E0AE85BF850E9444CBEE87FF87AD8995
:100A3800BB27EE89F0E00E9428CCEA1BFB0BAE85B1
:100A4800BF850E948ACB0FC0ABE3B7E0E12FF0E08F
:100A5800BD01A2E2B0E00E9444CBDB01AE0FBF1F94
:100A680015960E9486CC5E0F56C0A889A93B09F04E
:100A780052C0E0917708F091780834960E941DCB17
:100A88000E2FAAECB1E00E9486CCEE8BABECB1E065
:100A98000E9486CCED8BAE89A017E8F50E1758F5A5
:100AA800A02FBB27EE89F0E0AE1BBF0BAE87BF8738
:100AB800ABE3B7E0E12FF0E0BD01A2E2B0E00E94B5
:100AC80044CBDB01AE0FBF1F15960E9486CCF0E029
:100AD800AE85BF850E9444CBEE87FF87AD89BB27D3
:100AE800EE89F0E00E9428CCEA1BFB0BAE85BF859F
:100AF8000E948ACB0FC0ABE3B7E0E12FF0E0BD0165
:100B0800A2E2B0E00E9444CBDB01AE0FBF1F1596F6
:100B18000E9486CC5E0FA2E9B9E0E12FF0E00E94C6
:100B28000BCBAE0FBF1FEC91E07109F4C0C0ABE373
:100B3800B7E0E12FF0E0BD01A2E2B0E00E9444CBB3
:100B4800DB01AE0FBF1F13960E9486CCE88BA889E5
:100B5800A83B09F053C0E0917508F09176083496E7
:100B68000E941DCB0E2FA6ECB1E00E9486CCEE8B26
:100B7800A7ECB1E00E9486CCED8BAE89A017E8F512
:100B88000E1758F5A02FBB27EE89F0E0AE1BBF0B60
:100B9800AE87BF87ABE3B7E0E12FF0E0BD01A2E28B
:100BA800B0E00E9444CBDB01AE0FBF1F16960E9437
:100BB80086CCF0E0AE85BF850E9444CBEE87FF87E8
:100BC800AD89BB27EE89F0E00E9428CCEA1BFB0B1D
:100BD800AE85BF850E948ACB0FC0ABE3B7E0E12F9B
:100BE800F0E0BD01A2E2B0E00E9444CBDB01AE0F11
:100BF800BF1F16960E9486CC5E0F56C0A889A93BD7
:100C080009F052C0E0917708F091780834960E9474
:100C18001DCB0E2FAAECB1E00E9486CCEE8BABEC7C
:100C2800B1E00E9486CCED8BAE89A017E8F50E17CF
:100C380058F5A02FBB27EE89F0E0AE1BBF0BAE879F
:100C4800BF87ABE3B7E0E12FF0E0BD01A2E2B0E07F
:100C58000E9444CBDB01AE0FBF1F16960E9486CCC4
:100C6800F0E0AE85BF850E9444CBEE87FF87AD8953
:100C7800BB27EE89F0E00E9428CCEA1BFB0BAE856F
:100C8800BF850E948ACB0FC0ABE3B7E0E12FF0E04D
:100C9800BD01A2E2B0E00E9444CBDB01AE0FBF1F52
:100CA80016960E9486CC5E0F553608F054E6A2E9E7
:100CB800B9E0E12FF0E00E940BCBAE0FBF1FEC9123
:100CC800E07209F4C0C0ABE3B7E0E12FF0E0BD018A
:100CD800A2E2B0E00E9444CBDB01AE0FBF1F149626
:100CE8000E9486CCE88BA889A83B09F053C0E09104
:100CF8007508F091760834960E941DCB0E2FA6EC4D
:100D0800B1E00E9486CCEE8BA7ECB1E00E9486CCC5
:100D1800ED8BAE89A017E8F50E1758F5A02FBB2765
:100D2800EE89F0E0AE1BBF0BAE87BF87ABE3B7E041
:100D3800E12FF0E0BD01A2E2B0E00E9444CBDB016C
:100D4800AE0FBF1F17960E9486CCF0E0AE85BF8518
:100D58000E9444CBEE87FF87AD89BB27EE89F0E080
:100D68000E9428CCEA1BFB0BAE85BF850E948ACB6C
:100D78000FC0ABE3B7E0E12FF0E0BD01A2E2B0E0C5
:100D88000E9444CBDB01AE0FBF1F17960E9486CC92
:100D98005E0F56C0A889A93B09F052C0E0917708B8
:100DA800F091780834960E941DCB0E2FAAECB1E082
:100DB8000E9486CCEE8BABECB1E00E9486CCED8B2A
:100DC800AE89A017E8F50E1758F5A02FBB27EE89B6
:100DD800F0E0AE1BBF0BAE87BF87ABE3B7E0E12FF8
:100DE800F0E0BD01A2E2B0E00E9444CBDB01AE0F0F
:100DF800BF1F17960E9486CCF0E0AE85BF850E9483
:100E080044CBEE87FF87AD89BB27EE89F0E00E94CF
:100E180028CCEA1BFB0BAE85BF850E948ACB0FC08E
:100E2800ABE3B7E0E12FF0E0BD01A2E2B0E00E9441
:100E380044CBDB01AE0FBF1F17960E9486CC5E0F16
:100E4800553608F054E6A2E9B9E0E12FF0E00E9437
:100E58000BCBAE0FBF1FEC91E07461F0A2E9B9E0D3
:100E6800E12FF0E00E940BCBAE0FBF1F1296AC91A2
:100E7800A13008F483C0A2E9B9E0E12FF0E00E94B4
:100E88000BCBAE0FBF1F1296EC91E150EC93A2E989
:100E9800B9E0E12FF0E00E940BCBAE0FBF1F129616
:100EA800EC91E03071F4A2E9B9E0E12FF0E00E94A2
:100EB8000BCBAE0FBF1F1396E0E0F0E0ED93FC9371
:100EC8005DC0A2E9B9E0E12FF0E00E940BCBAE0FC4
:100ED800BF1F1396ED91FD91FF93EF93ABE3B7E03E
:100EE800E12FF0E0BD01A2E2B0E00E9444CBDB01BB
:100EF800AE0FBF1F1D960E9482CCAF91BF91EA230F
:100F0800FB23EE87FF87ABE3B7E0E12FF0E0BD01FD
:100F1800A2E2B0E00E9444CBDB01AE0FBF1F1F96D8
:100F28000E947ECCDF01CB01EE85FF8566277727FF
:100F38000E941FCD0E94A8CDEE83FF836887798722
:100F4800AE81BF8188859985E0E0F0E068EC72E4C5
:100F58000E943ACE09F008F401C00FC0EE81FF816B
:100F680068857985A0E0B0E080E09FE30E9459CDD4
:100F78000E94E6CC5E0F553608F054E6A2E9B9E0C7
:100F8800E12FF0E00E940BCBAE0FBF1FEC91E07891
:100F980061F0A2E9B9E0E12FF0E00E940BCBAE0FBF
:100FA800BF1F1596AC91A13008F483C0A2E9B9E03F
:100FB800E12FF0E00E940BCBAE0FBF1F1596EC910E
:100FC800E150EC93A2E9B9E0E12FF0E00E940BCBED
:100FD800AE0FBF1F1596EC91E03071F4A2E9B9E0AD
:100FE800E12FF0E00E940BCBAE0FBF1F1696E0E09A
:100FF800F0E0ED93FC935DC0A2E9B9E0E12FF0E0E9
:101008000E940BCBAE0FBF1F1696ED91FD91FF937B
:10101800EF93ABE3B7E0E12FF0E0BD01A2E2B0E06F
:101028000E9444CBDB01AE0FBF1F58960E9482CCB2
:10103800AF91BF91EA23FB23EE87FF87ABE3B7E0CD
:10104800E12FF0E0BD01A2E2B0E00E9444CBDB0159
:10105800AE0FBF1F5A960E947ECCDF01CB01EE85F2
:10106800FF85662777270E941FCD0E94A8CDEE83B3
:10107800FF8368877987AE81BF8188859985E0E09D
:10108800F0E068EC72E40E943ACE09F008F401C07E
:101098000FC0EE81FF8168857985A0E0B0E080E02F
:1010A8009FE30E9459CD0E94E6CC5E0F553608F0AA
:1010B80054E6A2E9B9E0E12FF0E00E940BCBAE0FB5
:1010C800BF1FEC91E072A1F0ABE3B7E0E12FF0E0D5
:1010D800BD01A2E2B0E00E9444CBDB01AE0FBF1F0E
:1010E80014960E9486CCAE2F0E947A3BE03009F419
:1010F8000EC0ABE3B7E0E12FF0E0BD01A2E2B0E043
:101108000E9444CBDB01AE0FBF1F17965BC0A2E95C
:10111800B9E0E12FF0E00E940BCBAE0FBF1FEC91BE
:10112800E071A1F0ABE3B7E0E12FF0E0BD01A2E28E
:10113800B0E00E9444CBDB01AE0FBF1F13960E94A4
:1011480086CCAE2F0E947A3BE03009F40EC0ABE3A8
:10115800B7E0E12FF0E0BD01A2E2B0E00E9444CB8D
:10116800DB01AE0FBF1F16962DC0A2E9B9E0E12F33
:10117800F0E00E940BCBAE0FBF1FEC91E870A1F01E
:10118800ABE3B7E0E12FF0E0BD01A2E2B0E00E94DE
:1011980044CBDB01AE0FBF1F12960E9486CCAE2F48
:1011A8000E947A3BE03009F410C0ABE3B7E0E12FCE
:1011B800F0E0BD01A2E2B0E00E9444CBDB01AE0F3B
:1011C800BF1F15960E9486CC5E2F533608F054E652
:1011D800ABE3B7E0E12FF0E0BD01A2E2B0E00E948E
:1011E80044CBDB01AE0FBF1F5E960E9486CC4E2F0C
:1011F800ABE3B7E0E12FF0E0BD01A2E2B0E00E946E
:1012080044CBDB01AE0FBF1F5F960E9486CCE88FF0
:10121800513010F0541708F002C0542F04C0E88D64
:101228005E1708F0588D303041F0513030F0A98900
:10123800A03011F0A13009F401C01FC0A2E9B9E043
:10124800E12FF0E00E940BCBAE0FBF1F1196E0E03C
:10125800EC93EC89A9E0EA9FF001E550F74FA0E094
:10126800A083EC89A9E0EA9FF001E750F74FDF017E
:10127800EC91E07FEC93E2E0E98B550FA989A2306D
:1012880019F0A33009F0EDC0A2E9B9E0E12FF0E0D0
:101298000E940BCBAE0FBF1F11962C91251708F09B
:1012A8006DC0ABE3B7E0E12FF0E0BD01A2E2B0E032
:1012B8000E9444CBDB01AE0FBF1F90960E9486CCE4
:1012C800EF8BAF89A13008F458C0AF3190F123FEFD
:1012D80018C0EF89F0E0A0E9B1E00E949DCB0E2F85
:1012E800023008F00150A22FBB27EE27A00FBE1F27
:1012F800E52FF0E0AE17BF071CF4E02FE20F5E2FDA
:1013080017C0AF89ECE3EA17E1E008F4EE270E2EE8
:10131800E22FF0E03296DF01E52FF0E00E9430CBBB
:10132800E02119F0E22FEE5F02C0E22FEF5F5E2F9F
:1013380024C0EF89F0E0A8ECB0E00E949DCB0E2F0E
:10134800023370F4A22FBB27EE27A00FBE1FE52F94
:10135800F0E0AE17BF071CF4E02FE20F5E2F0DC0C0
:10136800A22FBB27EE27A00FBE1FE52FF0E0AE1778
:10137800BF0718F4E02FE20F5E2F70C0521708F075
:101388006DC0ABE3B7E0E12FF0E0BD01A2E2B0E051
:101398000E9444CBDB01AE0FBF1F91960E9486CC02
:1013A800EF8BAF89A13008F459C0AF3190F123FE1B
:1013B80019C0EF89F0E0A0E9B1E00E949DCB0E2FA3
:1013C800023008F00150A52FBB27E02FF0E0EA0F0C
:1013D800FB1FA22FB0E0EA17FB071CF4E22FE01B6B
:1013E8005E2F16C0AF89ECE3EA17E1E008F4EE27B8
:1013F8000E2EE52FF0E03296A22FB0E00E9436CBF9
:10140800E02119F0E22FE25002C0E22FE1505E2FF6
:1014180025C0EF89F0E0A8ECB0E00E949DCB0E2F2C
:10142800023370F4A52FBB27F0E0EA0FFB1FA22FB1
:10143800B0E0EA17FB071CF4E22FE01B5E2F0EC09A
:10144800A52FBB27E02FF0E0EA0FFB1FA22FB0E08B
:10145800EA17FB0718F4E22FE01B5E2F593C08F04F
:1014680058ECA2E9B9E0E12FF0E00E940BCBEA0FBB
:10147800FB1F5183503009F430E0303029F4A9893A
:10148800A03011F0A13009F416C0EC89A9E0EA9F58
:10149800F001E750F74FDF01EC91E07FEC93EC8926
:1014A800A9E0EA9FF001E950F74FDF01EC91EB7FEB
:1014B800EC93E0E0E98BA989A43011F0A53009F498
:1014C80050E0E12FF0E0309709F054C05030B1F40B
:1014D800E0E0E093B000E0919209E47069F0ACE3D9
:1014E800B7E00E9486CCAE2F0E947A3BE03011F024
:1014F8002C9A01C02C9801C02C983BC0573CB0F0E6
:10150800E0E0E093B000E0919209E47069F0ACE3A8
:10151800B7E00E9486CCAE2F0E947A3BE03011F0F3
:101528002C9801C02C9A01C02C9A23C0E0919209F2
:10153800E47091F0ACE3B7E00E9486CCAE2F0E9435
:101548007A3BE03021F0E0918D09E06102C0E09142
:101558008D09E093B00004C0E0918D09E093B000DC
:10156800F52FE0E0DF01E8ECF0E00E948ACBE093A1
:10157800B3002FC3E130A0E0FA0709F083C0503070
:10158800C1F4E0918000EF73E0938000E0919A0944
:10159800E47069F0AEE5B7E00E9486CCAE2F0E94F9
:1015A8007A3BE03011F02D9A01C02D9801C02D989A
:1015B80068C0583CC0F0E0918000EF73E093800071
:1015C800E0919A09E47069F0AEE5B7E00E9486CC34
:1015D800AE2F0E947A3BE03011F02D9801C02D9A71
:1015E80001C02D9A4EC0E0918E09F0918F096627AF
:1015F8007727EA87FB876C877D87E52FF0E0AA8548
:10160800BB858C859D856F2F660F660B762F0E9494
:101618004CCBEA87FB876C877D87AA85BB858C8541
:101628009D85E8ECF0E060E070E00E94A2CBEE87D8
:10163800FF87E0918E09F0918F09AE85BF85EA1783
:10164800FB0710F4EE87FF87EF85E0938900EE85AE
:10165800E0938800E0918000E068E0938000AEE5C8
:10166800B7E00E9486CCAE2F0E947A3BE03021F092
:10167800E0918000E06403C0E0918000EB7FE0939C
:101688008000A7C2E230A0E0FA0709F083C050301A
:10169800C1F4E0918000EF7CE0938000E091A20922
:1016A800E47069F0A0E8B7E00E9486CCAE2F0E94F3
:1016B8007A3BE03011F02E9A01C02E9801C02E9886
:1016C80068C0583CC0F0E0918000EF7CE093800057
:1016D800E091A209E47069F0A0E8B7E00E9486CC26
:1016E800AE2F0E947A3BE03011F02E9801C02E9A5E
:1016F80001C02E9A4EC0E0918E09F0918F0966279D
:101708007727EA87FB876C877D87E52FF0E0AA8536
:10171800BB858C859D856F2F660F660B762F0E9483
:101728004CCBEA87FB876C877D87AA85BB858C8530
:101738009D85E8ECF0E060E070E00E94A2CBEE87C7
:10174800FF87E0918E09F0918F09AE85BF85EA1772
:10175800FB0710F4EE87FF87EF85E0938B00EE859B
:10176800E0938A00E0918000E062E0938000A0E8C6
:10177800B7E00E9486CCAE2F0E947A3BE03021F081
:10178800E0918000E06103C0E0918000EF7EE0938B
:1017980080001FC2E330A0E0FA0709F083C0503090
:1017A800C1F4E0918000E37FE0938000E091AA0912
:1017B800E47069F0A2EAB7E00E9486CCAE2F0E94DE
:1017C8007A3BE03011F02F9A01C02F9801C02F9872
:1017D80068C0583CC0F0E0918000E37FE09380004F
:1017E800E091AA09E47069F0A2EAB7E00E9486CC09
:1017F800AE2F0E947A3BE03011F02F9801C02F9A4B
:1018080001C02F9A4EC0E0918E09F0918F0966278A
:101818007727EA87FB876C877D87E52FF0E0AA8525
:10182800BB858C859D856F2F660F660B762F0E9472
:101838004CCBEA87FB876C877D87AA85BB858C851F
:101848009D85E8ECF0E060E070E00E94A2CBEE87B6
:10185800FF87E0918E09F0918F09AE85BF85EA1761
:10186800FB0710F4EE87FF87EF85E0938D00EE8588
:10187800E0938C00E0918000E860E0938000A2EAA9
:10188800B7E00E9486CCAE2F0E947A3BE03021F070
:10189800E0918000E46003C0E0918000EB7FE0937A
:1018A800800097C1E430A0E0FA0709F083C0503007
:1018B800C1F4E0919000EF73E0939000E091B209D9
:1018C800E47069F0A4ECB7E00E9486CCAE2F0E94C9
:1018D8007A3BE03011F0739A01C0739801C0739895
:1018E80068C0583CC0F0E0919000EF73E09390001E
:1018F800E091B209E47069F0A4ECB7E00E9486CCEC
:10190800AE2F0E947A3BE03011F0739801C0739AB1
:1019180001C0739A4EC0E0919009F0919109662731
:101928007727EA87FB876C877D87E52FF0E0AA8514
:10193800BB858C859D856F2F660F660B762F0E9461
:101948004CCBEA87FB876C877D87AA85BB858C850E
:101958009D85E8ECF0E060E070E00E94A2CBEE87A5
:10196800FF87E0919009F0919109AE85BF85EA174C
:10197800FB0710F4EE87FF87EF85E0939900EE856B
:10198800E0939800E0919000E068E0939000A4EC68
:10199800B7E00E9486CCAE2F0E947A3BE03021F05F
:1019A800E0919000E06403C0E0919000EF7BE09349
:1019B80090000FC1E530A0E0FA0709F083C050306D
:1019C800C1F4E0919000EF7CE0939000E091BA09B7
:1019D800E47069F0A6EEB7E00E9486CCAE2F0E94B4
:1019E8007A3BE03011F0749A01C0749801C0749881
:1019F80068C0583CC0F0E0919000EF7CE093900004
:101A0800E091BA09E47069F0A6EEB7E00E9486CCCE
:101A1800AE2F0E947A3BE03011F0749801C0749A9E
:101A280001C0749A4EC0E0919009F091910966271F
:101A38007727EA87FB876C877D87E52FF0E0AA8503
:101A4800BB858C859D856F2F660F660B762F0E9450
:101A58004CCBEA87FB876C877D87AA85BB858C85FD
:101A68009D85E8ECF0E060E070E00E94A2CBEE8794
:101A7800FF87E0919009F0919109AE85BF85EA173B
:101A8800FB0710F4EE87FF87EF85E0939B00EE8558
:101A9800E0939A00E0919000E062E0939000A6EE57
:101AA800B7E00E9486CCAE2F0E947A3BE03021F04E
:101AB800E0919000E06103C0E0919000EF7EE09338
:101AC800900087C0E630A0E0FA0709F082C05030E5
:101AD800C1F4E0919000E37FE0939000E091C209A7
:101AE800E47069F0A8E0B8E00E9486CCAE2F0E94AE
:101AF8007A3BE03011F0759A01C0759801C075986D
:101B080068C0583CC0F0E0919000E37FE0939000FB
:101B1800E091C209E47069F0A8E0B8E00E9486CCC0
:101B2800AE2F0E947A3BE03011F0759801C0759A8B
:101B380001C0759A4EC0E0919009F091910966270D
:101B48007727EA87FB876C877D87E52FF0E0AA85F2
:101B5800BB858C859D856F2F660F660B762F0E943F
:101B68004CCBEA87FB876C877D87AA85BB858C85EC
:101B78009D85E8ECF0E060E070E00E94A2CBEE8783
:101B8800FF87E0919009F0919109AE85BF85EA172A
:101B9800FB0710F4EE87FF87EF85E0939D00EE8545
:101BA800E0939C00E0919000E860E0939000A8E04A
:101BB800B8E00E9486CCAE2F0E947A3BE03021F03C
:101BC800E0919000E46003C0E0919000EB7FE09327
:101BD8009000E091EF08E770E23068F0EC89A9E046
:101BE800EA9FF001E950F74FE081E295E770AE2FE8
